:100000000C94AC170C94E5170C94E5170C94E517B9
:100010000C94A9440C94A9440C94A9440C94A944AC
:100020000C94E5170C94E5170C94E5170C94E51760
:100030000C94E5170C94432C0C94E5170C94E517DD
:100040000C94E5170C94AA280C948AD20C94E5170A
:100050000C944A8F0C94408F0C94E5170C94E51780
:100060000C94E5170C94E5170C94E5170C94E51720
:100070000C94E5170C94E5170C94E5170C94E51710
:100080000C94B3830C94E5170C94E5174E414E493C
:100090004E495459494E46CDCCCC3D0AD7233C1746
:1000A000B7D13877CC2B329595E6241FB14F0A0093
:1000B0000020410000C84200401C4620BCBE4CCA83
:1000C0001B0E5AAEC59D7400407A10F35A00A07200
:1000D0004E18090010A5D4E80000E8764817000083
:1000E000E40B54020000CA9A3B000000E1F5050051
:1000F0000080969800000040420F000000A086019A
:10010000000000102700000000E803000000006469
:1001100000000000000A00000000000100000000D4
:10012000002C76D888DC674F0823DFC1DFAE59E1A9
:10013000B1B796E5E3E453C63AE651997696E8E618
:10014000C28426EB898C9B62ED407C6FFCEFBC9CEB
:100150009F40F2BAA56FA5F490055A2AF75C936BFD
:100160006CF9676DC11BFCE0E40D47FEF520E6B5B8
:1001700000D0ED902E0300943577050080841E0892
:100180000000204E0A000000C80C333333330F98B0
:100190006E12831141EF8D2114893BE65516CFFE77
:1001A000E6DB18D1844B381BF77C1D901DA4BBE403
:1001B00024203284725E228100C9F124ECA1E53D45
:1001C000275045544700504C41005072696E7420CE
:1001D00041626F72746564004D3235005061757311
:1001E000696E672E2E2E004D323400454550524F19
:1001F0004D2056657273696F6E204572726F720082
:10020000454550524F4D20496E64657820457272C5
:100210006F7200454550524F4D2043524320457266
:10022000726F72003F0049676E6F726500526573AE
:10023000657400496E697469616C697A6520454529
:1002400050524F4D0000FE0003FF8007C7C007015A
:10025000E00000E00000F00000700400700E00708C
:100260001F00703F80F00E00E00F01E007C7C003E1
:10027000FF8000FE0000FE0003FF8007C7C00F01E3
:10028000E00E00E03F80F01F00700E007004007070
:100290000000700000F00000E00701E007C7C003A5
:1002A000FF8000FE000E000E000E000E000E000E7D
:1002B000000E000E007FC03F801F000E00040004EF
:1002C000000E001F003F807FC00E000E000E000ECB
:1002D000000E000E000E000E00FFFFFF7F80FFC02B
:1002E000FFC0FFC07F807F80FFC0FFC0FFC03F0016
:1002F0001E000C0050726F6265205A204F666673B4
:1003000065740020082046616374002008204D6158
:1003100078002008204D696E004F6666004F6E0021
:100320004175746F74656D700045207374657073EA
:100330002F6D6D005A2053746570732F6D6D0059C9
:100340002053746570732F6D6D0058205374657061
:10035000732F6D6D00416476616E63656420536533
:100360007474696E67730054656D7065726174753D
:1003700072650053746570732F6D6D00436F6E6608
:10038000696775726174696F6E003F004E657874BD
:1003900020436F726E657200446F6E65004E657823
:1003A0007400486F6D696E672058595A0053746F16
:1003B00072652053657474696E6773004C6F616475
:1003C0002053657474696E677300426564205472CB
:1003D000616D6D696E670050726F6265205A204FC3
:1003E0006666736574004661646520486569676880
:1003F00074004F6666004F6E00426564204C65765F
:10040000656C696E67004C6576656C2042656400BA
:100410004732394E00473239004175746F20486FBA
:100420006D65004D6F74696F6E0053572D4D6F648D
:10043000650053746F77004465706C6F7900536585
:100440006C662D5465737400526573657400436F58
:100450006E66696775726174696F6E005265737458
:100460006F72652044656661756C7473004C6F61D2
:10047000642053657474696E67730053746F72659A
:100480002053657474696E677300424C546F7563D2
:10049000680050726F6265205A204F6666736574FB
:1004A00000416476616E6365642053657474696E9F
:1004B0006773004D61696E003F004261636B0053DA
:1004C000746F70004D323200417474616368204D66
:1004D00065646961004D3231005072696E74206646
:1004E000726F6D204D656469610052656C65617362
:1004F00065204D6564696100436F6E66696775725A
:100500006174696F6E0054656D70657261747572A7
:1005100065004D6F74696F6E00526573756D65206F
:100520005072696E740054756E650053746F70205C
:100530005072696E74005061757365205072696EF7
:100540007400496E666F2053637265656E000A4DD4
:100550003234004D3233202573003F0053746172F2
:1005600074205072696E740043616E63656C005054
:1005700072696E740043616E6E6F7420656E74658F
:1005800072207375626469723A200002202E2E0078
:100590000152656672657368004D61696E002100E5
:1005A000486F74656E6420746F6F20636F6C6400B5
:1005B0004261636B0050726F63656564004D6F74D8
:1005C000696F6E0044697361626C65205374657075
:1005D00070657273004D383400426564204C657656
:1005E000656C696E67004175746F20486F6D6500BA
:1005F000473238004D61696E0050726568656174FC
:10060000202420426564005072656865617420246E
:1006100020456E640054656D706572617475726515
:1006200000C601C101436F6F6C646F776E0050723A
:10063000656865617420240046616E2053706565AD
:100640006400426564004E6F7A7A6C65004D6169A2
:100650006E0050726F6265205A204F666673657433
:1006600000466C6F770046616E20537065656400CC
:10067000426564004E6F7A7A6C65005370656564FC
:10068000004D61696E00486F6D696E672046616953
:100690006C6564006F70656E00545249474745525F
:1006A0004544003A20007A5F70726F6265007A5F9D
:1006B0006D696E00795F6D696E00785F6D696E00BF
:1006C0005265706F7274696E6720656E6473746FC3
:1006D00070207374617475730A0020746F6F206CDE
:1006E0006F6E6720657874727573696F6E207072B3
:1006F0006576656E7465640A0020636F6C642065BE
:100700007874727573696F6E2070726576656E7439
:1007100065640A00486F6D65202573257325732075
:100720004669727374005761726E696E673A204849
:100730006F6D696E672042756D70204469766973CC
:100740006F72203C20310A000202040000E0C00069
:100750000000C00000000000006843000063430088
:10076000007A430000A0400000A04000000040FFCD
:10077000FDFCFAF8F6F4F2F0EEECEAE9E7E5E3E185
:10078000E0DEDCDAD9D7D5D4D2D0CFCDCBCAC8C73A
:10079000C5C3C2C0BFBDBCBAB9B7B6B4B3B2B0AFBF
:1007A000ADACAAA9A8A6A5A4A2A1A09E9D9C9A9919
:1007B000989795949392908F8E8D8B8A898887864F
:1007C00084838281807F7E7D7B7A79787776757469
:1007D000737271706F6E6D6C6B6A69686766656461
:1007E000636261605F5E5D5C5B5A5958585756554D
:1007F0005453525150504F4E4D4C4B4A4A49484722
:100800004646454443424241403F3E3E3D3C3B3BE1
:100810003A39383837363535343332323130302F93
:100820002E2E2D2C2B2B2A29292827272625252437
:10083000232322212120201F1E1E1D1C1C1B1B1ACE
:100840001919181817161615151413131212111159
:10085000100F0F0E0E0D0D0C0C0B0A0A09090808DB
:100860000707060605050404030302020100000051
:1008700000000100000001000080005555550000F7
:1008800000400033333300AAAA2A00499224000012
:10089000002000C7711C0099991900D14517005517
:1008A0005515003BB113002449120011111100002D
:1008B0000010000F0F0F00E3380E0043790D00CC3D
:1008C000CC0C00C3300C00E8A20B0064210B00AA82
:1008D000AA0A00703D0A009DD80900427B090092D7
:1008E000240900DCD30800888808001042080000B2
:1008F000000800F0C10700878707007550070071E6
:100900001C07003EEB0600A1BC06006990060066CD
:10091000660600703E06006118060017F4050074B4
:10092000D105005BB00500B290050062720500556C
:1009300055050078390500B81E0500050505004E6F
:10094000EC040087D40400A1BD040090A704004972
:10095000920400C17D0400EE690400C756040044FF
:100960004404005C3204000821040041100400002B
:100970000004003FF00300F8E0030026D20300C3A8
:10098000C30300CCB503003AA803000A9B03003858
:100990008E0300C08103009F750300D069030050DF
:1009A0005E03001D53030034480300913D030033F0
:1009B00033030016290300381F0300971503003086
:1009C0000C0300030303000BFA020049F10200BA12
:1009D000E802005CE002002DD802002DD002005990
:1009E000C80200B0C0020031B90200DAB10200AAA8
:1009F000AA0200A0A30200BC9C0200FA9502005CBF
:100A00008F0200DF88020082820200457C020027FC
:100A100076020027700200436A02007C640200D064
:100A20005E02003F590200C853020000006143000B
:100A300000614300007A430000E0C0000000C000F5
:100A400000000053657474696E67732053746F728D
:100A50006564000000FA430000FA430000A0400073
:100A600000C8410000A0420000A0420000C84300AE
:100A700080C043F4010000F401000064000000881D
:100A800013000024F4D43050C38E20C2A240178239
:100A90008B7011127A910D816CD90AA861E108C797
:100AA000586607615143061E4B5D05C145A7041AF0
:100AB000411104093D9803713931034036DB026569
:100AC000339102D4305402802E1D02632CEE017546
:100AD0002AC501B028A001102781018F2564012BB0
:100AE000244B01E0223401AC211F018D200D018037
:100AF0001FFC00841EED00971DDF00B81CD200E62D
:100B00001BC600201BBC00641AB200B219A8000A60
:100B100019A0006A189900D117910040178B00B5F1
:100B200016840031167E00B31579003A157300C79C
:100B3000146F0058146A00EE1366008813630025D2
:100B4000135E00C7125B006C12570015125400C1EF
:100B500011510070114F0021114B00D61049008D2A
:100B60001047004610440002104200C00F400080B1
:100B70000F3E00420F3C00060F3B00CB0E380093A7
:100B80000E37005C0E3500270E3400F30D3200C125
:100B90000D3100900D3000600D2E00320D2D00053E
:100BA0000D2C00D90C2B00AE0C2900850C29005C03
:100BB0000C2700350C27000E0C2600E80B2400C47F
:100BC0000B2400A00B23007D0B23005A0B210039BE
:100BD0000B2100180B2000F80A1F00D90A1E00BBC9
:100BE0000A1E009D0A1D00800A1D00630A1C0047A2
:100BF0000A1B002C0A1B00110A1A00F7091A00DD53
:100C0000091900C4091900AB091900920917007BE2
:100C1000091800630917004C091600360916002050
:100C20000916000A091500F5081500E0081400CCA3
:100C3000081400B8081400A4081400900813007DDC
:100C40000812006B081300580812004608120034FE
:100C5000081100230811001208110001081100F00A
:100C6000071000E0071000D0071000C0071000B008
:100C7000070F00A107100091070E0083070F0074F3
:100C8000070F0065070E0057070E0049070E003BCF
:100C9000070D002E070E0020070D0013070D00069C
:100CA000070D00F9060C00ED060D00E0060C00D45F
:100CB000060C00C8060C00BC060C00B0060C00A414
:100CC000060B0099060C008D060B0082060B0077C0
:100CD000060B006C060B0061060A0057060B004C61
:100CE000060A0042060A0038060A002E060A0024F8
:100CF000060A001A060A001006090007060A00FD87
:100D0000050900F4050900EB050900E2050900D911
:100D1000050900D0050900C7050900BE050900B591
:100D2000050800AD050800A50509009C050800940C
:100D30000508008C050800840508007C050800747F
:100D40000508006C050700650508005D05070056ED
:100D50000508004E05070047050700400508003854
:100D6000050700310507002A050700230507001CB9
:100D7000050600160507000F050700080506000216
:100D8000050700FB040600F5040700EE040600E872
:100D9000040600E2040700DB040600D5040600CFC9
:100DA000040600C9040600C3040600BD040600B71B
:100DB000040600B1040500AC040600A6040600A069
:100DC0000405009B04060095040500900406008AB3
:100DD00004050085040500800406007A04050075FA
:100DE000040500700405006B04050066040500613D
:100DF0000405005C04050057040500520405004D7D
:100E000004050048040500430405003E0404003ABC
:100E100004050035040500300404002C04050027F7
:100E2000040400230405001E0404001A0404001630
:100E3000040500110404000D040400090405000465
:100E400004040000040400FC030400F8030400F49C
:100E5000030400F0030400EC030400E8030400E4CE
:100E6000030400E0030400DC030400D8030400D4FE
:100E7000030400D0030400CC030400C8030300C52E
:100E800003030024F404D9201BC40C5C0E9804C492
:100E9000095F0265077101F405F900FB04B300481E
:100EA000048700C10369005803550003034500BED1
:100EB000023A008402310053022A0029022500046C
:100EC000022000E4011C00C8011900AF01170098BE
:100ED0000114008401130071011000610110005120
:100EE000010E0043010D0036010B002B010B002009
:100EF000010B00150109000C01090003010800FBAA
:100F0000000800F3000800EB000700E4000600DE24
:100F1000000600D8000600D2000600CC000500C77D
:100F2000000500C2000500BD000400B9000400B5C2
:100F3000000400B1000400AD000400A9000400A5F5
:100F4000000300A20003009F0004009B0003009820
:100F50000003009500020093000300900003008D41
:100F60000002008B0003008800020086000200845B
:100F7000000300810002007F0002007D0002007B70
:100F80000002007900020077000100760002007480
:100F900000020072000100710002006F0002006D8B
:100FA0000001006C0002006A000100690002006795
:100FB000000100660001006500010064000200629B
:100FC00000010061000100600001005F0002005D9F
:100FD0000001005C0001005B0001005A00010059A3
:100FE00000010058000100570001005600010055A3
:100FF00000010054000100530000005300010052A2
:1010000000010051000100500001004F0001004E9E
:101010000000004E0001004D0001004C0001004B9B
:101020000000004B0001004A000100490001004897
:101030000000004800010047000100460000004693
:10104000000100450000004500010044000100438C
:101050000000004300010042000000420001004186
:1010600000000041000100400001003F0000003F7F
:101070000001003E0000003E0001003D0000003D78
:101080000001003C0000003C0000003C0001003B6F
:101090000000003B0001003A0000003A0001003966
:1010A000000000390001003800000038000000385E
:1010B0000001003700000037000100360000003654
:1010C000000000360001003500000035000000354A
:1010D000000100340000003400000034000100333F
:1010E0000000003300000033000100320000003235
:1010F000000000320001003100000031000000312A
:101100000001003000000030000000300001002F1E
:101110000000002F0000002F0000002F0001002E13
:101120000000002E0000002E0001002D0000002D08
:101130000000002D0000002D0001002C0000002CFC
:101140000000002C0000002C0001002B0000002BF0
:101150000000002B0000002B0001002A0000002AE4
:101160000000002A0000002A0001002900000029D8
:1011700000000029000000290000002900010028CB
:1011800000000028000000280000002800000028BF
:1011900000010027000000270000002700000027B2
:1011A00000000027000100260000002600000026A5
:1011B0000000002600000026000100250000002598
:1011C000000000250000002500000025000000258B
:1011D000000100240000002400000024000000247E
:1011E0000000002400010023000000230000002371
:1011F0000000002300000023000000230000002363
:101200000001002200000022000000220000002255
:101210000000002200000022000100210000002147
:10122000000000210000002100000021000000213A
:10123000000000210001002000000020000000202C
:10124000000000200000002000000020000000201E
:10125000000000200001001F0000001F0000001F10
:101260000000001F0000001F0000001F0000001F02
:101270000001001E0000001E0000001E0000001EF5
:10128000000000393000003325000087190000B04D
:101290000F0000DB080000BD040000740200003FE6
:1012A00001000020436F756E7420583A0042656457
:1012B000004531004500626564002C207379737429
:1012C000656D2073746F707065642120486561746A
:1012D00065725F49443A20004572723A204D415888
:1012E00054454D50004D415854454D50207472693D
:1012F0006767657265640048656174696E6720465A
:1013000061696C65640048656174696E6720666137
:10131000696C6564004572723A204D494E54454DE2
:1013200050004D494E54454D5020747269676765B1
:1013300072656400544845524D414C2052554E410F
:1013400057415900546865726D616C2052756E6129
:1013500077617900202F002042403A0020403A0077
:101360007C3C3E5E2B3D3F2F5B5D3B2C2A225C008C
:10137000434F4D4D554E49434154494F4E00445201
:101380005952554E004552524F525300494E464F06
:10139000004543484F0053544F505045442E2000C1
:1013A0005072696E7465722073746F70706564201A
:1013B00064756520746F206572726F72732E20469B
:1013C000697820746865206572726F7220616E643E
:1013D00020757365204D39393920746F207265731B
:1013E000746172742E202854656D70657261747515
:1013F00072652069732072657365742E205365745D
:1014000020697420616674657220726573746172FC
:1014100074696E67290A004E6F20436865636B73B9
:10142000756D2077697468206C696E65206E756DC6
:101430006265722C204C617374204C696E653A2091
:10144000004E6F20436865636B73756D2077697418
:1014500068206C696E65206E756D6265722C204C1B
:10146000617374204C696E653A2000636865636B34
:1014700073756D206D69736D617463682C204C61A8
:101480007374204C696E653A20004C696E65204E7D
:10149000756D626572206973206E6F74204C617384
:1014A00074204C696E65204E756D6265722B312C0F
:1014B000204C617374204C696E653A20004D3131C7
:1014C000300053657269616C2073746174757320A8
:1014D0006D69736D617463680A00534420726561BD
:1014E00064206572726F720A002121204B494C4CB6
:1014F0002063617573656420627920746F6F206D5D
:1015000075636820696E6163746976652074696DBE
:1015100065202D2063757272656E7420636F6D6D2A
:10152000616E643A20004D6564696120496E73659F
:101530007274656400627573793A207061757365C1
:101540006420666F7220696E7075740A006275732C
:10155000793A2070617573656420666F72207573C7
:1015600065720A00627573793A2070726F636573F1
:1015700073696E670A00506C65617365205265730C
:101580006574005052494E5445522048414C5445D0
:10159000440025533A202553004B494C4C45442EDA
:1015A00020005072696E7465722068616C746564A5
:1015B0002E206B696C6C28292063616C6C6564213A
:1015C0000A0053544F505045442E20005072696E0B
:1015D0007465722073746F70706564206475652023
:1015E000746F206572726F72732E20466978207452
:1015F0006865206572726F7220616E642075736514
:10160000204D39393920746F20726573746172749A
:101610002E202854656D706572617475726520693D
:10162000732072657365742E20536574206974206D
:1016300061667465722072657374617274696E6735
:10164000290A006563686F3A004572726F723A004A
:101650004F4646004F4E0042696C696E65617220CC
:101660004C6576656C696E6720477269643A0A005A
:1016700021212053544F502063616C6C65642062BB
:10168000656361757365206F6620424C546F7563A6
:1016900068206572726F72202D207265737461729A
:1016A000742077697468204D3939390A0021212066
:1016B00053544F502063616C6C65642062656361B4
:1016C000757365206F6620424C546F7563682065A2
:1016D00072726F72202D207265737461727420773C
:1016E000697468204D3939390A004F46460A004668
:1016F00061646520486569676874200042656420FC
:101700004C6576656C696E6720004661696C65643E
:1017100020746F20656E61626C6520426564204CA8
:101720006576656C696E670A00496E76616C6964FE
:10173000206D6573682E0A0050726F62696E6720B3
:10174000506F696E740025532025692F2569002E7E
:101750000A002F0050726F62696E67206D657368B2
:1017600020706F696E742000202844525952554EE3
:101770002900473239204175746F20426564204C3E
:101780006576656C696E67003F20284C2C522C46AC
:101790002C4229206F7574206F6620626F756E640D
:1017A000732E0A003F2856296572626F7365206C9C
:1017B0006576656C20696D706C61757369626C65C6
:1017C0002028302D34292E0A00426164205A2076C8
:1017D000616C75650A004E6F2062696C696E6561A7
:1017E0007220677269640A004732384C300020204A
:1017F0004D3230312058004D617820416363656C73
:1018000065726174696F6E2028756E6974732F73C9
:1018100032290020204D3230332058004D6178208D
:101820006665656472617465732028756E6974738A
:101830002F73290020520020204D323034205000D8
:10184000416363656C65726174696F6E2028756EA3
:101850006974732F7332292028503C7072696E743A
:101860002D616363656C3E20523C726574726163E6
:10187000742D616363656C3E20543C7472617665BF
:101880006C2D616363656C3E2900204A0020540082
:1018900020530020204D32303520420041647661D3
:1018A0006E6365642028423C6D696E5F7365676D89
:1018B000656E745F74696D655F75733E20533C6D32
:1018C000696E5F66656564726174653E20543C6D47
:1018D000696E5F74726176656C5F6665656472617E
:1018E00074653E204A3C6A756E635F6465763E2986
:1018F0000020440020490020204D3330312050008A
:10190000486F74656E6420504944002044002049AB
:101910000020204D3330342050004265642050496F
:1019200044002E0A00206E6F742064697361626C3B
:1019300065642E205368617265642077697468005D
:10194000203B204C6576656C696E67200020204D39
:101950003432302053004175746F20426564204C4E
:101960006576656C696E670020460020420020485D
:101970000020204D3134352053004D61746572696B
:10198000616C2068656174757020706172616D654D
:101990007465727300204A00202047323920572096
:1019A000490020204D3134392043203B20556E69B9
:1019B000747320696E2043656C736975730A0054F3
:1019C000656D706572617475726520556E697473AA
:1019D000002020473231203B004C696E6561722047
:1019E000556E6974730020496E76616C6964206578
:1019F000787472756465722000536C6565702E2E64
:101A00002E005A2050726F6265205061737420421C
:101A100065640A005A2050726F62652050617374C9
:101A20002042656400205A3A200020593A200042A2
:101A3000656420583A20004D65736820706F696EA8
:101A400074206F7574206F662072616E67650A007E
:101A5000436C69636B20746F20526573756D652EDE
:101A60002E2E00616C736F20656E61626C65642957
:101A70000A004E6F204D6F76652E004E6F206D650B
:101A80006469610A00456E642066696C65206C6952
:101A900073740A00426567696E2066696C65206C24
:101AA0006973740A00286E6F2066696C6529004EA0
:101AB0006F74205344207072696E74696E670A00F7
:101AC0005344207072696E74696E67206279746520
:101AD000200043757272656E742066696C653A20E9
:101AE000002E0A0044656C6574696F6E206661693A
:101AF0006C65642C2046696C653A200046696C650B
:101B00002064656C657465643A0025697300256915
:101B10006D20256973002569682025696D20256978
:101B20007300256964202569682025696D20256971
:101B30007300256979202569642025696820256955
:101B40006D20256973005072696E742074696D652B
:101B50003A20006F6B006F66660091138C1385133B
:101B60007E13701344454255473A004D31313220BF
:101B700053687574646F776E004D313133205300B4
:101B80004D656761205A65726F20322E30204F46B6
:101B9000462E00434F4E4649475F4558504F5254DA
:101BA000004D4541545041434B00434F4F4C45522B
:101BB0005F54454D504552415455524500434841AC
:101BC0004D4245525F54454D504552415455524542
:101BD00000424142595354455050494E47004152EA
:101BE0004353004D4F54494F4E5F4D4F44455300B2
:101BF000544845524D414C5F50524F54454354490F
:101C00004F4E00455854454E4445445F4D323000D8
:101C10004C4F4E475F46494C454E414D450041555E
:101C2000544F5245504F52545F53445F53544154A4
:101C300055530053445F575249544500524550454F
:101C40004154005344434152440050524F4D50546C
:101C50005F535550504F525400484F53545F4143C7
:101C600054494F4E5F434F4D4D414E445300454DF7
:101C7000455247454E43595F5041525345520043E8
:101C80004153455F4C494748545F42524947485485
:101C90004E45535300544F47474C455F4C494748C6
:101CA000545300534F4654574152455F504F574588
:101CB00052004255494C445F50455243454E5400F2
:101CC0004C4556454C494E475F44415441005A5F8C
:101CD00050524F42450052554E4F555400415554B5
:101CE0004F4C4556454C005052494E545F4A4F4266
:101CF0000050524F4752455353004155544F52459F
:101D0000504F52545F54454D50004155544F524529
:101D1000504F52545F504F5300564F4C554D455401
:101D200052494300454550524F4D0042494E4152A1
:101D3000595F46494C455F5452414E534645520007
:101D400053455249414C5F584F4E5F584F464600ED
:101D50004649524D574152455F4E414D453A4D61BE
:101D6000726C696E20322E302E392E332D6B6164E9
:101D7000312028446563203237203230323120311F
:101D8000333A34333A35312920534F555243455F66
:101D9000434F44455F55524C3A6769746875622EEB
:101DA000636F6D2F6B61642F4D61726C696E205093
:101DB000524F544F434F4C5F56455253494F4E3A42
:101DC000312E30204D414348494E455F54595045CE
:101DD0003A4D656761205A65726F20322E3020457A
:101DE000585452554445525F434F554E543A312052
:101DF000555549443A64626663636435352D6562BE
:101E000062612D343631352D616264372D313936BA
:101E10006161343338663330340A002F2F004D317E
:101E2000343520533C696E6465783E206F757420AC
:101E30006F662072616E67652028302D31290A0097
:101E40003F4A206F7574206F662072616E6765204F
:101E500028302E303120746F20302E33290A002094
:101E6000580020204D61783A2000200020204D6944
:101E70006E3A2000203B200020204D32313120538B
:101E80000046523A0020466C6F773A2000206F756A
:101E900074206F662072616E67650A005365727602
:101EA0006F20003A200020536572766F2000507238
:101EB0006F6265204F6666736574205A0050726FBA
:101EC0006265204F6666736574205A00646973000A
:101ED000656E0043290A0061626C656420286D69A3
:101EE0006E2074656D702000436F6C64206578749B
:101EF00072756465732061726520004D3432312043
:101F0000696E636F727265637420706172616D6572
:101F10007465722075736167650A004D657368208A
:101F2000706F696E74206F7574206F662072616EB9
:101F300067650A00454550524F4D204F4B0A002916
:101F40000A0020746F20003F5A206F7574206F665E
:101F50002072616E6765202800290A0020746F20B6
:101F6000003F59206F7574206F662072616E67653F
:101F700020282D00290A0020746F20003F58206F70
:101F80007574206F662072616E676520282D004D84
:101F9000383400446F6E65207072696E74696E67C4
:101FA0002066696C650A004D3737004D33310049B2
:101FB0006E76616C69642065787472756465720A06
:101FC000004361703A0020286D6D2900203B0020FD
:101FD000204D3835312058005A2D50726F626520DF
:101FE0004F666673657400436F6F6C696E672E2E63
:101FF0002E0048656174696E672E2E2E00453120D3
:1020000025530020573A0020573A00426564204388
:102010006F6F6C696E672E2E2E00426564204865D6
:102020006174696E672E2E2E0023646566696E6585
:102030002044454641554C545F00626564004B6442
:1020400020004B6920004B7020005049442041750E
:10205000746F74756E652066696E69736865642156
:102060002050757420746865206C617374204B7007
:102070002C204B6920616E64204B6420636F6E736B
:1020800074616E74732066726F6D2062656C6F7719
:1020900020696E746F20436F6E6669677572617434
:1020A000696F6E2E680A00504944204175746F7440
:1020B000756E65206661696C6564212074696D6563
:1020C0006F75740A00504944204175746F74756EC1
:1020D00065206661696C6564212054656D70657268
:1020E000617475726520746F6F20686967680A0093
:1020F000504944204379636C65730025532025695A
:102100002F256900204B643A2000204B693A2000BB
:10211000204B703A200020436C6173736963205038
:102120004944200A00204E6F206F76657273686FF5
:102130006F740A002054753A2000204B753A200035
:10214000206D61783A2000206D696E3A200020648D
:102150003A200020626961733A2000576169742057
:10216000666F7220686561742075702E2E2E005087
:102170004944204175746F74756E65207374617283
:10218000740A00504944204175746F74756E65205F
:102190006661696C6564212054656D706572617457
:1021A00075726520746F6F20686967680A0050490E
:1021B00044204175746F74756E6500504944204128
:1021C00075746F74756E65206661696C6564212035
:1021D000426164206865617465722069640A004523
:1021E00072723A207574663820666F6E74206E6F56
:1021F0007420696E697469616C697A65642E004542
:1022000072723A207574663820666F6E74206E6F35
:102210007420696E697469616C697A65642E004521
:1022200072723A207574663820666F6E74206E6F15
:102230007420696E697469616C697A65642E004204
:10224000656400456E636C6F737572650025687513
:102250003A25303268750025303268753A253032BB
:102260006875002530326875272530326875002082
:1022700020202020202000202020200065727200D5
:102280001FE02010201020101020102020102010FF
:1022900030300840048003001FE03FF03FF03FF083
:1022A0001FE01FE03FF03FF03FF00FC0078003004A
:1022B0003FFFF038007030FC3020FC1020781020F8
:1022C00030102C00D02E31D02F7BD02F7BD02E3150
:1022D000D02C00D020301020781020FC1030FC30A2
:1022E0003800703FFFF03FFFF03800703186302338
:1022F00087102787902F87D02F03D0203010207889
:10230000102078102030102F03D02F87D0278790EF
:102310002387103186303800703FFFF01FFFF81F11
:10232000FFF8041040020820020820041040082092
:10233000801041001041000820800410400000007F
:102340001FFFF81FFFF8001DC43F0000000C861996
:102350008000000D0E198000000F0B198000000D89
:102360009F198000000DD3998000001CFBFF000026
:10237000000000000000000000000000F380001FCB
:1023800080007700001980005B1CF6131DAE5B35E2
:10239000AB0635FB5B3DA70CBD9B4B30EB19B19BEE
:1023A000E39D8E9F9D8E0001E00000000001200053
:1023B00000000001E0000000000C0F00FE070225F5
:1023C00003BB017FFE08FE08FE050808060000406A
:1023D000F0C88888987810050808060000C0F888BA
:1023E00088888888F80505050600012030F8302027
:1023F0000508080600002070F820202020E00509CC
:10240000090600FF2070A8A8B88888702007050575
:10241000070001D86C366CD80509090600FFF8A83A
:102420008888888888A8F8050A0A0600FE20505087
:10243000505088A8A8887003030306000340A040FA
:10244000FFFFFFFFFFFFFFFFFFFFFFFFFFFFFFFF9C
:10245000FFFFFFFFFFFF0000000605FF0107070663
:10246000020080808080800080030303060105A0B5
:10247000A0A005060606000050F85050F8500509C7
:10248000090600FF2070A8A07028A8702005070783
:10249000060000C8C81020409898050707060000ED
:1024A00040A0A040A8906801030306020580808038
:1024B0000309090601FF204040808080404020033E
:1024C00009090601FF804040202020404080050788
:1024D0000706000020A8702070A82005050506004A
:1024E000012020F820200203030601FFC0408005E0
:1024F0000101060003F8020202060100C0C0050740
:10250000070600000810102040408005070706005D
:1025100000708898A8C8887003070706010040C0AB
:1025200040404040E0050707060000708808102082
:1025300040F8050707060000F80810300888700505
:10254000070706000010305090F810100507070626
:102550000000F880F00808887005070706000030C2
:102560004080F0888870050707060000F808101002
:102570002020200507070600007088887088887072
:1025800005070706000070888878081060020505B6
:10259000060100C0C000C0C00206060601FFC0C0A0
:1025A00000C0408003050506010120408040200551
:1025B0000303060002F800F8030505060101804048
:1025C00020408005070706000070881020200020AA
:1025D0000507070600007088B8A8B88070050707CF
:1025E000060000708888F8888888050707060000BC
:1025F000F04848704848F0050707060000708880DA
:1026000080808870050707060000F0484848484861
:10261000F0050707060000F88080F08080F80507C5
:1026200007060000F88080F080808005070706001C
:1026300000708880809888700507070600008888E9
:1026400088F8888888030707060100E0404040407A
:1026500040E00507070600003810101010906005D4
:1026600007070600008890A0C0A09088050707060D
:102670000000808080808080F805070706000088C1
:10268000D8A8888888880507070600008888C8A811
:1026900098888805070706000070888888888870F1
:1026A000050707060000F08888F08080800507078E
:1026B00006000070888888A8906805070706000053
:1026C000F08888F0A09088050707060000708880D1
:1026D00070088870050707060000F82020202020D9
:1026E0002005070706000088888888888870050705
:1026F00007060000888888885050200507070600D4
:102700000088888888A8A8500507070600008888E0
:102710005020508888050707060000888850202030
:102720002020050707060000F80810204080F80365
:1027300009090601FFE080808080808080E0050735
:102740000706000080404020101008030909060118
:10275000FFE020202020202020E0050303060005C4
:102760002050880501010600FEF803030306010559
:102770008040200505050600007008788878050768
:10278000070600008080F0888888F00505050600AF
:1027900000708080887005070706000008087888A8
:1027A0008888780505050600007088F080700507A8
:1027B00007060000304840E040404005070706009B
:1027C000FE708888887808700507070600008080FA
:1027D000F0888888880307070601004000C0404051
:1027E00040E00409090601FE10003010101010909E
:1027F0006005070706000080808890E09088030746
:1028000007060100C04040404040E00505050600C5
:1028100000D0A8A8A8A8050505060000B0C88888AB
:10282000880505050600007088888870050707067A
:1028300000FEF0888888F080800507070600FE7893
:10284000888888780808050505060000B0C88080DB
:102850008005050506000078807008F0050707066A
:1028600000002020F820202018050505060000881B
:102870008888986805050506000088888850200526
:1028800005050600008888A8A85005050506000073
:1028900088502050880507070600FE888888502049
:1028A0004080050505060000F8102040F8030909DE
:1028B0000601FF20404040804040402001090906B9
:1028C00002FF80808080808080808003090906016B
:1028D000FF80404040204040408005030306000246
:1028E00048A890FF43616E6E6F74206F70656E2014
:1028F00073756264697220005344206361726420BE
:102900006F6B0A006F70656E526F6F74206661693D
:102910006C65640A00766F6C756D652E696E6974FE
:10292000206661696C65640A004E6F205344206321
:102930006172640A002E0A006F70656E206661691C
:102940006C65642C2046696C653A200046696C65AC
:102950002073656C65637465640A002053697A6549
:102960003A200046696C65206F70656E65643A2098
:1029700000454E4420535542524F5554494E450A46
:10298000002220706F73002220706172656E743AAD
:102990002200535542524F5554494E452043414C15
:1029A0004C207461726765743A22005375626361EA
:1029B0006C6C204F766572666C6F77004578636546
:1029C00065646564206D617820535542524F5554BB
:1029D000494E452064657074683A00667265736894
:1029E00000646F696E67002066696C653A20004E6E
:1029F0006F77200057726974696E6720746F206664
:102A0000696C653A20006D61726C696E66772E6F35
:102A1000726700322E302E392E332D6B61643100F7
:102A20001FFFFFFFFFFFFF600000000001FF4000ED
:102A300000000000FF8000000000007F83CF000046
:102A40000C303F87FF80000C301F867980000C001F
:102A50000F8C30C7838C30E78C30CFC7CC31F38CF0
:102A600030DCECEC33B98C30D86C6C33198C30D052
:102A70006C0C33198C30D86C0C33198C30DC6C0E28
:102A80003B198C30CF7C079F198C30C77C038F1982
:102A900040000000000002600000000000061FFF70
:102AA000FFFFFFFFF870012C0190012701B0012208
:102AB00001C0011D01F00118011002130130020EC6
:102AC000016002090190020401C002FF000003FA44
:102AD000004003F5008003F000D003EB002004E683
:102AE000007004E100E004DC004005D700C005D21E
:102AF000004006CD00D006C8008007C3003008BEE5
:102B000000F008B900C009B400B00AAF00B00BAAC9
:102B100000D00CA500000EA000500F9B00C0109626
:102B2000005012910000148C00C0158700B017826D
:102B300000B0197D00D01B7800001E730040206E8D
:102B40000090226900F024640040275F0090295A19
:102B500000E02B5500102E500020304B0010324664
:102B600000E033410090353C0010373700703832B8
:102B700000A0392D00B03A2800A03B2300603C1E85
:102B800000103D1900903D1400103E0F00703E0AE9
:102B900000C03E0500003F0000403FFBFF803FF6C5
:102BA000FFC03FF1FF2020506C616E6E6572427570
:102BB0006666657242797465733A200020467265D4
:102BC00065204D656D6F72793A200020436F6D70FE
:102BD000696C65643A2044656320323720323032B4
:102BE000310A00204C61737420557064617465640F
:102BF0003A20323032312D30392D3033207C204193
:102C00007574686F723A20286B61642C20416E796C
:102C10006375626963204D656761205A65726F2034
:102C2000322E302041424C20323456290A004D6168
:102C3000726C696E20322E302E392E332D6B61640A
:102C4000310A0020536F6674776172652052657394
:102C500065740A00205761746368646F6720526569
:102C60007365740A002042726F776E206F7574204E
:102C700052657365740A002045787465726E616CE4
:102C80002052657365740A00506F77657255700A3B
:102C90000073746172740A004732385859004D311C
:102CA000303031006572726F722077726974696EAC
:102CB0006720746F2066696C650A00446F6E65203A
:102CC000736176696E672066696C652E0A004D3205
:102CD0003900456E6473746F70730025532025634B
:102CE0002025632025632025630020503A00205AC8
:102CF0003A0020593A0020583A00656E6473746FA8
:102D00007073206869743A20000000000102000915
:102D10000A00000000040308070000000000000093
:102D2000000000000000000000004D6F76652025C7
:102D3000736D6D004D6F766520302E316D6D004DD9
:102D40006F766520316D6D004D6F76652031306D89
:102D50006D004D6F76652041786973004D6F766523
:102D6000204578747275646572004D6F7665205ADF
:102D7000004D6F76652059004D6F766520580050E4
:102D800072696E742066726F6D204D6564696100B2
:102D9000FFFFFF205A3A200020593A200042656484
:102DA00020583A20004D656761205A65726F2032C5
:102DB0002E302052656164792E005072696E7469FC
:102DC0006E672E2E2E005072696E742050617573DE
:102DD000656400204500205A0020590020204D390C
:102DE0003220580053746570732070657220756EC0
:102DF0006974003B2000220A00556E6B6E6F776E7F
:102E000020636F6D6D616E643A2022006F6B00DB92
:102E10000FC93F45BCDA3F8FB30240FCF027405654
:102E2000946140FE4B9B4084A5D840E02318413478
:102E30006A5641E859974164DBD5416E271742B481
:102E4000B75542CE1A9742C8AED542B5885A43D438
:102E50000684BFA65FA7BF7443E0BF10B11AC01CB1
:102E60002C58C0E8F697C0B849D6C04E4E17C124BA
:102E7000D355C1802497C1A0B5D5C1121A17C24439
:102E8000AE55C2781797C26CACD5C267885AC320BA
:102E9000746F6F206C6F6E672065787472757369DC
:102EA0006F6E2070726576656E7465640A002063CB
:102EB0006F6C6420657874727573696F6E207072C0
:102EC0006576656E7465640A006F6B0A00526573FF
:102ED000656E643A200020453A00205A3A00205995
:102EE0003A00583A0000002200250028002B00007C
:102EF000002100240027002A00020202020202022E
:102F0000020404040404040404030303030303038A
:102F10000301010101010101010102040810204027
:102F200080010204081020408001020408102040A3
:102F30008080402010080402014572726F72207771
:102F4000726974696E6720746F20454550524F4D09
:102F5000210A0000A7DDCBE411241FBECFEFD0E48F
:102F6000DEBFCDBF84B780937A1514BE0FB6F89438
:102F7000A895809160008861809360001092600045
:102F80000FBE12E0A0E0B1E0E4ECF5EE01E00BBF13
:102F900002C007900D92A239B107D9F725E1A2E945
:102FA000B2E001C01D92AA37B207E1F717E1CBEA00
:102FB000D7E104C02197FE010E9430F0CA3AD10740
:102FC000C9F70E946DDE0C94D6F20C940000A0E1CB
:102FD000B0E0EDEEF7E10C9459F08C01DC01ED91DD
:102FE000FC910280F381E02DBE016F5F7F4F099558
:102FF000882309F45DC08981807C91F56F816370BD
:1030000070E0762F6627770F770F8885B4E08B9F67
:10301000C0011124682B792B898582958695869528
:103020008370682B6F5F7F4F90E080E02A8523706C
:10303000220F3B8537FB332730F9232B3E813F702E
:10304000230F3327331F2750310904C0660F771F22
:10305000881F991F2A95D2F76096E4E00C9475F0CA
:10306000803419F568856695669570E090E080E09B
:10307000CB01772766272A85622B098510E0102F60
:103080000027012E000C220B330B602B712B822B9F
:10309000932B6F5F7F4F8F4F9F4F4AE0660F771FD5
:1030A000881F991F4A95D1F7D7CF8BE0F801848309
:1030B00060E070E0CB01D0CF0895FC0182810895DB
:1030C0004F925F926F927F928F929F92AF92BF9238
:1030D000CF92DF92EF92FF92CF93DF93CDB7DEB71F
:1030E00028970FB6F894DEBF0FBECDBF60913407AE
:1030F000709135076115710511F18091300790913C
:103100003107A0913207B091330789839A83AB834B
:10311000BC83072E000C880B990B0E946BE9298158
:103120003A814B815C810E9482F04B015C0120E07E
:1031300030E040E251EC0E9465E987FF07C081E082
:1031400080933201C12CD12C760113C020E030E0F5
:1031500040E251E4C501B4010E94E6F1181604F5FD
:1031600081E080933201C12CD12C9FE7E92E93E4BA
:10317000F92EC701B60128960FB6F894DEBF0FBE30
:10318000CDBFDF91CF91FF90EF90DF90CF90BF90B8
:10319000AF909F908F907F906F905F904F90089529
:1031A00080913B0790913C07A0913D07B0913E076D
:1031B0008D839E83AF83B88780913201882391F0FD
:1031C0001092960410929704109298041092990409
:1031D0001092920410929304109294041092950409
:1031E00010923201209196043091970440919804F6
:1031F00050919904C501B4010E9483F02B013C0158
:1032000020E030E0A9010E94E6F1C12CD12C76012A
:1032100087FD14C02D813E814F81588560E070E0AC
:103220008FE793E40E94FAF06B017C01A301920105
:103230000E9465E9181614F473016201C0929604A5
:10324000D0929704E0929804F09299042091370765
:10325000309138074091390750913A07C501B401C0
:103260000E94CAE94B015C0180928A0490928B040F
:10327000A0928C04B0928D04A70196016D817E818D
:103280008F8198850E94CAE96B017C01C0928E04EF
:10329000D0928F04E0929004F092910440909204B6
:1032A00050909304609094047090950429813A8121
:1032B0004B815C81609186047091870480918804C1
:1032C000909189040E9482F020913F07309140073D
:1032D00040914107509142070E94CAE9A30192011F
:1032E0000E9482F020ED3CEC4CE45DE30E94CAE9D0
:1032F000A30192010E9483F09B01AC0120939204F0
:1033000030939304409394045093950489819A8157
:10331000AB81BC818093860490938704A09388043A
:10332000B0938904C501B4010E9483F0A7019601FE
:103330000E9483F06B017C0120E030E04FE753E412
:103340000E9465E9181634F4C12CD12C8FE7E82EC1
:1033500083E4F82E20E030E0A901C701B6010E9405
:10336000E6F187FF06CFEECE60913007709131070E
:1033700080913207909133070895FC0190E1A5E711
:10338000B4E001900D929A95E1F70895EF92FF92C3
:103390000F931F93E0928E03F0928F03009390039C
:1033A00010939103B62F172F022FF32E242F582F8F
:1033B000B093920310939303509394036FEFFF27FE
:1033C000B01B1F09520B30F450951095B195160B98
:1033D000560B66276093AB04A6E0BA9F00929F0449
:1033E000712DEE271A9F700DE11D5A9FE00D70930D
:1033F000A004E093A104AFE0BA9F0092A304712D52
:10340000EE271A9F700DE11D5A9FE00D7093A404E2
:10341000E093A504AAE0BA9F0092A704712DEE27BD
:103420001A9F700DE11D5A9FE00D7093A804E09360
:10343000A9041F910F91FF90EF900895A5E0B0E0CF
:10344000E4E2FAE10C9452F06F36710581059105C2
:1034500078F4FB01EE0FFF1FEE0FFF1FE159F74F4E
:1034600065917591859194912596EBE00C946EF0A1
:10347000F62EE72E282FEFE6F7E00027BB275F2D7B
:103480008E2D922F992341F4982F852FB85F992381
:1034900019F4982F8827B85F903138F48295929567
:1034A000582F5F70807F952BBC5F903428F4880F75
:1034B000991F880F991FBE5F903818F4880F991FC5
:1034C000B395880F991FE90FF01F549181E0992758
:1034D000B85079F1C0F0B0FF02C0550F881FB1FF9E
:1034E00004C0550F881F550F881FB2FF06C0829574
:1034F0005295152F1F70507F812BB3FF1AC0982F44
:10350000852F552716C0B195B0FF02C085955795F8
:10351000B1FF04C08595579585955795B2FF05C0B5
:103520008295507F5295582B8F70B3FF02C0582F51
:103530008827BB247727AA27B2E0F59EB018710927
:10354000A00BB00BE59E7019A109B00B259FA01927
:10355000B109F89E7019A109B00BE89EA019B10934
:10356000289FB019F99EA019B109E99EB0195B9D79
:10357000A12C99244427662733278B9DA00C911CEE
:10358000401F601F301F9B9D900C411D601F301F0E
:10359000579FA00C911C401F601F301F879F900CED
:1035A000411D601F301F979F400D611D301F5A9FA6
:1035B000900C411D601F301F8A9F400D611D301F00
:1035C0009A9F600D311D5B9F400D611D301F8B9FC9
:1035D000600D311D9B9F300DB1E0AA277727BB24DA
:1035E000F49EB0187109A00BB00BE49E7019A109EC
:1035F000B00B249FA019B109F69E7019A109B00B58
:10360000E69EA019B109269FB019F39EA019B10931
:10361000E39EB019BF187E09A20B20F0B1E04B0F5A
:10362000601F301F1124762F642F90E0832F1CCF52
:10363000FC017081472F50E0062E02C0559547953A
:103640000A94E2F740FF14C040910D0450E0062EAA
:1036500002C0559547950A94E2F740FF09C021E062
:1036600030E001C0220F6A95EAF7209527232083D6
:1036700008958F929F92AF92BF92CF92DF92EF9276
:10368000FF92FC01C080D180E280F38020E030E036
:1036900048EC52E4C701B6010E94CAE94B015C0143
:1036A00020E030E0A901C701B6010E9465E920E0F1
:1036B00030E040EA50E487FF04C020E030E040EA18
:1036C00050ECC501B4010E9483F02DEC3CEC4CECB5
:1036D0005DE30E94CAE90E9462F19B018BE237FF21
:1036E00005C022273327261B370B8DE280939C02CF
:1036F000C90168EE73E00E941DF0CB01EAE0F0E042
:10370000BF010E941DF0805D80939D02C90164E6A7
:1037100070E00E941DF0CB01BF010E941DF0805D92
:1037200080939E02C901BF010E941DF09C01CB0144
:10373000BF010E941DF0805D80939F028EE2809306
:10374000A002205D2093A1028CE992E0FF90EF900F
:10375000DF90CF90BF90AF909F908F9008954F9241
:103760005F926F927F928F929F92AF92BF92CF9211
:10377000DF92EF92FF92FC01C080D180E280F38063
:1037800020E030E04AE754E4C701B6010E94CAE9EC
:103790004B015C0120E030E040E251ECC701B60192
:1037A0000E9465E9181654F420E030E048EC52E439
:1037B000C701B6010E94E6F187FD8AC020E030E033
:1037C000A901C701B6010E9465E987FF72C060E0E8
:1037D00070E080EA90ECA50194010E9483F02DEC4A
:1037E0003CEC4CEC5DE30E94CAE90E9462F16B0183
:1037F0007C01F7FC63C020E137E240E050E00E942A
:10380000B5EFCA01B9012AE030E040E050E00E9483
:10381000B5EF605D60939C02C701B60128EE33E00E
:1038200040E050E00E94B5EF9AE0892E912CA12C47
:10383000B12CCA01B901A50194010E94B5EF605DE8
:1038400060939D02C701B60124E630E040E050E0FD
:103850000E94B5EFCA01B901A50194010E94B5EF1C
:10386000605D60939E028EE280939F02C701B60165
:10387000A50194010E94B5EF6B01CA01B901A50130
:1038800094010E94B5EF605D6093A002F0E3CF0E5B
:10389000C092A1028CE992E0FF90EF90DF90CF9070
:1038A000BF90AF909F908F907F906F905F904F9060
:1038B000089560E070E080EA90E48DCFF094E094A9
:1038C000D094C094C11CD11CE11CF11C6DE2A2CFAC
:1038D00020E030E0A901C701B6010E9465E987FF39
:1038E0006BC060E070E080EA90ECA50194010E945A
:1038F00083F02DEC3CEC4CEC5DE30E94CAE90E94A5
:1039000062F14B015C0120E030E0A901C701B60182
:103910000E9465E987FD0BC020E030E040E251E401
:10392000C701B6010E94E6F160E287FD13C0B7FC53
:1039300048C0C501B40128EE33E040E050E00E94E9
:10394000B5EFCA01B9012AE030E040E050E00E9442
:10395000B5EF605D60939D02C501B40124E630E0DF
:1039600040E050E00E94B5EF8AE0482E512C612CD7
:10397000712CCA01B901A30192010E94B5EF605DEB
:1039800060939E028EE280939F02C501B401A30161
:1039900092010E94B5EF6B01CA01B901A301920126
:1039A0000E94B5EF605D6093A00280E3C80EC092F4
:1039B000A1028DE992E070CF60E070E080EA90E4CF
:1039C00094CFB094A09490948094811C911CA11CDD
:1039D000B11C6DE2BFCF282F81E3243609F080E2CD
:1039E00080939E0290E22A3040F03AE0822F632FCB
:1039F0000E94F0EF0E94F0EF905D90939F02822F63
:103A00006AE00E94F0EF905D9093A00285E28093BF
:103A1000A1028EE992E0089560912C0170912D0130
:103A2000072E000C880B990B0E946BE92AE037EDFA
:103A300043E25CE30E94CAE960936F0170937001F6
:103A400080937101909372010895CF93DF93EC01FD
:103A5000CB01BA010E946BE923E333E343E250E474
:103A60000E94CAE920E030E040E05FE30E9483F07A
:103A70000E9467F16883DF91CF9108950E946BE9FE
:103A800023E333E343E250E40E94CAE920E030E05C
:103A900040E05FE30E9483F00E9467F124E6629FAA
:103AA000C001112481589F4F6FEF70E00E941DF0FC
:103AB000862F91CF80917407811104C080912807CF
:103AC0008093A70708958091BF148823C1F0815087
:103AD0008093BF14E9EFF2E1882351F08150990BF4
:103AE0002BE1289FF001299FF00D1124EF54FC4E8B
:103AF0008BE1AEEDB2E101900D928A95E1F7209154
:103B0000BF14211105C08091C91480648093C91429
:103B100081E090E0A0E0B0E0211103C080E090E0FF
:103B2000DC0180936A0790936B07A0936C07B093B6
:103B30006D071092650781E08093670783E08093AB
:103B40006A010895CF93DF93EC01CB01BA010E9483
:103B50006BE9688379838A839B83DF91CF91089592
:103B6000CF93DF93EC01CB01BA010E946BE92DECFE
:103B70003CEC4CEC5DE30E94CAE9688379838A835C
:103B80009B83DF91CF910895CF93DF93EC01CB011D
:103B9000BA010E946BE92AE037ED43E25CE30E9440
:103BA000CAE9688379838A839B83DF91CF910895E3
:103BB000CF92DF92EF92FF92CF93DF9300D000D0AD
:103BC000CDB7DEB70E946BE92AE037ED43E25CE354
:103BD0000E94CAE96B017C0120E030E0A9010E944B
:103BE00065E92DEB37E346E055E387FF04C02DEB95
:103BF00037E346E055EBC701B6010E9483F06983C5
:103C00007A838B839C83CE010196A9DD0F900F9060
:103C10000F900F90DF91CF91FF90EF90DF90CF90BA
:103C20000895CF93DF93EC01CB01BA010E946BE9B9
:103C30000E9462F179836883DF91CF9108958F921A
:103C40009F92AF92BF92CF92DF92EF92FF92FC01D0
:103C5000C080D180E280F38020E030E0A901C7017C
:103C6000B6010E9465E987FD99C06DEB77E386E0B8
:103C700095E3A70196010E9483F09F7720E030E052
:103C800048EC52E40E94CAE920E030E040EA50E407
:103C90000E9483F02DEC3CEC4CEC5DE30E94CAE901
:103CA0000E9462F16B017C0180E280939B0260E2E2
:103CB000F0E1CF16F7E2DF06E104F1048CF0C70172
:103CC000B60120E137E240E050E00E94B5EFCA01C2
:103CD000B9012AE030E040E050E00E94B5EF605DBD
:103CE00060939C0260E288EEC81683E0D806E10487
:103CF000F1048CF0C701B60128EE33E040E050E05B
:103D00000E94B5EFCA01B9012AE030E040E050E07E
:103D10000E94B5EF605D60939D0260E2E4E6CE161E
:103D2000D104E104F1048CF0C701B60124E630E0CF
:103D300040E050E00E94B5EFCA01B9012AE030E04E
:103D400040E050E00E94B5EF605D60939E028AE023
:103D5000882E912CA12CB12CC701B601A50194018C
:103D60000E94B5EF6B01CA01B901A50194010E943F
:103D7000B5EF605D60939F028EE28093A002F0E356
:103D8000CF0EC092A1028BE992E0FF90EF90DF90FE
:103D9000CF90BF90AF909F908F9008956DEB77E399
:103DA00086E095EB66CFA4E0B0E0E9EDFEE10C948F
:103DB0005BF00E946BE92DEC3CEC4CEC5DE30E9467
:103DC000CAE969837A838B839C83CE01019637DFAE
:103DD0002496E2E00C9477F0CF93DF93EC018D8191
:103DE0000E94808F60E08B810E94F1D0DF91CF91A3
:103DF0000895CF92DF92EF92FF920F931F93CF938C
:103E00008C01C62F69017A01E7DF0E946AD28C2FEC
:103E100080640E94748F8F2D0E94748F8E2D0E945B
:103E2000748F8D2D0E94748F8C2D0E94748F87E863
:103E3000C11101C085E90E94748FCC3011F40E9439
:103E4000798FC0E00E94798FF801868387FF04C0D4
:103E5000CF3F11F0CF5FF6CFCF911F910F91FF9021
:103E6000EF90DF90CF90089561E0FC0183810E9484
:103E7000F1D08FEF0C94748F0F931F93CF938C011D
:103E8000ABDF0E946AD2C82F882369F08DEF0E94B1
:103E9000748F0E946AD2C82FC801E6DF8C2FCF91A1
:103EA0001F910F91089582E1F8018483F5CFB0E06E
:103EB000A0E0EDE5FFE10C9451F0EC016A017B011B
:103EC0004801590120E030E0A90167E392DFA50134
:103ED000980167E1CE018DDF81111DC08F81833094
:103EE00039F089E0CC0CDD1CEE1CFF1C8A95D1F763
:103EF000A701960169E1CE017CDF11E0882319F06A
:103F000010E087E08C83CE01AFDF812FCDB7DEB725
:103F1000ECE00C946DF089E08C8310E0F4CFCF934B
:103F2000DF93EC016EBDFA01CA019E5F0DB407FE7E
:103F3000FDCF20812EBD0DB407FEFDCF21812EBD0A
:103F40003296E817F90791F70DB407FEFDCF8FEF12
:103F50000E94748F8FEF0E94748F0E94798F8E83DE
:103F60008F71853041F083E18C83CE017DDF80E06D
:103F7000DF91CF91089581E0FBCF0F931F93CF93F3
:103F8000DF93EC018B0128DF0E946AD281110BC004
:103F900085E18C8310E0CE0167DF812FDF91CF9127
:103FA0001F910F910895A8016CEFCE01B8DF182F73
:103FB000882371F3F0CF0F931F93CF93DF93EC011E
:103FC00089018F81833039F089E0440F551F661FC6
:103FD000771F8A95D1F79A01AB0168E1CE0109DF1D
:103FE000811127C0A8016EEFCE0199DF182F882319
:103FF000A9F00E946AD2182F8823C1F020E030E097
:10400000A9016DE0CE01F5DE882321F086E18C83E5
:1040100010E004C00E94798F8111F8CFCE0124DF17
:10402000812FDF91CF911F910F91089587E18C83AC
:10403000F5CF86E0ECCF1F93CF93DF93EC01CCDE7E
:1040400020E030E0A9016CE0CE01D3DE11E088234E
:1040500019F010E083E08C83CE0106DF812FDF9121
:10406000CF911F9108951F93CF93DF93EC018F8120
:10407000833039F089E0440F551F661F771F8A95FA
:10408000D1F79A01AB0162E1CE01B3DE11E08823E2
:1040900019F010E085E08C83CE01E6DE812FDF9100
:1040A000CF911F9108958F929F92AF92BF92EF92FE
:1040B000FF920F931F93CF93DF938C01EB017A0153
:1040C0000E94D6D14B015C012CE2820E21E0921EAF
:1040D000A11CB11C0E94798FF80186838F3F69F47F
:1040E0000E94D6D1681979098A099B0997FDF2CFF8
:1040F00081E1F8018483C0E021C08E3F69F5F1E0E1
:10410000EF1AF1088FEF8EBDFE012FEF0DB407FE01
:10411000FDCF8EB581932EBDCF018C1B9D0B8E15CF
:104120009F05A0F30DB407FEFDCF8EB5CE0DDF1DAC
:1041300088830E94798F0E94798FC1E0C80194DE44
:104140008C2FDF91CF911F910F91FF90EF90BF9037
:10415000AF909F908F9008958FE0CBCF0F931F93D8
:10416000CF93DF93EC018B0137DE40E052E0B801E2
:10417000CE0199DFDF91CF911F910F9108950F9399
:104180001F93CF93DF93EC0189018F81833039F046
:1041900089E0440F551F661F771F8A95D1F79A0152
:1041A000AB0161E1CE0125DE882351F084E08C83F0
:1041B000CE015ADE80E0DF91CF911F910F910895DB
:1041C00040E052E0B801CE016EDFF5CFB0E0A0E0F4
:1041D000ECEEF0E20C9451F0EC01162F1F821C82E1
:1041E0004B830E94D6D16B017C0120EDC20E27E0EB
:1041F000D21EE11CF11CA89561E08B810E94F1D0D8
:104200008B810E9417B6249A2C9A279A2698259A71
:1042100081E00E94808F85E08D830E94808F0AE07C
:104220008FEF0E94748F0150D9F7A89520E030E0FD
:10423000A90160E0CE01DDDD8E83813079F00E943E
:10424000D6D16C197D098E099F0997FDEFCF81E0CA
:104250008C83CE0109DE1A8280E065C0A8952AEA27
:1042600031E040E050E068E0CE01C3DD853031F55B
:1042700081E08F83A8958F81812C912C540182300D
:1042800029F4812C912CA12C80E4B82E20E030E080
:10429000A90167E3CE01ADDDA501940169E2CE017C
:1042A000A8DD8E838823F1F00E94D6D16C197D0998
:1042B0008E099F0997FDEACF8AE0CACF04E00E94E9
:1042C000798F8E830150D9F78A3A11F482E0D1CFE9
:1042D0000E94D6D16C197D098E099F0997FDBFCF29
:1042E00082E0B6CF8F818230B9F420E030E0A901BE
:1042F0006AE3CE017EDD882311F088E0A9CF0E9419
:10430000798F807C803C11F483E08F830E94798FC9
:104310000E94798F0E94798FCE01A6DD81E08A8389
:10432000173030F41D83CDB7DEB7ECE00C946DF0A0
:1043300088E18C8391CF0F931F93CF93DF93EC0190
:104340008B0120E030E0A90169E053DD882351F0C2
:1043500080E18C83CE0188DD80E0DF91CF911F91D9
:104360000F91089540E150E0B801CE019CDEF5CFF9
:10437000CF93C82FCB010E94938483EA96E00E94DA
:10438000938484E996E0CC2311F089E996E00E94B9
:1043900093848AE00E947284CF910895EF92FF92F5
:1043A0000F931F93CF937B018A01C2E48F3F09F0E3
:1043B000C4E580E20E9472848C2F0E9472848AE39A
:1043C0000E947284F701608171818281938142E051
:1043D0000E9436B684E593E10E949384F8016081DF
:1043E00071818281938142E00E9436B662E070E082
:1043F00080E090E00E944DD1CF911F910F91FF90EE
:10440000EF9008950C94E2D140918C0321E0422773
:104410006CE070E00C94EBB540918C0321E04227F6
:1044200064E070E00C94EBB540918C0321E04227EE
:1044300061E070E00C94EBB540918C0321E04227E1
:1044400061E070E00C94EBB540918C0321E04227D1
:1044500068E070E00C94EBB540918C0321E04227BA
:104460006CE070E00C94EBB541E061E070E00C941E
:10447000EBB540918C0321E042270C94EBB56CE046
:1044800070E00C9480D161E070E00C9480D161E028
:1044900070E00C9480D16CE070E00C9480D164E00A
:1044A00070E00C9480D19091B30281E089270C9444
:1044B0000A7A61E088E297E00C94967A20E030E096
:1044C000A901BC0185E791E00C94ADC780E090E0C4
:1044D000A0E8B0E480937D0190937E01A0937F01DA
:1044E000B09380018AE192E0E9DF80E090E0A0EF04
:1044F000B1E48093750190937601A0937701B09316
:1045000078018093790190937A01A0937B01B09315
:104510007C01E091EA03EE0FFF0BE650FE4F808135
:1045200091818330910539F184309105C9F1029769
:1045300061F480E090E0A3E4B3E48093750190938C
:104540007601A0937701B093780182E092E0B6DF24
:1045500010927D0110927E0110927F0110928001D5
:104560008AE192E0ABDF8091EA038F5F8430ECF464
:104570008093EA03089580E090E0A3E4B3E480939D
:10458000750190937601A0937701B09378018093A1
:10459000790190937A01A0937B01B0937C01D5CFF0
:1045A00080E090E0A3E4B3E4F2CF1092EA03089530
:1045B000A4E0B0E0EEEDF2E20C945BF084EF91E069
:1045C000A0E0B0E089839A83AB83BC83BE016F5FB8
:1045D0007F4F88E70E9439832496E2E00C9477F0BD
:1045E000B0E0A0E0E6EFF2E20C945BF020E24F8155
:1045F00058856E818D810E94A4CCE2E00C9477F006
:1046000080912807909129070C9417D26091280770
:104610008FEF0C9421D280912807682F0C9421D21F
:104620006FEF809128070C9421D26AE673E582E04F
:104630000C94B2CE6EE673E581E00C94B2CE62E7E4
:1046400073E580E00C94B2CE66E773E583E00C94EA
:10465000B2CE109265070C9462DA4FE350E064EC3E
:1046600074E086EE96E00C94BCF280915F1390911A
:104670006013891B8F7011F40C94EA7B81E008951C
:1046800080916A01882341F06091E2037091E30315
:1046900041E081E00C9444CC0895B0E0A0E0E3E573
:1046A000F3E20C944BF0EC014B018A018B818111F8
:1046B00007C08FEF9FEFCDB7DEB7E2E10C9467F054
:1046C000898180FFF6CF89899A89AB89BC89488521
:1046D00059856A857B85841B950BA60BB70BA801B2
:1046E00070E060E084179507A607B70708F48C010F
:1046F00068011E0124E0220E311CC114D10409F40A
:10470000AAC0488559856A857B855A0181E0B8220F
:10471000898D9A8D2A013B0139E0769467945794EC
:1047200047943A95D1F72B81FC01223089F5628DAF
:10473000738D848D958D640D751D861D971DE12CDF
:1047400022E0F22EEA18FB08CE14DF0408F476010A
:10475000E114E2E0FE0671F440909512509096123A
:1047600060909712709098126415750586059705EC
:1047700009F04EC040E00E94D2D8882309F499CFB6
:10478000B5016B567F4EA701C4010E9479F252C059
:10479000F480FA94F420A114B10471F4F1100CC067
:1047A000452B462B472B51F58D899E89AF89B88DB6
:1047B0008C839D83AE83BF83E98DFA8D4C805D80B1
:1047C0006E807F8022E0421A510861087108858559
:1047D00004C0440C551C661C771C8A95D2F786854C
:1047E0009785A089B189480E591E6A1E7B1EC30198
:1047F000B2016F0D711D811D911DA1CF4C815D8195
:104800006E817F8191010E9444DB8111D5CF51CF10
:10481000A0919A12B0919B12ED91FC911197008892
:10482000F189E02D9401AB01BC01CD0109958823EC
:1048300009F43FCF8E0C9F1C88859985AA85BB857E
:104840008E0D9F1DA11DB11D88879987AA87BB87E3
:10485000CE18DF0852CFC8012ECF0F931F93CF93EE
:10486000DF93FC012381222331F080E0DF91CF919F
:104870001F910F9108958B01EC01FB018789803115
:1048800039F582E08B831D8A1E8A1F8A188E808DDF
:10489000918DB0E0A0E025E0880F991FAA1FBB1FF3
:1048A0002A95D1F7898B9A8BAB8BBC8B1A8F098F8A
:1048B00081E08983188619861A861B861C821D82D0
:1048C0001E821F82188A1C861D861E861F86CECFDA
:1048D000803259F683E08B83428D538D648D758DC4
:1048E0004D8B5E8B6F8B788F9E012F5E3F4FC80183
:1048F0000E94C0DB8111DACFB8CFCF93DF93EC01F8
:104900000E9429DC1B82DF91CF910895CF93DF9322
:10491000EC01462F41706C857D858E859F850E94B8
:10492000D2D8882351F0888920E2829FC0011124C7
:104930008B569F4EDF91CF91089590E080E0FACFA3
:10494000CF93DF93EB01FC012381211104C080E0B0
:10495000DF91CF9108952250223028F48FE288838E
:10496000198281E0F5CF60E0D1DF009781F3DC01AF
:1049700060E080E09EE22D91203299F0883031F4A1
:104980009E01260F311DF90190836F5F9E01260F56
:10499000311DAD0141505109FA014081F9014083B7
:1049A0006F5F8F5F8B3039F7FE01E60FF11D1082CC
:1049B000D8CFACE0B0E0EFEDF4E20C944CF05C0149
:1049C000DC0159968D909C90F40181859285A38598
:1049D000B4859C01AD012F5F3F4F4F4F5F4F29873B
:1049E0003A874B875C87D50114964D905D906D900A
:1049F0007C901797411451046104710409F459C063
:104A0000BFEF4B1A5B0A6B0A7B0A312C7301620100
:104A10001D821E821F821886F40181859285A385DE
:104A2000B4852D813E814F815885281739074A0763
:104A30005B0708F056C089859A85AB85BC858C15C7
:104A40009D05AE05BF0550F482E0C82ED12CE12CA7
:104A5000F12C92E0492E512C612C712C9E012F5F7C
:104A60003F4FB701A601C4010E9444DB8823C9F16E
:104A700089819A81AB81BC81892B8A2B8B2B01F197
:104A8000260137019FEF491A590A690A790A2D81CF
:104A90003E814F8158852F5F3F4F4F4F5F4F2D8392
:104AA0003E834F8358873FEFC31AD30AE30AF30AC2
:104AB000B3CF408051806280738033243394A6CF7B
:104AC000C414D504E604F70411F70FEF1FEF2FEF1E
:104AD0003FE0B701A601C4010E94CADA782E811115
:104AE00006C0712C872D2C96E1E10C9468F0F5013D
:104AF00044815581668177814115510561057105B4
:104B000039F097018601C4010E94CADA882349F36B
:104B1000D5011496CD92DD92ED92FC921797332039
:104B200051F0D701C6010196A11DB11DF40180838A
:104B30009183A283B383F50185899689A789B08D76
:104B4000892B8A2B8B2B71F6C58AD68AE78AF08E41
:104B5000818180688183C6CF40E050E0BA010C9427
:104B600072DC4F925F926F927F92AF92BF92CF9220
:104B7000DF92EF92FF920F931F93CF93DF931F92D9
:104B8000CDB7DEB78C017B015A01C22EDB015996ED
:104B90008D919C91F801928F818FCB01DDDF712C7B
:104BA000F70180859185A285B38541895289638902
:104BB000748984179507A607B70708F051C055E018
:104BC000B695A795979587955A95D1F7F82FFF70C9
:104BD000DF2ED70113968C91823010F480E0D9C07B
:104BE00041E050E0BE016F5F7F4FC70156DD019786
:104BF000A9F7F70180859185A285B3854F96A11D00
:104C0000B11D80879187A287B387F0E2DF9EB00154
:104C100011246B567F4E6115710501F3DB018C91F8
:104C2000882341F0853E09F04BC0772029F0772496
:104C30007394B6CF71100EC0809195129091961218
:104C4000A0919712B0919812F80184879587A68752
:104C5000B787D08ADB018C918111E9CF77247394D7
:104C60008C2D8274823409F0B9CF772009F4A1C069
:104C7000F801D08861E0C80149DE009709F4AECFA1
:104C800020E2DC011D922A95E9F72BE0F501DC0119
:104C900001900D922A95E1F721E238E2FC01318B77
:104CA000208B40E058E057874687338B228B318F2B
:104CB000208F578B468B0E9489D8811109C08ECFD7
:104CC0004BE050E0C5010E946CF2892B09F068CFDF
:104CD000F0E2DF9ED00111249D012B563F4EF901D9
:104CE0008385817121F08C2D827109F000C1F8015A
:104CF000818D928D409195125091961260919712EC
:104D0000709198124487558766877787D08AFD010E
:104D1000EB56FF4E44885588712C612C3201552486
:104D20004424D80155964D925D926D927C9258978D
:104D3000428D538D70E060E044295529662977291A
:104D400055964D935D936D937C935897D9011B961F
:104D50002C91287109F0BDC0848D958DA68DB78DDD
:104D6000F801818B928BA38BB48B81E083838C2D94
:104D70008F70F80181831482158216821782108643
:104D800011861286138681E0C4FE03C0C8010E940A
:104D9000F7DC0F90DF91CF911F910F91FF90EF9073
:104DA000DF90CF90BF90AF907F906F905F904F90CB
:104DB0000895D70113968C911397823009F40ECF82
:104DC00051968D919D910D90BC91A02D803E9F4F4D
:104DD000AF41B10508F002CFC701EBDD882309F42C
:104DE000FDCE0E9489D8882309F4F8CED7015996C0
:104DF000ED91FC915A9714964D905D906D907C903A
:104E00001797B2E04B1A510861087108858504C0F4
:104E1000440C551C661C771C8A95D2F786859785AD
:104E2000A089B189480E591E6A1E7B1E81E08093BD
:104E30009912409295125092961260929712709227
:104E40009812E5E9F0E180E092E0DF019C011D921B
:104E500021503040E1F7DD24D394D7015996ED91EC
:104E6000FC918481D816C0F480919A1290919B1283
:104E7000DC01ED91FC910288F389E02D25E930E118
:104E8000B301A2014D0D511D611D711D09958823AE
:104E900009F4A4CED394E1CF258580E092E0A0E090
:104EA000B0E004C0880F991FAA1FBB1F2A95D2F734
:104EB000F7014189528963897489840F951FA61F60
:104EC000B71F818B928BA38BB48B85E990E1D12C9A
:104ED000D7CE203161F498012F5E3F4F0E94C0DB96
:104EE000882329F084E0D80113968C9340CFD80111
:104EF00013961C9273CEFC0123812111FECC0895E0
:104F0000A1E4B0E0E6E8F7E20C944BF04C015B0161
:104F10007A01222E19821C821C8E1F8E611571054A
:104F200069F410E0CE014C96E6DFCE010196E3DF96
:104F3000812FCF5BDF4FE2E10C9467F0FC018381AE
:104F40008111EFCFFA0180818F3251F18B01CE01B7
:104F500001966C012C0180E2382E360122963FAE7C
:104F6000229721963FAE21973FAE3EAE3DAE3CAE7E
:104F70003BAE3AAE39AE38AE3FAA970190E047E07B
:104F8000D9018D91882309F446C08F3209F443C0BA
:104F90008E3201F54A3029F298E04AE09D01F0CFC7
:104FA000FB0183818250823098F0618D728DCE0139
:104FB0004C9653DC882309F4B4CF8E01045E1F4F56
:104FC000C7017C010196F70120812F32D1F3BFCFB9
:104FD0008B01F6CFE0E6F3E12491222321F0319614
:104FE0008213FACF9ECF491708F49BCF813208F481
:104FF00098CF8F3709F495CF3FE9380F3A3108F44D
:1050000020EEE7E3F0E0EC0FFD1FE90FF11D820F4A
:1050100080839F5FC3CF8FA9803209F482CF79014B
:10502000F90180812F5F3F4F8F32C9F38823C1F090
:1050300021E0AE01495C5F4FB801C60192DD8823D3
:1050400009F46FCF0A151B0511F0C80156DCCE011B
:105050004C964C145D0409F0C30186016C017ECFAF
:10506000222DAE01495C5F4FB801C4017ADD182FD3
:1050700059CFEF92FF921F93CF93DF93CDB7DEB757
:1050800028970FB6F894DEBF0FBECDBF182F8AEA5F
:10509000E82E82E1F82EF70160857185072E000C5D
:1050A000880B990B0E946BE96D837E838F839887B1
:1050B000F70184819581A681B78189839A83AB8327
:1050C000BC83AE014B5F5F4FBE016F5F7F4F80E0DF
:1050D00065D99CE2E92E97E0F92EF701608571858C
:1050E000072E000C880B990B0E946BE96D837E8361
:1050F0008F839887F70184819581A681B781898301
:105100009A83AB83BC83AE014B5F5F4FBE016F5F81
:105110007F4F8FEF43D987E11802F0011124E65544
:10512000FD4E628570E08CE593E10E94F08DF70101
:10513000628570E087E593E10E94F08D28960FB6B6
:10514000F894DEBF0FBECDBFDF91CF911F91FF90CE
:10515000EF9008950F930FB70F9300916E000B7FA0
:1051600000936E0078940F930BB70F930CB70F92C8
:105170001F922F933F934F935F936F937F938F93E0
:105180009F93AF93BF93EF93FF9311240E943F66C9
:10519000FF91EF91BF91AF919F918F917F916F910F
:1051A0005F914F913F912F911F900F900CBF0F91E6
:1051B0000BBF0F910460F89400936E000F910FBF26
:1051C0000F911895CF93DF9310929C03CAEAD2E116
:1051D000198618860E94E2D11A865D98CCE2D7E043
:1051E000198618860E94856A1A865C98DF91CF918D
:1051F0000895B0E0A0E0EFEFF8E20C9451F0B0E4D5
:10520000A0E06A2F70E0AB014B0F511D55954795FB
:10521000411111C0E7EAFAE265917491072E000C82
:10522000880B990B0E946BE9CDB7DEB7ECE00C94CC
:105230006DF0B42FE8CFA41711F0B41303C0E3EA64
:10524000FBE2EACF9A0121503109220F331F220FCE
:10525000331FF901EB55F54DE590F490F901E75551
:10526000F54DC591D4918E159F051CF3A42FC81739
:10527000D9070CF4C6CFF901E955F54D0591149104
:10528000F901E555F54DC590D490BC016E197F0923
:10529000072E000C880B990B0E946BE94B015C01F7
:1052A000B601601B710B072E000C880B990B0E9436
:1052B0006BE99B01AC01C501B4010E94CAE94B0135
:1052C0005C01BE016E197F09072E000C880B990B3B
:1052D0000E946BE99B01AC01C501B4010E94FAF088
:1052E0006B017C01B801012E000C880B990B0E9408
:1052F0006BE99B01AC01C701B6010E9483F094CF1A
:10530000EF92FF920F931F93CF93C82F7B018A01D7
:1053100080912707833090F00E94008BC7010E9484
:1053200093848AEB92E10E949384CF3FF1F486EB61
:1053300092E10E9493848AE00E94728443DFA895E0
:1053400080918504811123C081E08093850482E0EF
:105350008093270737DF6DEA72E1CF3F11F061EBF1
:1053600072E140E0C8010E94A28EC7FDE4CF84EB49
:1053700092E10E9493846C2F0C2E000C770B880B0B
:10538000990B0E94ECB38AE00E947284D4CFCF9133
:105390001F910F91FF90EF900895B0E0A0E0E3ED32
:1053A000F9E20C944DF0EC016B014A01B22EFA01C6
:1053B0004080518062807380A30192016D817E8163
:1053C0008F8198850E9465E98823A1F04D825E82D5
:1053D0006F827886AA24A39420E030E0A901F4012A
:1053E00060817181828193810E94E6F118160CF030
:1053F000A12CAC828C818230A1F0833009F44FC0A3
:105400008130D1F52D813E814F815885F601608133
:105410007181828193810E9465E987FD2DC082E0C0
:105420008C83B7010F2C000C880B990B0E946BE941
:105430009B01AC016D817E818F8198850E9482F0F5
:105440009B01AC01F60160817181828193810E9490
:10545000E6F187FD16C00E94D6D16B017C01980150
:10546000A8EEB3E00E94E1EFC60ED71EE81EF91EBB
:10547000C882D982EA82FB82CDB7DEB7E0E10C9424
:1054800069F00E94D6D1088119812A813B81601B75
:10549000710B820B930B97FDEFCF83E08C8344E37A
:1054A00053E164E473E18B2D2BDFE6CF48ED52E14D
:1054B00065EE72E125CFCF93DF93A8958091AC1272
:1054C0009091AD120E9464B56093AE127093AF12CA
:1054D0008093B0129093B11280912E0790912F0774
:1054E00088DE609330077093310780933207909382
:1054F0003307C091AC12D091AD12809163019091AD
:105500006401C817D90714F480E0D0DF8091B2128B
:105510009091B312181619066CF480916101909164
:1055200062018C179D0734F445E153E162E273E1B7
:1055300080E0E6DE20912E0730912F078091DD0676
:105540009091DE062817390714F48FEFAFDF8091B2
:10555000340790913507181619068CF420912E0700
:1055600030912F0780915F0190916001821793071E
:1055700034F445E153E162E273E18FEFC1DEDF9184
:10558000CF910895A4E0B0E0E8ECFAE20C9451F079
:1055900080912707811106C0A8952496ECE00C9411
:1055A0006DF028C180919A048111F7CF81E080933A
:1055B0009A0480919D03811107C010929A04249649
:1055C000ECE00C946DF016C176DF10929D030E9402
:1055D000D6D14B015C010E9407B46B017C01609144
:1055E000670170916801072E000C880B990B0E94CF
:1055F0006BE99B01AC01C701B6010E94E6F11816E8
:105600000CF4E7C06091B2127091B312072E000C37
:10561000880B990B0E946BE969837A838B839C8347
:1056200034E0E32EF12C08E210E020E0AE014F5F01
:105630005F4F6EEA72E184E193E1AFDEC090AE129B
:10564000D090AF12E090B012F090B112609165016D
:1056500070916601072E000C880B990B0E946BE974
:105660009B01AC01C701B6010E94E6F11816CCF40B
:105670006091670170916801072E000C880B990BEF
:105680000E946BE99B01AC01C701B6010E9465E96C
:1056900087FF07C00E9410B40E9462F1759567955C
:1056A00001C060E06093B4128091A6129091A7129D
:1056B000A091A812B091A9120097A105B105C1F05F
:1056C000A5019401281B390B4A0B5B0BDA01C901B8
:1056D000B7FD0EC00E9407B40E9462F12091A4128F
:1056E0003091A512621773070CF47DC00E94E2D1BD
:1056F0000E94B41920E030E04AEF52E40E94E6F143
:1057000018160CF463C08091980390919903A091AE
:105710009A03B0919B030097A105B105A1F0881AE7
:10572000990AAA0ABB0AB7FC0EC00E94B4190E94CB
:1057300062F12091960330919703621773070CF47E
:105740004BC00E94856A6091340770913507072E1F
:10575000000C880B990B0E946BE969837A838B8319
:105760009C8392E0E92EF12C04E110E02FEFAE01D2
:105770004F5F5F4F60E377E08DE193E10EDE809055
:10578000300790903107A0903207B090330720E0A7
:1057900030E040EA50E4C501B4010E94E6F187FD23
:1057A00011C020E030E04AEF52E4C501B4010E948C
:1057B00065E918163CF00E9460180E9462F1759528
:1057C000679501C060E060933607F7CE8FEF6EDE1D
:1057D0009ACF80E06BDE16CF47EF52E166E073E1CF
:1057E0008FEF8EDDB0CF47EF52E166E073E180E0EE
:1057F00087DD7ECFCF92DF92EF92FF92CF93DF9340
:10580000EC01C880D980EA80FB8083EA92E10E94A3
:105810009384C701B6010E945776CC80DD80EE806C
:10582000FF808EED9EE20E949384C701B6010E9424
:105830005776C884D984EA84FB848AED9EE20E946C
:105840009384C701B6010E9457768AE00E94728451
:10585000DF91CF91FF90EF90DF90CF900895BC0142
:10586000209166043091670440916604509167046A
:105870002417350731F481E02617370709F080E057
:1058800008959A01F1CF0F930FB70F9300916E0017
:105890000F930B7F00936E0000916F000D7F0093BC
:1058A0006F000F930BB70F930CB70F921F922F93AC
:1058B0003F934F935F936F937F938F939F93AF9398
:1058C000BF93EF93FF931124F9D4FF91EF91BF9110
:1058D000AF919F918F917F916F915F914F913F9188
:1058E0002F911F900F900CBF0F910BBF0F91026073
:1058F000F89400936F000F9100936E000F910FBF0B
:105900000F91189500C000C08091E10680FF1FC074
:10591000459A8FEF80931F048091E10681FF1AC0A2
:10592000479A8FEF809320048091E10682FF15C093
:105930002A988FEF809321048091E10683FF10C0A5
:1059400028988FEF8093220400C000C008954598E6
:1059500081E0E0CF479881E0E5CF2A9A81E0EACF65
:10596000289A81E0EFCF80918D03982F977F9093B5
:105970008D03982F937081E011F080E008955E9A76
:1059800008955E9880918D03886080938D030895BB
:10599000E82FF0E021E030E0082E02C0220F331F94
:1059A0000A94E2F72095309590918D03922390937D
:1059B0008D03EA50FE4F2081922321E019F020E070
:1059C000822F0895813079F038F08230C9F7159A26
:1059D000909177079B7F04C05E9A909177079E7F96
:1059E00090937707EDCF5E9A909177079D7FF8CFE0
:1059F00080E0CEDF81E0CCDF82E0CADFB4CF81304F
:105A000079F070F0823071F021E030E001C0220FB7
:105A10008A95EAF780918D03822B80938D030895F8
:105A20005E98F2CF1598F0CFB0E0A0E0EAE1FDE299
:105A30000C9453F0C9E6DDE00FE817E089E7A82EE3
:105A40008DE0B82EC12CD12C7601C3946991799147
:105A5000899199910E9469E9288939894A895B89E4
:105A60000E94CAE90E9467F1F801619371938193E2
:105A700091938F01C616D706E806F90610F46B015C
:105A80007C01AC16BD0611F76FEF7FEFCB01A701CC
:105A900096010E9493EF20939F073093A0074093B5
:105AA000A1075093A207CDB7DEB7EAE00C946FF0E0
:105AB0000F931F93CF93DF930DE71DE0C8EAD7E064
:105AC000F80121913191419151918F0160E070E095
:105AD00080E89FE30E94FAF0699379938993999300
:105AE000F7E0C83BDF0761F70E94D0C79DDFDF9179
:105AF000CF911F910F910895DBCFDACFD9CFD8CFB7
:105B000090915F1380916013981306C08091B10D3E
:105B10009091B20D892B21F080E00E94918FF0CFFF
:105B2000089590915F1380916013981307C080913E
:105B3000B10D9091B20D892B09F45ACF80E00E94EB
:105B4000918FEFCFCF92DF92EF92FF92CF93DF93BF
:105B50002091B302222319F1EC0108960E94BB7731
:105B60006B017C0120E030E0A9010E9465E920E0A2
:105B700030E0A901882349F0CE010E943378A701C3
:105B800096010E94CAE99B01AC01688579858A85E6
:105B90009B850E9482F0688779878A879B87DF913F
:105BA000CF91FF90EF90DF90CF900895CF92DF924A
:105BB000EF92FF92CF93DF932091B302222319F14A
:105BC000EC0108960E94BB776B017C0120E030E07D
:105BD000A9010E9465E920E030E0A901882349F08D
:105BE000CE010E943378A70196010E94CAE99B0169
:105BF000AC01688579858A859B850E9483F06887DA
:105C000079878A879B87DF91CF91FF90EF90DF9014
:105C1000CF900895AEE1B0E0E0E1FEE20C944DF0EB
:105C20009E8F8D8F5B018A01FC01EA5BFF4F208113
:105C3000318142815381298B3A8B4B8B5C8BCA011A
:105C4000B9010E9469E96B017C01D5012D913D915B
:105C50004D915C910E94CAE90E94E7F02B013C0142
:105C6000F8012081318142815381C701B6010E9430
:105C7000CAE90E94E7F04B015C01C301B2010E9436
:105C800067F16D8B7E8B8F8B988F683771058105DF
:105C9000910540F428E730E040E050E02D8B3E8B4A
:105CA0004F8B588FC501B4010E9467F1698F7A8FBD
:105CB0008B8F9C8F683771058105910540F488E7CB
:105CC00090E0A0E0B0E0898F9A8FAB8FBC8FED8D14
:105CD000FE8DEE5AFF4F2081318142815381298709
:105CE0003A874B875C87CA01B9010E946BE92B0197
:105CF0003C016D897E898F89988D0E9469E96D8349
:105D00007E838F83988720E030E0A901C301B20130
:105D10000E9465E9882309F4BBC1A7019601C70168
:105D2000B6010E94CAE94B015C012D813E814F8181
:105D30005885CA01B9010E94CAE99B01AC01C5019D
:105D4000B4010E9482F04B015C01A3019201C301E6
:105D5000B2010E9483F09B01AC01C501B4010E9415
:105D6000FAF00E94E7F00E9467F169837A838B83DF
:105D70009C8369857A858B859C85909580957095A7
:105D800061957F4F8F4F9F4F0E946BE94B015C01E4
:105D9000698D7A8D8B8D9C8D0E9469E969877A87E0
:105DA0008B879C8720E030E0A901C501B4010E94E7
:105DB00065E9882309F470C129853A854B855C859E
:105DC000CA01B9010E94CAE96D877E878F87988BC7
:105DD000A7019601C701B6010E94CAE99B01AC0167
:105DE0006D857E858F8598890E9482F06B017C018C
:105DF000A5019401C501B4010E9483F09B01AC018F
:105E0000C701B6010E94FAF00E9493F1AD8DBE8DDC
:105E100095962D913D914D915C9198972D873E8758
:105E20004F87588B69017A0129813A814B815C81C6
:105E3000C21AD30AE40AF50A0E9467F1C61AD70A01
:105E4000E80AF90AF7FE8CC02D813E814F81588502
:105E5000CA01B9010E94CAE96B017C0120E030E06F
:105E6000A901C301B2010E9465E9882309F418C1A0
:105E70006D857E858F8598890E9469E99B01AC01BB
:105E80000E9483F0A30192010E94CAE94B015C01C8
:105E900029853A854B855C85CA01B9010E94CAE90A
:105EA0009B01AC01C501B4010E9483F0A7019601DA
:105EB0000E9482F04B015C0120E030E040E850E4B9
:105EC000C301B2010E94CAE99B01AC01C501B40142
:105ED0000E94FAF00E94E7F04B015C0120E030E004
:105EE000A9010E94E6F187FF03C0812C912C540187
:105EF000C501B4010E9467F169837A838B839C8317
:105F00002D853E854F85588926173707480759073D
:105F100020F429833A834B835C8369817A818B8166
:105F20009C810E9469E94B015C01A3019201C301BC
:105F3000B2010E9483F09B01AC01C501B4010E9433
:105F4000CAE9A70196010E9483F00E941FF20E94F5
:105F500067F1698B7A8B8B8B9C8BC12CD12C760152
:105F600069897A898B899C892D893E894F89588DC9
:105F7000621B730B840B950B0E9469E9A3019201CC
:105F80000E94FAF020E034E244EF59E40E94CAE9AA
:105F90000E9467F14B015C0169897A898B899C8930
:105FA000298D3A8D4B8D5C8D621B730B840B950B89
:105FB0000E9469E9A30192010E94FAF020E034E214
:105FC00044EF59E40E94CAE90E9467F16D837E8321
:105FD0008F839887C501B4010E941E1A2B013C01D2
:105FE0006D817E818F8198850E941E1A29813A8158
:105FF0004B815C81AD8DBE8D99962D933D934D93D4
:106000005C939C9789019A010C0D1D1D2E1D3F1D4F
:10601000FD0105A716A727A730ABE65BFF4F2D892B
:106020003E894F89588D2083318342835383D5968F
:106030008D929D92AD92BC92D8972D813E814F81D9
:106040005885D9962D933D934D935C93DC973D975E
:10605000408251826282738234966083718382832C
:10606000938329893A894B895C89D1962D933D93F5
:106070004D935C93D4973D96298D3A8D4B8D5C8DD5
:1060800020833183428353836E96E0E10C9469F060
:1060900060E070E0CB0165CE60E070E0CB01B4CE93
:1060A00060E070E0CB0116CF90916F0081E091FD30
:1060B00002C080E0089590916F009D7F90936F00E3
:1060C0000895EFE6F0E08081826080830895CF93A9
:1060D000C82FEADF94E0C99F90011124F901E75924
:1060E000FB4F2B583B4FD9014D915D916D917C91A8
:1060F000408351836283738391E09093680481119C
:10610000E0DFCF910895CF93DF938091E006811176
:1061100005C08091E206882309F464C08091FA03E7
:10612000329B63C081608093FA038091FA03339BB2
:106130005EC082608093FA038091FA03349B59C059
:1061400084608093FA038091FA03029B54C08860B4
:106150008093FA03C0915904C0FF0FC08091E106FB
:1061600080FF0BC08091FA0380FF07C08091260753
:1061700081608093260780E0AADFC1FF0FC0809175
:10618000E10681FF0BC08091FA0381FF07C0809177
:10619000260782608093260781E099DFC2FF22C034
:1061A0008091E10682FF1EC08091E20681110BC042
:1061B0008091FA0382FF07C0809126078460809354
:1061C000260782E084DF8091E206882359F08091DF
:1061D000FA0383FF07C08091260788608093260713
:1061E00082E075DFDF91CF9108958E7F9CCF8D7F08
:1061F000A1CF8B7FA6CF877FABCF56DF1092A307AF
:106200001092A4071092A5071092A607811159CFEA
:1062100008950F931F9380915F1390916013891BD2
:106220008F7009F449C090915C13992361F0833019
:1062300040F48FEF890F29F080935C1390E080E0A9
:1062400038C010925C13809160132BE5829FC001CF
:1062500011248854984FFC01208120FDEFCF4091FC
:10626000A3075091A4076091A5077091A607E95A6A
:10627000FF4F0081118122813381401B510B620B42
:10628000730B4093A3075093A4076093A5077093E3
:10629000A607209160132F5F2F7020935D1330911C
:1062A000601320915E13321304C020915D1320937C
:1062B0005E131F910F910895A0DFC0CFA3E1B0E05E
:1062C000E4E6F1E30C944BF08FEF9FEF909389009D
:1062D000809388002AE02983312C212C78948091A6
:1062E000620490916304A0916404B0916504892BC9
:1062F0008A2B8B2B09F0C2C1809168048823D1F0CE
:10630000809166049091670410926804892B91F043
:1063100010926704109266041092590490915F13D2
:1063200080916013981731F0809160138F5F8F70A8
:10633000809360138091660490916704892B09F41F
:106340009DC140915E0450915F0460916004709122
:10635000610480915A0490915B04A0915C04B09117
:106360005D040091500410E030E020E0841B950BA8
:10637000A60BB70B081719072A073B0710F4D9011A
:10638000C8018A8B840F951FA61FB71F80935E04D8
:1063900090935F04A0936004B0936104E1E0C09027
:1063A0002704D0902804E0902904F0902A048091DA
:1063B000370490913804A0913904B0913A04C80E82
:1063C000D91EEA1EFB1EC0923704D0923804E09218
:1063D0003904F0923A04F7FC33C040911F04042EB4
:1063E000000C550B660B770B809175049091760429
:1063F000A0917704B0917804840F951FA61FB71F52
:106400008093750490937604A0937704B0937804F6
:106410008091230490912404A0912504B091260436
:10642000B701A601481B590B6A0B7B0BDB01CA01A4
:106430008093370490933804A0933904B0933A04BE
:1064400000912B0410912C0420912D0430912E04E6
:1064500080913B0490913C04A0913D04B0913E0496
:10646000080F191F2A1F3B1F00933B0410933C0485
:1064700020933D0430933E0437FD33C04091200407
:10648000042E000C550B660B770B809179049091CC
:106490007A04A0917B04B0917C04840F951FA61F01
:1064A000B71F8093790490937A04A0937B04B093F0
:1064B0007C048091230490912404A0912504B09140
:1064C000260428013901481A590A6A0A7B0AD301AD
:1064D000C20180933B0490933C04A0933D04B0938D
:1064E0003E0440912F04509130046091310470912A
:1064F000320480913F0490914004A0914104B091F6
:106500004204480F591F6A1F7B1F40933F0450935A
:106510004004609341047093420477FD33C080903F
:106520002104082C000C9908AA08BB0880917D045E
:1065300090917E04A0917F04B0918004880D991DF4
:10654000AA1DBB1D80937D0490937E04A0937F04BD
:10655000B09380048091230490912404A091250499
:10656000B09126043A014B01681A790A8A0A9B0AFB
:10657000D401C30180933F0490934004A09341044D
:10658000B09342048090330490903404A09035047A
:10659000B09036048091430490914404A091450446
:1065A000B0914604880D991DAA1DBB1D809343041C
:1065B00090934404A0934504B0934604B7FD33C0C0
:1065C00040902204042C000C55086608770880903F
:1065D000810490908204A0908304B0908404840C81
:1065E000951CA61CB71C8092810490928204A092F4
:1065F0008304B09284048090230490902404A0909B
:106600002504B09026042C013D01481859086A0859
:106610007B08530142018092430490924404A0926B
:106620004504B0924604E11104C0E0918400F09169
:106630008500F7FE5F9A37FF469A77FF2B9AB7FFE0
:10664000299AE0918400F0918500E0918400F09116
:106650008500F7FE5F9837FF469877FF2B98B7FFC6
:1066600029985A88552021F08091840090918500C6
:106670002A8921502A8BE0E0211191CE8091620479
:1066800090916304A0916404B0916504892B8A2BD6
:106690008B2B09F0B0C640906604509067045B8A6B
:1066A0004A8A4114510409F402C780915E04909112
:1066B0005F04A0916004B091610440915A0450912C
:1066C0005B0460915C0470915D0484179507A607D4
:1066D000B70708F449C0109267041092660410923C
:1066E000590490915F1380916013981709F4DFC6E5
:1066F000809160138F5F8F7080936013A0EDCA2E1E
:10670000A7E0DA2EE12CF12C8091660490916704C9
:10671000892B09F068C67DDD909367048093660439
:10672000892B09F460C640906604509067045B8A28
:106730004A8AD2018C9183FF08C5C20145960E9406
:10674000BD1910926704109266041092590490913A
:106750005F13809160139817F1F2809160138F5F3F
:106760008F7080936013D7CF409155045091560499
:106770006091570470915804481759076A077B07BE
:1067800008F40FC240915104509152046091530497
:1067900070915404EA89FB8985A996A9A7A9B0AD8F
:1067A000481759076A077B0708F0D0C14115510502
:1067B0006105710509F066C0809092039090930383
:1067C000A0909403B090950383E892E1A1E0FC01CE
:1067D0000591159125913491081519052A053B0558
:1067E00058F4B694A79497948794AA0F0496EFE967
:1067F000F2E1E817F90759F7A0935004F0E28F1679
:106800009104A104B10428F4E0E28E2E912CA12C75
:10681000B12C20E2821A9108A108B108811438E055
:106820009306A104B10408F49AC1A4E09A9EC001A1
:1068300011248D57914FFC01329625913491B82D3A
:10684000EE27B39F8001B29F010D1E1F06940E1FFD
:106850001E1F112430E020E0FC01C590D490F12CE3
:10686000E12CC01AD10AE20AF30A4C0D5D1D6E1D1F
:106870007F1D4093510450935204609353047093CE
:10688000540442CF10E00A81942F852E862FBC81BC
:10689000AD81FE81EF81388529854B80E0918E03A3
:1068A000E99FA12DFF2730918F03399FA00DF11D86
:1068B00010909003199EF00DE89DA00DF11D389DDC
:1068C000F00DE89FF00D4A2EBF2F4A9EE12D332791
:1068D00022274F9EE00D311D211FBA9FE00D311D73
:1068E000211FBF9F300D211D432EB22F4A9E012D27
:1068F000332722274F9E000D311D211FBA9F000D07
:10690000311D211FBF9F300D211D432EB22FEE27B9
:106910009091920380909303809194030090AB0434
:10692000012A09F483C03091A704349DE119910B29
:10693000810A810B2091A804249DE0199109810A04
:10694000810B0091A904049D90198108810B3B9F44
:10695000E0199109810A810B2B9F90198108810B05
:106960000B9F801881094A9E012D332722274F9EB5
:10697000000D311D211FBA9F000D311D211FBF9F2A
:10698000300D211D432EB22F3091A304349DE10D13
:10699000911F811E811F2091A404249DE00D911D53
:1069A000811E811F0091A504049D900D811C811FF3
:1069B0003B9FE00D911D811E811F2B9F900D811C1F
:1069C000811F0B9F800C811D4A9E012D332722279A
:1069D0004F9E000D311D211FBA9F000D311D211F3B
:1069E000BF9F300D211D432EB22F30919F04349D47
:1069F000E119910B810A810B2091A004249DE019DB
:106A00009109810A810B0091A104049D90198108CC
:106A1000810B3B9FE0199109810A810B2B9F9019F3
:106A20008108810B0B9F8018810982C03091A704D7
:106A3000349DE10D911F811E811F2091A804249D8A
:106A4000E00D911D811E811F0091A904049D900DF0
:106A5000811C811F3B9FE00D911D811E811F2B9F7B
:106A6000900D811C811F0B9F800C811D4A9E012D62
:106A7000332722274F9E000D311D211FBA9F000D85
:106A8000311D211FBF9F300D211D432EB22F30918C
:106A9000A304349DE119910B810A810B2091A40478
:106AA000249DE0199109810A810B0091A504049DA0
:106AB00090198108810B3B9FE0199109810A810B94
:106AC0002B9F90198108810B0B9F801881094A9E8A
:106AD000012D332722274F9E000D311D211FBA9F04
:106AE000000D311D211FBF9F300D211D432EB22FE0
:106AF00030919F04349DE10D911F811E811F2091D3
:106B0000A004249DE00D911D811E811F0091A10410
:106B1000049D900D811C811F3B9FE00D911D811EE6
:106B2000811F2B9F900D811C811F0B9F800C811D4D
:106B300011244B820A83BC83AD83FE83EF833887A5
:106B40002987982C892EB12CA82E3ECEAA89BB89E4
:106B5000D1968D909D90AD90BC90D49735CED501B7
:106B6000C401B695A795979587958C7F8D57954FBE
:106B7000FC01C590D490FC01329625913491E82D0A
:106B8000E7708E2EE29FC001E39F900D112433E049
:106B9000969587953A95E1F7C81AD90AF12CE12C18
:106BA00064CE40914C0450914D0460914E0470911C
:106BB0004F04481759076A077B0708F030C28090D6
:106BC000470490904804A0904904B0904A048091F2
:106BD0004B04EA89FB8981117CC0EF5BFF4FE080A9
:106BE000F18002811381EA89FB89E25BFF4F2081FA
:106BF000318142815381AA89BB89D1966D917D9162
:106C00008D919C91D4970E94C619B1E0B0934B042A
:106C1000EA89FB8941A952A963A974A983E892E191
:106C2000A1E0FC01059115912591349104171507F8
:106C30002607370758F47695679557954795AA0F15
:106C40000496EFE9F2E1E817F90759F7A093500429
:106C5000403251056105710520F440E250E060E0EA
:106C600070E040525109610971094115F8E05F0770
:106C70006105710508F4B3C124E0529FC0011124DD
:106C80008D57914FFC01329625913491AA27439F4D
:106C9000F001429FE10DFA1F0694EA1FFA1F11242A
:106CA000AF0170E060E0FC01C590D490F12CE12CC4
:106CB000C41AD50AE60AF70A8C0C9D1CAE1CBF1C30
:106CC0008092470490924804A0924904B0924A04EA
:106CD0001BCD81AD92ADA3ADB4AD88169906AA06C1
:106CE000BB0608F072C181149104A104B10449F4F7
:106CF0004091920350919303609194037091950396
:106D00008DCFA0E0BA85982D492D8A2DFB85EC8585
:106D10007D856E855F853889298950918E03599FBD
:106D2000712D662730918F03399F700D611D109072
:106D30009003199E600D549F700D611D349F600D6E
:106D4000589F600DF72FE62FF79F512D33272227ED
:106D5000F69F500D311D2A1FE79F500D311D2A1F30
:106D6000E69F300D211DF32FE22FF79FB12D332722
:106D70002227F69FB00D311D2A1FE79FB00D311D50
:106D80002A1FE69F300D211DF32FE22F55279091EA
:106D9000920340919303809194030090AB040A2ADC
:106DA00009F483C03091A7043F9F51199A0B4A0BF5
:106DB0008A0B2091A8042F9F501991094A0B8A0B26
:106DC000B091A904BF9F901941098A0B3E9F5019A9
:106DD00091094A0B8A0B2E9F901941098A0BBE9F7D
:106DE00040198109F79FB12D33272227F69FB00D57
:106DF000311D2A1FE79FB00D311D2A1FE69F300D60
:106E0000211DF32FE22F3091A3043F9F510D9A1FB4
:106E10004A1F8A1F2091A4042F9F500D911D4A1FC5
:106E20008A1FB091A504BF9F900D411D8A1F3E9FF0
:106E3000500D911D4A1F8A1F2E9F900D411D8A1FC4
:106E4000BE9F400D811DF79FB12D33272227F69F4E
:106E5000B00D311D2A1FE79FB00D311D2A1FE69F7F
:106E6000300D211DF32FE22F30919F043F9F5119C8
:106E70009A0B4A0B8A0B2091A0042F9F501991095D
:106E80004A0B8A0BB091A104BF9F901941098A0B4C
:106E90003E9F501991094A0B8A0B2E9F9019410968
:106EA0008A0BBE9F4019810982C03091A7043F9F81
:106EB000510D9A1F4A1F8A1F2091A8042F9F500D21
:106EC000911D4A1F8A1FB091A904BF9F900D411DBB
:106ED0008A1F3E9F500D911D4A1F8A1F2E9F900DA5
:106EE000411D8A1FBE9F400D811DF79FB12D332785
:106EF0002227F69FB00D311D2A1FE79FB00D311DCF
:106F00002A1FE69F300D211DF32FE22F3091A3049D
:106F10003F9F51199A0B4A0B8A0B2091A4042F9F73
:106F2000501991094A0B8A0BB091A504BF9F901983
:106F300041098A0B3E9F501991094A0B8A0B2E9FDB
:106F4000901941098A0BBE9F40198109F79FB12D05
:106F500033272227F69FB00D311D2A1FE79FB00D62
:106F6000311D2A1FE69F300D211DF32FE22F309196
:106F70009F043F9F510D9A1F4A1F8A1F2091A00412
:106F80002F9F500D911D4A1F8A1FB091A104BF9FD2
:106F9000900D411D8A1F3E9F500D911D4A1F8A1F53
:106FA0002E9F900D411D8A1FBE9F400D811D1124F3
:106FB000BA87FB87EC877D876E875F87388B298B45
:106FC000542F492F70E0682F29CE2A893B89225BF4
:106FD0003F4FD9014D915D916D917C911FCEDB01A9
:106FE000CA01B695A795979587958C7F8D57954F34
:106FF000FC01C590D490FC013296259134914770E4
:10700000429FC001439F900D1124A3E09695879560
:10701000AA95E1F7C81AD90AF12CE12C4DCE80913E
:107020002E0190912F01A0913001B0913101B7FF55
:1070300061C0EA89FB89EA5BFF4FC080D180E280B2
:10704000F38083E892E121E0FC014591559165913F
:1070500074914C155D056E057F0558F4F694E79420
:10706000D794C794220F04964FE952E14817590765
:1070700059F72093500450E2C516D104E104F104FD
:1070800028F470E2C72ED12CE12CF12C60E2C61A54
:10709000D108E108F108C11478E0D706E104F10451
:1070A00008F431C0A4E0DA9EC00111248D57914F3D
:1070B000FC01329625913491BC2D6627B39FA00127
:1070C000B29F410D561F0694461F561F112470E0B3
:1070D00060E0FC0185919491B0E0A0E0841B950BE9
:1070E000A60BB70B80932E0190932F01A093300134
:1070F000B0933101C0902E01D0902F01E09030016B
:10710000F090310101CBD701C601B695A7959795AF
:1071100087958C7F8D57954FFC0125913491FC010B
:10712000329645915491EC2DE770E49FC001E59FA4
:10713000900D112463E0969587956A95E1F7281BD9
:10714000390BC901B0E0A0E0CDCFEA89FB89858881
:107150009688A788B08C81E081149104A104B104C1
:1071600009F480E0AA89BB895996CD90DD90ED9015
:10717000FC905C97C114D104E104F10409F0826031
:10718000EA89FB89458D568D678D70A141155105A2
:107190006105710509F084608093590410924704D9
:1071A000109248041092490410924A04109251041B
:1071B000109252041092530410925404EA89FB89ED
:1071C00085A196A1A7A1B0A580935A0490935B04D2
:1071D000A0935C04B0935D04442455243201481A02
:1071E000590A6A0A7B0A4092370450923804609226
:1071F000390470923A0440923B0450923C046092ED
:107200003D0470923E0440923F04509240046092CC
:1072100041047092420441A052A063A074A0440CA7
:10722000551C661C771C880C991CAA1CBB1C8092E0
:10723000270490922804A0922904B0922A04CC0C2E
:10724000DD1CEE1CFF1CC0922B04D0922C04E0929B
:107250002D04F0922E04440F551F661F771F409394
:107260002F045093300460933104709332044092A1
:107270003304509234046092350470923604880FBF
:10728000991FAA1FBB1F8093230490932404A093EB
:107290002504B093260410925E0410925F041092AD
:1072A00060041092610481A592A5A3A5B4A5809362
:1072B000550490935604A0935704B093580485A5A1
:1072C00096A5A7A5B0A980934C0490934D04A093D4
:1072D0004E04B0934F04EB5BFF4F80819091E10629
:1072E000891721F08093E1060E94822C0E9483304E
:1072F00044244A94542C320140922E0150922F0182
:107300006092300170923101EA89FB89FD96E0803C
:10731000F18002811381AA89BB89D1962D913D917B
:107320004D915C91D4976D01BAE4CB0ED11CF6015E
:1073300060817181828193810E94C61910924B04F1
:10734000D6014D915D916D917C9183E892E1A1E030
:10735000FC01059115912591349104171507260715
:10736000370758F47695679557954795AA0F049671
:10737000EFE9F2E1E817F90759F7A093500440321A
:1073800051056105710520F440E250E060E070E0D5
:1073900040525109610971094115F8E05F07610523
:1073A000710508F462C024E0529FC00111248D577A
:1073B000914FFC01329625913491AA27439FF00109
:1073C000429FE10DFA1F0694EA1FFA1F1124AF0134
:1073D00070E060E0FC01C590D490F12CE12CC41A5F
:1073E000D50AE60AF70AC0926204D0926304E092DA
:1073F0006404F09265048091620490916304A0910A
:107400006404B0916504AC01BD01009731E0A307AD
:10741000B10520F04FEF5FEF60E070E0841B950B4B
:10742000A60BB70B8093620490936304A09364044B
:10743000B0936504F8948091840090918500409603
:10744000A981A150A983AA2381F1240E351E2816F3
:10745000390610F40C946E31309289002092880025
:1074600078946396E2E10C9467F0DB01CA01B6956B
:10747000A795979587958C7F8D57954FFC01C59063
:10748000D490FC013296259134914770429FC001FF
:10749000439F900D112433E0969587953A95E1F737
:1074A000C81AD90AF12CE12C9ECF1C01D5CF80ED52
:1074B000C82E87E0D82EE12CF12C2DC9CF93DF9375
:1074C00080915F1390916013891B80958F7019F4E0
:1074D0000E94918FF5CF80915F138F5F8F70A09185
:1074E0005F139BE5A99FD0011124FD01E854F84FDB
:1074F000EF0119929A95E9F798E09083A353B84F5A
:1075000090E1E1E6F3E101900D929A95E1F7209187
:107510005F1390916013291303C094E690935C135A
:1075200080935F130E946130DF91CF910895FC0139
:1075300020813181428153816091890D70918A0D42
:1075400080918B0D90918C0D0E94CAE90E94EBF105
:1075500060936D1370936E1380936F1390937013F9
:1075600090915F1380916013981709F0A7CF0E9444
:10757000802D0E94543040916D1350916E13609194
:107580006F13709170134093810450938204609341
:1075900083047093840481110C94613008954F9298
:1075A0005F926F927F928F929F92AF92BF92CF9293
:1075B000DF92EF92FF92CF93DF93EC012091890D40
:1075C00030918A0D40918B0D50918C0D6C857D858D
:1075D0008E859F850E94CAE90E94EBF16B017C01B8
:1075E0002091850D3091860D4091870D5091880D29
:1075F000688579858A859B850E94CAE90E94EBF19E
:107600004B015C012091810D3091820D4091830DE1
:107610005091840D6C817D818E819F810E94CAE989
:107620000E94EBF12B013C0120917D0D30917E0DEC
:1076300040917F0D5091800D688179818A819B8175
:107640000E94CAE90E94EBF1609361137093621388
:107650008093631390936413409265135092661362
:1076600060926713709268138092691390926A1304
:10767000A0926B13B0926C13C0926D13D0926E13E4
:10768000E0926F13F092701390915F1380916013EA
:10769000981781F013DFDF91CF91FF90EF90DF908B
:1076A000CF90BF90AF909F908F907F906F905F90A2
:1076B0004F9008950E94802D0E945430C82F81E67B
:1076C00093E10E94BD19CC2331F30E946130E3CFD6
:1076D000CF92DF92EF92FF92CF93DF93C82F0E9459
:1076E000543094E0C99FE0011124FE01EB58FB4F98
:1076F000C080D180E280F38081110E946130C85542
:10770000D84FC701B6010E946BE9288139814A81AF
:107710005B810E94CAE9DF91CF91FF90EF90DF90EB
:10772000CF9008958F929F92AF92BF92CF92DF92A7
:10773000EF92FF921F93CF93DF93CDB7DEB76097A1
:107740000FB6F894DEBF0FBECDBF182F80E0C0DFAC
:107750004B015C018092FB039092FC03A092FD031D
:10776000B092FE0381E0B4DF6B017C01C092FF03A5
:10777000D0920004E0920104F092020482E0A8DFBB
:1077800060930304709304048093050490930604AB
:107790001D861E861F86188A89829A82AB82BC82C9
:1077A000CD82DE82EF82F88669877A878B879C8715
:1077B00083E08EDF6D877E878F87988BCE01019661
:1077C0000E94A22D1E3FD9F480E1FE013196A5E76B
:1077D000B1E001900D928A95E1F760960FB6F894AA
:1077E000DEBF0FBECDBFDF91CF911F91FF90EF9015
:1077F000DF90CF90BF90AF909F908F90089584E0DE
:10780000189FF0011124DF01AB58BE4F81E090E0DA
:107810008C0F9D1FE80FF91F408151816281738198
:107820004D935D936D937C931397D7CFCF92DF9257
:10783000EF92FF92CF93DF93C82F0E94543094E0D1
:10784000C99FE0011124FE01E759FB4FC080D180A0
:10785000E280F38081110E946130C855D84FC70182
:10786000B6010E946BE9288139814A815B810E94BF
:10787000CAE9DF91CF91FF90EF90DF90CF9008950C
:10788000A1E0B0E0E6E4FCE30C945BF0898360E007
:10789000CE0101960E94181B61E0CE0101960E9464
:1078A000181B62E0CE0101960E94181B8981219667
:1078B000E2E00C9477F0A2E1B0E0E1E6FCE30C94A6
:1078C00057F0DEDF8823C1F1EDB6FEB641E952E0A4
:1078D00082FF02C048E852E021E932E081FF02C0A5
:1078E0002AE832E080FD25C081E992E05F934F9362
:1078F0003F932F939F938F9384E197E09F938F9370
:107900008E010F5F1F4F1F930F930E94FEE80E948E
:10791000038BC8010E948484C8010E9491C50FB6E0
:10792000F894DEBF0FBECDBF81E06296E6E00C9416
:1079300073F08CE892E0DACF80E0F7CFA0E2B0E01D
:10794000E4EAFCE30C944BF080911201882309F4E3
:10795000BEC080910D04082F10E080FF3CC0C09095
:107960001401D0901501E0901601F09017012091BC
:10797000A3023091A4024091A5025091A602C70132
:10798000B6010E94E6F1181644F4C092A302D09208
:10799000A402E092A502F092A602C0902001D0902D
:1079A0002101E0902201F09023012091A302309167
:1079B000A4024091A5025091A602C701B6010E94FF
:1079C00065E987FF08C0C092A302D092A402E092AA
:1079D000A502F092A60201FF3CC0C0901801D09011
:1079E0001901E0901A01F0901B012091A70230913B
:1079F000A8024091A9025091AA02C701B6010E94B3
:107A0000E6F1181644F4C092A702D092A802E092C0
:107A1000A902F092AA02C0902401D0902501E09022
:107A20002601F09027012091A7023091A8024091F1
:107A3000A9025091AA02C701B6010E9465E987FF19
:107A400008C0C092A702D092A802E092A902F092C8
:107A5000AA0202FF3CC0C0901C01D0901D01E09022
:107A60001E01F0901F012091AB023091AC024091B9
:107A7000AD025091AE02C701B6010E94E6F11816A0
:107A800044F4C092AB02D092AC02E092AD02F0920C
:107A9000AE02C0902801D0902901E0902A01F09018
:107AA0002B012091AB023091AC024091AD0250917C
:107AB000AE02C701B6010E9465E987FF08C0C09207
:107AC000AB02D092AC02E092AD02F092AE02809195
:107AD000680D83FD61C02091810130918201409148
:107AE0008301509184016091AF027091B002809146
:107AF000B1029091B2020E9465E9882309F44CC05A
:107B00000E94E4B6182F882331F00E94038B89EF7E
:107B100096E00E94938420918101309182014091EE
:107B20008301509184016091AF027091B002809105
:107B3000B1029091B2020E9482F09F7720916F0172
:107B40003091700140917101509172010E94CAE917
:107B500020E030E046E154E40E94E6F11816D4F447
:107B60000E94038B8AED96E00E9493848091AF027D
:107B70009091B002A091B102B091B20280938101C4
:107B800090938201A0938301B09384018FEA92E0E5
:107B9000CEDC02C01111EACF2AE037ED43E25CE30C
:107BA00060910C0170910D0180910E0190910F0177
:107BB0000E94CAE96B017C01609110017091110172
:107BC000072E000C880B990B0E946BE99B01AC01FE
:107BD000C701B6010E94CAE9698B7A8B8B8B9C8B9B
:107BE0008091B302882309F18090B4029090B5028D
:107BF000A090B602B090B702C090AB02D090AC0299
:107C0000E090AD02F090AE0220E030E0A901C501A5
:107C1000B4010E9465E98823F9F0A7019601C50126
:107C2000B4010E94E6F11816BCF020E030E0A90192
:107C3000BE016F5E7F4F83EA92E00E94ADC780E194
:107C4000E3EAF2E0A5E7B1E001900D928A95E1F751
:107C5000A096E2E10C9467F02091750130917601D5
:107C600040917701509178016091A3027091A40234
:107C70008091A5029091A6020E9482F04B015C01C6
:107C80002091790130917A0140917B0150917C01E2
:107C90006091A7027091A8028091A9029091AA0216
:107CA0000E9482F06D8B7E8B8F8B988F20917D014F
:107CB00030917E0140917F0150918001C701B60152
:107CC0000E9482F06D8F7E8F8F8F98A3209181010B
:107CD0003091820140918301509184016091AF0203
:107CE0007091B0028091B1029091B2020E9482F034
:107CF000698F7A8F8B8F9C8F20E030E0A901C501BE
:107D0000B4010E9465E981110CC020E030E0A901B6
:107D10006D897E898F89988D0E9465E9882309F491
:107D200084CFA5019401C501B4010E94CAE96B0189
:107D30007C012D893E894F89588DCA01B9010E9465
:107D4000CAE99B01AC01C701B6010E9483F06B0137
:107D50007C012D8D3E8D4F8D58A1CA01B9010E9425
:107D6000CAE99B01AC01C701B6010E9483F06B0117
:107D70007C01298D3A8D4B8D5C8DCA01B9010E9421
:107D8000CAE99B01AC01C701B6010E9483F06B01F7
:107D90007C010E941FF22B013C012CEC3CEB4CE8D7
:107DA0005BE2C701B6010E9465E987FF06C0498C06
:107DB0005A8C6B8C7C8CE89477F82DEB37E346E893
:107DC00055E3C301B2010E9465E987FD38CF2DEC70
:107DD0003CEC4CE45EE3C301B2010E94CAE90E949C
:107DE00067F11B01672B19F422242394312CB10174
:107DF00090E080E00E9469E99B01AC0160E070E0E6
:107E000080E89FE30E94FAF06B017C01AC019B01CA
:107E1000C301B2010E94CAE92B013C01A7019601EE
:107E2000C501B4010E94CAE94B015C01A70196019A
:107E30006D897E898F89988D0E94CAE96D8B7E8BB2
:107E40008F8B988FA70196016D8D7E8D8F8D98A158
:107E50000E94CAE96D8F7E8F8F8F98A3A70196012C
:107E6000698D7A8D8B8D9C8D0E94CAE9698F7A8F7E
:107E70008B8F9C8F80E1E5E7F1E08E010F5F1F4F54
:107E8000D80101900D928A95E1F70E94D6D16B013D
:107E90007C0128ECC20ED11CE11CF11C81E0281AE7
:107EA000310809F454C00E94D6D19B01AC012C19B1
:107EB0003D094E095F0957FD4DC06B017C0128EC5F
:107EC000C20ED11CE11CF11C80E00E94918FA50123
:107ED000940169817A818B819C810E9483F06983FE
:107EE0007A838B839C832D893E894F89588D6D8140
:107EF0007E818F8198850E9483F06D837E838F833E
:107F000098872D8D3E8D4F8D58A169857A858B85FB
:107F10009C850E9483F069877A878B879C87298D4F
:107F20003A8D4B8D5C8D6D857E858F8598890E94FD
:107F300083F06D877E878F87988BA3019201BE01A6
:107F40006F5E7F4FC8010E94ADC78111A7CFA3010B
:107F500092016ECE0E94C22ABACF809109049091FC
:107F60000A04A0910B04B0910C0480930C0190932F
:107F70000D01A0930E01B0930F0180910704909121
:107F800008049093110180931001089580910C01D1
:107F900090910D01A0910E01B0910F018093090401
:107FA00090930A04A0930B04B0930C0480911001E9
:107FB00090911101909308048093070484E690E067
:107FC00090931101809310010895ACE0B0E0EBEEC6
:107FD000FFE30C944DF02B013C0129873A874B8736
:107FE0005C8747015801D601CD90DD90ED90FC9063
:107FF00020E030E0A901C701B6010E9465E98111C6
:1080000071C080916B0190916C01A0916D01B09154
:108010006E0189839A83AB83BC8320E030E0A901A1
:10802000C701B6010E9465E9811106C0C12CD12C9F
:1080300080E8E82E80E4F82ECD82DE82EF82F8869A
:10804000A501940160917D0170917E0180917F0175
:10805000909180010E9465E987FF0CC080927D01AC
:1080600090927E01A0927F01B0928001CE01059690
:108070000E945E22409275015092760160927701D3
:108080007092780189859A85AB85BC85809379014A
:1080900090937A01A0937B01B0937C01CE0101966D
:1080A0000E945E22A501940160917D0170917E0184
:1080B00080917F01909180010E94E6F1181664F48E
:1080C00080927D0190927E01A0927F01B09280010A
:1080D000CE0105960E945E220E94802D2C96E0E142
:1080E0000C9469F0D701C60194CFCF92DF92EF9242
:1080F000FF920F931F936B01FC01E080F1800281DE
:108100001381E5E7F1E02481358146815781608163
:1081100071818281938159DF1F910F91FF90EF90C0
:10812000DF90CF9008950C94D0C70F931F93CF93F7
:10813000DF93EC018B010E945B8E882331F081E09C
:10814000DF91CF911F910F910895B801CE01CDDF3E
:1081500080912607C82FC87083FD0AC01092260799
:1081600082E0E0DAE0DF81E0CC2351F380E0E8CF89
:108170000E941A8E882391F3E2CFCF930E9454304D
:10818000C82F8091601380935F1380935E13809358
:108190005D1384E680935C130E94FD3080ED93E0D4
:1081A0009093B20D8093B10DC1110E94613081E0B6
:1081B000809368040E94802D8EEFB4DAB4DFCF91F3
:1081C0000895ACE0B0E0E7EEF0E40C945BF00E94C0
:1081D000A3B60E9454309CE0E5E7F4E0DE0111967E
:1081E00001900D929A95E1F781110E946130CE01C4
:1081F00001960E94FA2B2C96E2E00C9477F0B0E006
:10820000A0E0E5E0F1E40C944DF040907501509051
:10821000760160907701709078018090790190905C
:108220007A01A0907B01B0907C01C0907D01D0903C
:108230007E01E0907F01F09080010E94142D6091FA
:108240002C0170912D01072E000C880B990B0E94B8
:108250006BE92AE037ED43E25CE30E94CAE96093F0
:108260006F0170937001809371019093720104E12A
:1082700011E0D0E0C0E0CE01895C954F0E94B57757
:10828000F80161937193819391938F01CE01855D84
:10829000954F0E94B577F801608771878287938731
:1082A0002496CC30D10539F760E08BE194E00E9450
:1082B000967A0E94637B0E94582DA30192016091DF
:1082C00075017091760180917701909178010E94FB
:1082D00065E981111BC0A50194016091790170913C
:1082E0007A0180917B0190917C010E9465E9811166
:1082F0000DC020917D0130917E0140917F01509110
:108300008001C701B6010E9465E981115ADFCDB72E
:10831000DEB7E0E10C9469F0A4E0B0E0E2E9F1E45A
:108320000C945BF084EF91E0A0E0B0E089839A8345
:10833000AB83BC83BE016F5F7F4F8CE30E943983A8
:1083400080EC96E00E94938486B16AEB76E082FB33
:10835000882780F90E94B82186B164EB76E083FB20
:10836000882780F90E94B82186B16EEA76E082956E
:1083700081700E94B82180B166EA76E082FB88278E
:1083800080F90E94B821029907C00E946E8324964A
:10839000E2E00C9477F006C00E9457832496E2E056
:1083A0000C9477F08091E006811103C08091E20681
:1083B00081110C9483300895ACE0B0E0E2EEF1E47A
:1083C0000C945BF0A9E6BDE090E080E0FC01ED5884
:1083D000F54F45915591659174914D935D936D93D2
:1083E0007D93FC01ED59F54F45915591659174913F
:1083F00050964D935D936D937C935397FC01ED5A8A
:10840000F54F459155916591749190964D935D937B
:108410006D937C939397049680319105B9F680E231
:108420009EE4A0E0B0E08093790D90937A0DA09344
:108430007B0DB0937C0D80E090E0AAEFB3E48093D5
:108440009D0D90939E0DA0939F0DB093A00D8093D2
:10845000A10D9093A20DA093A30DB093A40D8093B2
:10846000A50D9093A60DA093A70DB093A80D109203
:10847000A90D1092AA0D1092AB0D1092AC0D109296
:10848000AD0D1092AE0D1092AF0D1092B00D8AE0AE
:1084900097EDA3EABDE380938B0790938C07A0939D
:1084A0008D07B0938E0780E090E0A0E2B1E4809366
:1084B0001B0490931C04A0931D04B0931E040E94FF
:1084C0004C7A8CE0E5E8F1E0DE01119601900D9226
:1084D0008A95E1F789819A81AB81BC8180934E13A3
:1084E00090934F13A0935013B09351138D819E819D
:1084F000AF81B8858093521390935313A093541374
:10850000B093551389859A85AB85BC8580935613A6
:1085100090935713A0935813B09359138EEB90E098
:1085200090934407809343078CE390E09093460731
:1085300080934507109248071092470786EE90E017
:1085400090934A078093490786E490E090934C0704
:1085500080934B0710924E0710924D078FE892ECD4
:10856000ADE8B1E48093B5129093B612A093B71220
:10857000B093B8128CE998EFA5E4BEE38093B912EA
:108580009093BA12A093BB12B093BC1281E49CEBFF
:10859000ABECB3E48093BD129093BE12A093BF12D4
:1085A000B093C01280E090E0AFEAB3E48093370765
:1085B00090933807A0933907B0933A0785E996E27C
:1085C000A5E2B1E480933B0790933C07A0933D075D
:1085D000B0933E0780EA9CE6ACE2B5E480933F07A7
:1085E00090934007A0934107B09342071092E00692
:1085F0001092DF06D7DE03DE2C96E2E00C9477F0D3
:10860000DBCEA4E0B0E0E7E0F3E40C944CF0909112
:10861000E206981709F455C0382E80E090E0A0E2F9
:10862000B1E489839A83AB83BC83C0905613D09006
:108630005713E0905813F090591320E030E0A9014F
:10864000C701B6010E9465E987FF0CC0A70196012A
:1086500060E070E080E291E40E9482F069837A83B6
:108660008B839C83CE0101960E9461C84090750166
:108670005090760160907701709078018090790138
:1086800090907A01A0907B01B0907C013320F1F0B2
:108690000E945B8E19821A821B821C82E0907D01EF
:1086A000F0907E0100917F0110918001CE01019632
:1086B0006C01A5019401C301B20187DC3092E2068E
:1086C00071DE80E02496E1E10C9468F00E941A8E3D
:1086D000E1CFB0E0A0E0EFE6F3E40C944DF0C82F5A
:1086E000E82EF12CF701E057F24DD491823071F46D
:1086F00081E087DF811105C00E945B8E882309F429
:10870000E2C0CDB7DEB7E0E10C9469F06D2FDD0F6C
:10871000770B880B990B0E946BE92B013C01C70179
:10872000880F991F880F991F8D59984F0E94B57710
:108730004B015C01A3019201C501B4010E94CAE989
:108740004B015C016701CC0CDD1CCC0CDD1CC601AF
:10875000895A984F0E94B577A30192010E94CAE9F5
:1087600020E030E040EC5FE30E94CAE9AB01BC01CD
:1087700000E010E098018C2F0E9497CBC23009F0E6
:10878000CCC00E941A8E20E030E0A901C501B401DE
:108790000E9465E9882329F100E010E020E830E438
:1087A000B501A40170588C2F0E9497CBC23009F4F8
:1087B00067C0A5019401C501B4010E9483F04B017B
:1087C0005C01C23009F062C000E010E020E030E45B
:1087D000B501A4018C2F0E9497CBC23011F40E94E6
:1087E0001A8E81E090E00C2E01C0880F0A94EAF7FF
:1087F00090917707982B9093770790910D04892B90
:1088000080930D04C601855B984F0E94B577F601F1
:10881000EB58FE4F6083718382839383C230D1F41F
:10882000209156133091571340915813509159137A
:1088300060917D0170917E0180917F019091800116
:108840000E9482F060937D0170937E0180937F018E
:108850009093800168DCF601ED55FD4FD601AB58D1
:10886000BE4F8D919D910D90BC91A02D80839183E1
:10887000A283B383C23009F044CF80E0C2DE41CF8F
:108880000E945B8E882309F494CF3BCFF701E85B0D
:10889000F84F6491611107C00E94038B86E297E054
:1088A0000E9493846AE070E090E080E00E9469E9B1
:1088B0009B01AC0161E070E088E492E40E94FAF070
:1088C0008B019C0185CF8BE697E00E94B57720E075
:1088D00030E0A9010E9465E9882309F417CF6D2FC4
:1088E000DD0F770B880B990B0E946BE92B013C0184
:1088F0008BE697E00E94B5774B015C0120E030E009
:1089000040EA50E40E94E6F187FF14CF812C912CBD
:1089100090EAA92E90E4B92E0DCF20E030E0A90115
:10892000C501B4010E9465E9882309F45ACF00E02B
:1089300010E0980135CF80912607882319F0109216
:108940002607089540E070E060E086E896E00E9427
:10895000A28E1F920F920FB60F9211240BB60F9298
:108960002F933F934F935F936F937F938F939F9337
:10897000AF93BF93EF93FF930E948330FF91EF91EA
:10898000BF91AF919F918F917F916F915F914F9127
:108990003F912F910F900BBE0F900FBE0F901F9025
:1089A00018950F931F9380918707813019F50E94C6
:1089B000D6D10091F2031091F3032091F40330918A
:1089C000F503601B710B820B930B28EE33E040E044
:1089D00050E00E9493EF6091EE037091EF0380915D
:1089E000F0039091F103620F731F841F951F1F9175
:1089F0000F9108956091F6037091F7038091F80349
:108A00009091F903D6CF109287071092F20310923B
:108A1000F3031092F4031092F5031092F6031092F0
:108A2000F7031092F8031092F9031092EE031092DC
:108A3000EF031092F0031092F103089580918707DD
:108A40008130E1F08230C1F4ACDF6093EE037093CB
:108A5000EF038093F0039093F10381E08093870705
:108A60000E94D6D16093F2037093F3038093F403D2
:108A70009093F50381E00895C6DFEFCF80E008957D
:108A80000E94AFC80E94FD7B882351F08091C914D9
:108A900082FD06C087EE91E09093E5068093E406A0
:108AA000CDCF80918707813079F482E0809387076A
:108AB0000E94D6D16093F6037093F7038093F80376
:108AC0009093F90381E0089580E0089580918707ED
:108AD0008150823070F4109287070E94D6D1609343
:108AE000F6037093F7038093F8039093F90381E002
:108AF000089580E008952091B2123091B312263586
:108B000031053CF42091340730913507263031058A
:108B10001CF0882331F092CF662319F0D7DF0C9434
:108B2000AFC808959C0197FF26C0EE27FF27E81BDA
:108B3000F90B2D398FEF38070CF05DC08DE2809373
:108B40009E02CF0164E670E00E941DF0CB012AE096
:108B500030E0B9010E941DF0805D80939F02CF013B
:108B6000B9010E941DF0CB01B9010E941DF0805D8A
:108B70008093A0022AC0283E83E03807B4F1C901DF
:108B800068EE73E00E941DF0CB01EAE0F0E0BF0167
:108B90000E941DF0805D80939E02C90164E670E032
:108BA0000E941DF0CB01BF010E941DF0805D8093EB
:108BB0009F02C901BF010E941DF0CB01BF010E94AD
:108BC0001DF0805D8093A002F901CF016AE070E0A2
:108BD0000E941DF0805D8093A1028EE992E00895CD
:108BE0008DE237FDC5CF80E2C3CFF90180E22436A4
:108BF00031050CF0A4CF80E280939E0280939F0207
:108C0000EA30F1056CF38DE237FF80E280939F023A
:108C1000CF016AE070E00E941DF0605D6093A002E9
:108C2000D4CF9C0197FD2DC080E2243631055CF045
:108C3000C90164E670E00E941DF0CB016AE070E0BB
:108C40000E941DF0805D80939F0280E22A303105F2
:108C50005CF0EAE0F0E0C901BF010E941DF0CB0129
:108C6000BF010E941DF0805D8093A002C9016AE0EF
:108C700070E00E941DF0805D8093A1028FE992E078
:108C800008953195219531098DE2DDCFCF92DF92A4
:108C9000EF92FF92FC01C080D180E280F38020E05F
:108CA00030E0A901C701B6010E9465E987FD26C031
:108CB0006DEB77E386E095E3A70196010E9483F0D0
:108CC0006B017C0120E030E0A9010E9465E920E011
:108CD00030E040E05FE387FF04C020E030E040E0A8
:108CE0005FEBC701B6010E9483F00E9462F1CB01E5
:108CF00098DFFF90EF90DF90CF9008956DEB77E3D2
:108D000086E095EBD9CFA4E0B0E0E9E8F6E40C9476
:108D10005BF00E946BE969837A838B839C83CE012D
:108D20000196B4DF2496E2E00C9477F0FC016081B8
:108D30007181828193810E9462F1CB0172CFA4E0A4
:108D4000B0E0E5EAF6E40C945BF00E946BE969831D
:108D50007A838B839C83CE010196E8DF2496E2E040
:108D60000C9477F08F929F92AF92BF92EF92FF9206
:108D70000F931F93CF93DF93EC018B01E42EF22E20
:108D800080917113909172138C179D07C9F123E69E
:108D9000CF38D20709F03FC08B509C4771F40E9436
:108DA000D6D16E517B4F8F4F9F4F6093DE037093F0
:108DB000DF038093E0039093E103D0937213C09399
:108DC000711330E020E000936A0710936B07209343
:108DD0006C0730936D07E0926507F0926607CB5001
:108DE000DC4721F410929A021092DD0382E0809316
:108DF0006A0181E080936707109299021092E9035B
:108E0000DF91CF911F910F91FF90EF90BF90AF90A6
:108E10009F908F9008952CE7CB30D20771F68F5832
:108E20009346D9F40E94D6D18090DE039090DF0360
:108E3000A090E003B090E103681979098A099B09C1
:108E400097FF0BC0809177078770873031F40E94BD
:108E50003523C1E6D8E58111B0CFCBE0DCE7ADCF5B
:108E600020E040E070E060E084E293E27BCF0E948B
:108E7000E4B6882339F020E040E070E060E083E869
:108E800097E570CFEDCF21E020939A02FC0180811D
:108E90009181A281B3818093080190930901A093ED
:108EA0000A01B0930B0120E040E070E060E08091A7
:108EB00054079091550756CFA4E0B0E0E2E6F7E4FE
:108EC0000C945BF08DEC9CECACECBCE389839A8356
:108ED000AB83BC83CE010196D6DF2496E2E00C94EE
:108EE00077F0A4E0B0E0E7E7F7E40C945BF08DECFA
:108EF0009CECACECBDE389839A83AB83BC83CE014D
:108F00000196C1DF2496E2E00C9477F0A4E0B0E093
:108F1000ECE8F7E40C945BF080E090E0A0E8BFE3BD
:108F200089839A83AB83BC83CE010196ACDF249600
:108F3000E2E00C9477F0A4E0B0E0E1EAF7E40C940E
:108F40005BF080E090E0A0E2B1E489839A83AB8398
:108F5000BC83CE01019697DF2496E2E00C9477F073
:108F600081E080939A02809177078770873051F073
:108F70001092770710920D0480EF95E09093E5062C
:108F80008093E4068091B3028093EB0380E00E941B
:108F90000A7A20E040E070E060E080ED97E4E2CE05
:108FA00080916A01882331F041E062EA73E082E057
:108FB0000E9444CC80910D048770873071F4109228
:108FC000EA0320E040E070E060E083E098E5CADE7C
:108FD00081E08093E9030C946622089520E040E04C
:108FE00070E060E08BE09CE7BDCE1092A7070E9486
:108FF000E228F4CFB0E0A0E0E0E0F8E40C9455F013
:10900000CDB6DEB6EAE7F7E0DF010D900020E9F724
:10901000CD01825797402DB73EB7281B390B0FB6AD
:10902000F8943EBF0FBE2DBF0DB71EB70F5F1F4F89
:10903000FF93EF9383E595E09F938F931F930F9397
:109040000E94FEE8780134E0E30EF11C0F900F90CF
:109050000F900F900F900F90D7018D917D01882375
:1090600049F0082E000C990B0E9464F2F701319729
:109070008083F2CF6EE475E0C8010E9497E84FE369
:1090800050E0B80186EE96E00E94BCF20FB6F8946C
:10909000DEBE0FBECDBEA2DF0E94AFC8E8E00C94DA
:1090A00071F08093280720E040E070E060E081E20A
:1090B00098E558CEA2E8B0E0E0E6F8E40C944BF076
:1090C000ADB6BEB684E690E090939E1280939D125A
:1090D0001092C2121092C11241E064E070E0CE0121
:1090E00087589F4F0E94EBB543E050E0BE016758A0
:1090F0007F4F86E292E00E94AEF2892BF9F0ED9666
:109100008FADED97882339F08FE3EA968FAFEA971A
:10911000EB961FAEEB9782E0C4DF81E080931A04E8
:1091200090911A0481E089270FB6F894BEBE0FBE55
:10913000ADBECE57DF4FE2E10C9467F041E062E054
:1091400070E0CE0183589F4F0E94EBB5E9961CAEAC
:109150001DAE1EAE1FAEE9971092C2121092C11240
:10916000CE018F579F4F0E943422EDB6FEB6CF57E7
:10917000DF4FC880C158D040D12C23E0C20ED11C93
:10918000CC0CDD1CCC0CDD1C8DB79EB78C199D0959
:109190000FB6F8949EBF0FBE8DBFEDB7FEB73196E8
:1091A0003F018C199D090FB6F8949EBF0FBE8DBF6D
:1091B000EDB7FEB731964F018C199D090FB6F894A3
:1091C0009EBF0FBE8DBF0DB71EB70F5F1F4FB601FD
:1091D000C3010E94392240918C0381E0482764E05A
:1091E00070E089E79DE00E94EBB5B601C4010E94E2
:1091F0003922B601C8010E94392290918C03CE57C2
:10920000DF4F9883C258D04091114BC0CF57DF4FEA
:109210008881C158D04090E00296A9E6BDE050E0B8
:1092200040E030E020E06FE77AE0EFE6CE2EEAE0C3
:10923000DE2E821793070CF495C0F301E40FF51F9F
:1092400020803180428053802D923D924D925D92DC
:10925000821793070CF48CC0F401E40FF51F2080F3
:1092600031804280538050962D923D924D925C9277
:109270005397821793070CF481C0F801E40FF51F90
:10928000208031804280538090962D923D924D9265
:109290005C9293972F5F3F4F4C5F5F4F24303105B7
:1092A00041F68DE99DE00E940C2281EA9DE00E943A
:1092B0000C2285EA9DE00E940C2289EA9DE00E9432
:1092C0000C228DEA9DE00E940C22CE018B589F4F0C
:1092D0000E940C22CE018B589F4F0E940C22CE017F
:1092E0008B589F4F0E940C22CE018B589F4F0E949B
:1092F0000C228BE897E00E940C220FB6F894FEBE79
:109300000FBEEDBE8E010F5F1F4FC8010E942C22C1
:10931000CE0183599F4F0E941422C8010E940C2243
:109320008BE194E00E940C22CE018B589F4F0E944B
:109330000C22CE0183599F4F0E943422C8010E9403
:109340003422AE96CFACAE978981C89E60011124BD
:10935000E1E0CE1AD108C8F0CE018B589F4F0E9491
:109360000C22F6CFFB0125903590459054906CCFA0
:10937000F601259035904590549075CFEFE5FAE0D1
:1093800025903590459054907FCF8EE493E10E94D4
:109390002C228AE0D82EDA94CE01DD2029F08B58D9
:1093A0009F4F0E940C22F7CF80589F4F0E9434227B
:1093B000CE0181589F4F0E943422C058DF4F8881D0
:1093C000C058D040873009F05EC1C158DF4F888156
:1093D000CF57D040873009F056C1CE57DF4F288194
:1093E000C258D040211103C080E00E940A7A84E86C
:1093F00093E00E9424228CE793E00E942422409173
:109400008C0381E0482764EC70E088EB92E00E94D6
:10941000EBB5C8010E941C22CE0183599F4F0E94C8
:10942000142240918C03FF24F3944F2564E070E0F4
:10943000C8010E94EBB583EE96E00E941C22409189
:109440008C034F256CE070E083E497E00E94EBB55D
:1094500040918C034F2564E170E0C8010E94EBB598
:10946000F0908C03F11030C089819A81AB81BC816E
:109470008093B5129093B612A093B712B093B8121E
:109480002CEA35EC47E25EE36D817E818F81988521
:109490000E94CAE96093B9127093BA128093BB120A
:1094A0009093BC1220E030E543EC50E469857A8566
:1094B0008B859C850E94CAE96093BD127093BE1291
:1094C0008093BF129093C01241E04F2562E070E09C
:1094D000C8010E94EBB5C8010E940422D0908C0301
:1094E000D11030C089819A81AB81BC8180933707CC
:1094F00090933807A0933907B0933A072CEA35ECDC
:1095000047E25EE36D817E818F8198850E94CAE982
:1095100060933B0770933C0780933D0790933E0711
:1095200020E030E543EC50E469857A858B859C85A5
:109530000E94CAE960933F077093400780934107F8
:1095400090934207C8010E940422C8010E9414227D
:10955000C8010E941422C8010E94142285E0F8016B
:1095600011928A95E9F7FF24F3944D2D4F2565E07C
:1095700070E0C8010E94EBB5C8010E941C22409116
:109580008C034F2560E270E0C8010E94EBB5CE016C
:1095900083599F4F0E941C2240918C034F2569E004
:1095A00070E0C8010E94EBB540918C034F2562E149
:1095B00070E0C8010E94EBB540918C034F2564E236
:1095C00070E0C8010E94EBB540918C034F2560E12B
:1095D00070E0C8010E94EBB540918C034F2569E013
:1095E00070E0C8010E94EBB5C8010E940C224091B6
:1095F0008C034F256CE070E0C8010E94EBB54091F0
:109600008C034F256CE670E0C8010E94EBB519820F
:109610001A821B821C821D821E821F821886198656
:109620001A861B861C86C8010E94042240918C0366
:109630004F2568E070E0C8010E94EBB5C8010E94A8
:109640002C22CE0181589F4F0E941422CE018359B3
:109650009F4F0E940C2280919D1290919E12803704
:10966000934089F510921A042091C1123091C212D0
:10967000EF968EAD9FADEF972817390741F1F09225
:109680001A0480E023C0CE0183599F4F0E942422F8
:10969000C8010E942422C058DF4FC880C058D04063
:1096A000C158DF4F8881CF57D040C89E6001112438
:1096B00081E0C81AD10808F4ACCECE018B589F4F78
:1096C0000E940C22F5CFF0921A0481E0EADC80912E
:1096D0008C03811125CD80911A04811121CD0E9426
:1096E000FF401ECD81E080938C03E4DC10928C035C
:1096F000882309F0DFCC0E94DC4180E00895F2CF9E
:10970000CF93DF93C091DD03CC23B1F0C150C09360
:10971000DD0389E0C89FE0011124C955DC4F6A814F
:109720007B812F814E81888199811CDB8885809384
:109730009A02DF91CF91089551DCFBCFA4E0B0E015
:10974000E4EAFBE40C944EF00E9458CDF0906507DB
:109750006F2C85E0782E7F0C86E0E82EEF1885E0F0
:10976000D82EDF18AA24AA94B12C84E0C82ECF18D2
:1097700082E0982E9F1881E0882E8F185F2C5194DC
:10978000F1105AC080916807882309F444C0809181
:109790006A01882359F081E090916807911180E077
:1097A00024E041E856E0652D0E94A4CC8091A707F3
:1097B0008093280724E0F212F7C01092740780917A
:1097C0006807843009F4DDC080916A018823E1F0E4
:1097D00011E080916807843009F010E0809128073B
:1097E00024E6829FC001112481589F4FB5010E9439
:1097F0001DF0862F0E94EB1C00E09C0146E656E01F
:109800006C2D812F0E94B375F394F710B9CF87E0C8
:10981000809366070DC080914F0710924F078823F1
:1098200009F4B5CF6DDF80916707882309F4AFCFC6
:109830002496EFE00C946AF021E0F21243C080918C
:109840006807813041F180916A018823F9F011E0C5
:1098500080916807813009F010E0609110017091EB
:109860001101072E000C880B990B0E946BE969838C
:109870007A838B839C83CE01019658DA00E09C01A9
:109880004BE756E0682D812F0E94B3758091A707A2
:1098900080932807B9CF80914F0710924F078823F4
:1098A00091F210E000E027EE33E04AE050E060E1A2
:1098B00071E08BE796E00E941DCE809167078823B8
:1098C00011F2B6CF82E0F812D7C0809168078230DB
:1098D00021F180916A018823C9F211E08091680723
:1098E000823009F010E06091B2127091B312072E2D
:1098F000000C880B990B0E946BE969837A838B8338
:109900009C83CE01019612DA00E09C0144E756E008
:10991000692D812F0E94B37549CF80914F07109216
:109920004F078823B1F20E944CCD02E012E225EFEE
:1099300030E050E040E062EB72E184E796E00E94A4
:109940001DCE80916707882321F272CF80914F0747
:1099500010924F07882309F497C00E944CCD05E868
:109960001AE623E730E050E040E064E377E080E788
:1099700096E00E941DCE80916707882309F484C079
:1099800057CF80914F0710924F07882309F41CCFBF
:109990000E944CCD86E696E00E9492D080916707A7
:1099A000882309F411CF44CF85E0F8123DC080919F
:1099B0006807853011F180916A01882309F424CF6A
:1099C00011E080916807853009F010E060912C016A
:1099D00070912D01072E000C880B990B0E946BE9EA
:1099E00069837A838B839C83CE0101969FD900E0A3
:1099F0009C0141E656E06D2D04CF80914F071092F7
:109A00004F078823C1F20CE01DE127EE33E04AE066
:109A100050E06CE271E081E696E00E941DCE8091FC
:109A20006707882341F204CF26E0F212EDCE809141
:109A30006807863091F080916A01882309F4E4CEAA
:109A400081E090916807963009F080E023E042E5DC
:109A500056E06E2D0E94A4CCD7CE80914F07109275
:109A60004F07882341F381E698E50E94AECD8091AF
:109A70006707882301F3DCCE83E0F81297CE80914C
:109A80006807833009F462CF80916A01882309F462
:109A9000FDCE11E080916807833009F010E06091FD
:109AA000340770913507072E000C880B990B0E9424
:109AB0006BE969837A838B839C83CE01019636D9C7
:109AC00063E0661900E09C0140E756E022CFA4E085
:109AD000B0E0EDE6FDE40C944CF0EE24E3948091CC
:109AE000B2129091B312892B09F4E12C0E9458CD47
:109AF000F09065074F2C95E0592E5F0C88248A94CE
:109B0000912C83E0B82EBF1882E0A82EAF1881E018
:109B1000782E7F183F2C319486E0682E6F18F11054
:109B200015C080916807882309F4D7C080916A0125
:109B3000882309F475C181E090916807911180E054
:109B400024E04DE456E0632D0E94A4CC8091B21233
:109B50009091B312909329078093280721E0F21285
:109B6000E8C080916807813009F4C8C080916A011B
:109B7000882309F44DC011E080916807813009F015
:109B800010E06091280770912907072E000C880BC0
:109B9000990B0E946BE969837A838B839C83CE0146
:109BA0000196C4D800E09C0146E456E0672D812F61
:109BB0000E94B3758091A7078093280793E0F9125C
:109BC00027C01092740780916807833009F4F4C0AD
:109BD00080916A018823E1F011E080916807833069
:109BE00009F010E08091280724E6829FC00111242B
:109BF00081589F4FB4010E941DF0862F0E94EB1CDC
:109C000000E09C0148E356E06B2D812F0E94B37564
:109C1000D12CC12C14E00F2D0419C0922807F11289
:109C20001FC0F601EE0FFF1FEF5DF94F8591949174
:109C30009093760780937507809168078F1509F4D4
:109C4000CEC080916A01882359F081E09091680725
:109C5000911380E023E04EE256E0602F0E94A4CCF6
:109C6000812F9FEFC91AD90A15E08530B1F680918E
:109C7000340790913507892B19F4EE2009F4CEC0F2
:109C800026E0F21221C080916807863009F4B8C03E
:109C900080916A018823C1F085EF97E49F938F93A9
:109CA00085E296E09F938F936F9281E09091680791
:109CB000963009F080E08F930E94F0220F900F9071
:109CC0000F900F900F900F9087E0EE24E394F394A1
:109CD000F51025CF809366070DC080914F07109235
:109CE0004F07882309F422CF0BDD80916707882373
:109CF00009F41CCF2496E1E10C9468F080914F07A1
:109D000010924F07882309F431CF0E944CCD00E018
:109D100013E225EF30E050E040E068E277E086E4CF
:109D200096E00E941DCE80916707882309F41ECF1C
:109D3000E1CF82E0F8123ECF80916807823019F1BE
:109D400080916A01882309F463CF11E0809168074C
:109D5000823009F010E06091340770913507072ECA
:109D6000000C880B990B0E946BE969837A838B83C3
:109D70009C83CE0101960E94964600E09C0142E43D
:109D800056E06A2D14CF80914F0710924F07882319
:109D9000B9F20E944CCD05E81AE623E730E050E026
:109DA00040E064E377E082E496E00E941DCE80917B
:109DB0006707882329F29ECF80914F0710924F07A3
:109DC000882309F405CF0E944CCD88E396E00E94D9
:109DD00092D080916707882309F4FACE8BCF8091C7
:109DE0004F0710924F07882309F42BCF89E19FE496
:109DF0000E94AECD80916707882309F422CF7ACFE5
:109E000080914F0710924F07882309F441CFEDD876
:109E100080916707882309F43BCF6CCF86E057CF4A
:109E20008091B2129091B3129093290780932807E2
:109E3000C1CEB0E0A0E0EFE1FFE40C944DF0009162
:109E400028070E9458CDC091650710E0000F111F30
:109E50000F5D194F95E0592E5C0E29EFE22E25E09B
:109E6000F22ED3E0DC1B30E1C32E33E2D32E47E0E9
:109E7000A42E46E0B42E82E0782E7C1A5EE2852E77
:109E800056E0952E81E0682E6C1A4C2E4194C1113B
:109E90002AC0809168078823B1F080916A018823E5
:109EA00059F081E090916807911180E024E045E14C
:109EB00056E0642D0E94A4CCCF5FC511E8CF84E0AA
:109EC000809366070BC080914F0710924F0788233D
:109ED00021F316DC809167078823F9F2CDB7DEB74E
:109EE000E0E10C9469F0C13059F5F8018591949145
:109EF000909376078093750780916807813081F091
:109F000080916A018823C1F21F929F928F926F9273
:109F100081E090916807913009F474C080E072C0CC
:109F200080914F0710924F07882351F380912807A3
:109F3000682F0E9421D280916707882309F3CECF32
:109F4000C23009F042C0F801859194919093760750
:109F500080937507809168078230D1F080916A0103
:109F6000882309F4A9CFDF92CF92BF92AF927F925C
:109F700081E090916807923009F080E08F930E9411
:109F8000F0220F900F900F900F900F900F9094CFA2
:109F900080914F0710924F07882301F30E941023EE
:109FA000809167078823D1F299CF80914F07109253
:109FB0004F078823C1F0609128078FEF0E9421D2BC
:109FC00080916707882379F089CFC33009F074CF77
:109FD000F80185919491909376078093750780910D
:109FE0006807833011F380916A01882309F464CFF4
:109FF0001F92FF92EF92DF9381E090916807933078
:10A0000009F08CCF8F930E94F0220F900F900F9049
:10A010000F900F9051CFB0E0A0E0E1E1F0E50C949B
:10A0200052F00E9458CDC091650785E0E82EEC0EF5
:10A0300095EDC92E95E0D92ED4E0DC1B13E01C1B56
:10A0400020EFA22E25E0B22E02E00C1B81E0F82EBC
:10A05000FC1A9C2E9194C1112AC080916807882314
:10A06000B1F080916A01882359F081E090916807EE
:10A07000911180E024E044EF55E0692D0E94A4CCCA
:10A08000CF5FEC12E8CF85E0809366070BC080912C
:10A090004F0710924F07882321F332DB8091670727
:10A0A0008823F9F2CDB7DEB7EBE00C946EF0C13047
:10A0B00011F580916807813079F080916A018823D9
:10A0C000F9F281E090916807913009F080E023E097
:10A0D00042E55DE26F2DD2CF80914F0710924F077E
:10A0E000882359F388EE90E50E94AECD80916707F2
:10A0F000882319F3D7CFC23009F053C09091680775
:10A10000923071F080916A01882309F4B9CF81E01F
:10A11000923009F080E020E246EE55E0602FAECFAD
:10A1200080914F0710924F07882361F3B092E506A4
:10A13000A092E40680916707882321F3B3CF809132
:10A140006807833081F080916A01882309F498CFF1
:10A1500081E090916807933009F080E023E049EDB9
:10A1600055E0612F8BCF80914F0710924F078823C6
:10A1700051F38BEE90E60E94AECD80916707882365
:10A1800011F390CF80914F0710924F07882391F0E1
:10A19000D092E506C092E40680916707882351F0CB
:10A1A00081CFC33061F2C43009F06ACF9091680763
:10A1B000943041F380916A01882309F461CF81E0F2
:10A1C000943009F080E020E244EC55E06D2F56CF4A
:10A1D000B0E0A0E0EEEEF0E50C9456F00E9458CD11
:10A1E000C091650785E0E82EEC0ED4E0DC1B13E09F
:10A1F0001C1B02E00C1B81E0F82EFC1ADC2ED19413
:10A20000C1112AC0809168078823B1F080916A014A
:10A21000882359F081E090916807911180E024E053
:10A220004DEB55E06D2D0E94A4CCCF5FEC12E8CF32
:10A2300085E0809366070BC080914F0710924F070F
:10A24000882321F35DDA809167078823F9F2CDB77F
:10A25000DEB7E7E00C9472F0C13011F58091680729
:10A26000813079F080916A018823F9F281E0909140
:10A270006807913009F080E023E048E75DE26F2D48
:10A28000D2CF80914F0710924F07882359F38FE167
:10A2900093E20E94AECD80916707882319F3D7CF50
:10A2A000C23009F055C080916807823081F08091FA
:10A2B0006A01882309F4B9CF81E090916807923050
:10A2C00009F080E023E041E75DE2602FACCF8091B0
:10A2D0004F0710924F07882351F38AE193E20E94BF
:10A2E000AECD80916707882311F3B1CF80916807C5
:10A2F000833081F080916A01882309F496CF81E050
:10A3000090916807933009F080E023E04AE65DE22F
:10A31000612F89CF80914F0710924F07882351F307
:10A3200085E193E20E94AECD80916707882311F307
:10A330008ECF80914F0710924F07882391F087E3CB
:10A3400097E40E94AECD80916707882351F07FCFBC
:10A35000C33061F2C43009F068CF8091680784305F
:10A3600041F380916A01882309F45FCF81E09091E5
:10A370006807943009F080E023E04CE55DE26D2F42
:10A3800052CFACE0B0E0E7ECF1E50C944CF09C87E8
:10A390008B87362E80914F0710924F07882339F014
:10A3A00010929A02ADD92C96E1E10C9468F060917C
:10A3B0006A0770916B0780916C0790916D0761152A
:10A3C00071058105910509F45CC0209112012223D9
:10A3D00009F4AEC0209113012111AAC021E0321668
:10A3E00009F484C0E2E03E1609F491C0C090140163
:10A3F000D0901501E0901601F090170140902001D7
:10A400005090210160902201709023010E946BE91D
:10A41000209108013091090140910A0150910B01EE
:10A420000E94CAE96F83788789879A87F4E03F9E04
:10A4300080011124C8018B589E4F9E838D83FC019F
:10A4400020813181428153816F81788589859A8508
:10A450000E9483F04B015C01A3019201C701B60188
:10A460000E9465E9811173C0F801EB58FE4F8082AC
:10A470009182A282B382832D0E94706E81E08093CC
:10A480006A0110926A0710926B0710926C07109283
:10A490006D0780916A01882309F485CF24E0329EFC
:10A4A000F0011124EB58FE4FC080D180E280F38090
:10A4B000C982DA82EB82FC822DEC3CEC4CEC5DE351
:10A4C000609108017091090180910A0190910B013E
:10A4D0000E94E6F187FD65C0CE0101960E94391BFE
:10A4E000BC018B859C850E944C755DCFC090180186
:10A4F000D0901901E0901A01F0901B0140902401C6
:10A500005090250160902601709027017FCFC09068
:10A510001C01D0901D01E0901E01F0901F014090A1
:10A5200028015090290160902A0170902B016ECF74
:10A53000412C20E5522E23EC622E27E4722EC12CF2
:10A5400030E5D32E33ECE32E37ECF32E5FCF20E053
:10A5500030E0A9016F81788589859A850E9465E937
:10A5600087FF0FC0A7019601C501B4010E9465E9EC
:10A5700087FF7ACFED81FE81C082D182E282F382B1
:10A580007ACFA3019201C501B4010E94E6F1181629
:10A590000CF06ACFED81FE8140825182628273822B
:10A5A0006ACF20E030E44CE156E4C701B6010E94D6
:10A5B000CAE94B015C0120E030E0A901C701B60106
:10A5C0000E9465E920E030E040EA50E487FF04C0E3
:10A5D00020E030E040EA50ECC501B4010E9483F075
:10A5E0002DEC3CEC4CEC5DE30E94CAE90E9462F168
:10A5F0006B017C01F7FC64C020EA36E841E050E0E2
:10A600000E94B5EFCA01B9012AE030E040E050E015
:10A610000E94B5EF605D60939B02C701B60120E127
:10A6200037E240E050E00E94B5EF8AE0882E912C9E
:10A63000A12CB12CCA01B901A50194010E94B5EF6A
:10A64000605D60939C02C701B60128EE33E040E0F4
:10A6500050E00E94B5EFCA01B901A50194010E9422
:10A66000B5EF605D60939D028EE280939E02C7010C
:10A67000B60124E630E040E050E00E94B5EFCA01A8
:10A68000B901A50194010E94B5EF605D60939F023E
:10A69000C701B601A50194010E94B5EF6B017C01D1
:10A6A000CA01B901A50194010E94B5EF605D6093F4
:10A6B000A00280E3C80EC092A1028BE992E010CF05
:10A6C000F094E094D094C094C11CD11CE11CF11C06
:10A6D0006DE2A1CF62E08AE69DE253CE61E081E7C0
:10A6E0009DE24FCE60E088E79DE24BCEA4E0B0E073
:10A6F000ECE7F3E50C945BF080914F0710924F0765
:10A70000882341F010929A020E94804B2496E2E046
:10A710000C9477F060916A0770916B0780916C07D9
:10A7200090916D07611571058105910561F10E9498
:10A730006BE9209108013091090140910A01509183
:10A740000B010E94CAE92091810130918201409160
:10A750008301509184010E9483F060938101709382
:10A760008201809383019093840183E00E94706E44
:10A7700081E080936A0110926A0710926B07109231
:10A780006C0710926D0780916A01882309F4BECF8F
:10A790002091500730915107409152075091530733
:10A7A0006091810170918201809183019091840177
:10A7B0000E9482F069837A838B839C83CE01019609
:10A7C0000E94391BBC018CE59DE20E944C759ECF16
:10A7D000B0E0A0E0EEEEF3E50C9456F00E943523D5
:10A7E000082F0E9458CDC0916507FC2E85E0E82E09
:10A7F000EC0E11E01C1BDC2ED194C11114C0809111
:10A8000068078823F9F080916A01882309F474C0ED
:10A8100081E090916807911180E024E04CE753E0DB
:10A820006D2D0E94A4CC01113AC0D2E0C130C1F517
:10A83000809168078130B9F080916A01811122C04E
:10A84000D2E044C080914F0710924F078823D9F27D
:10A850000E94804B809167078823A9F2CDB7DEB7AD
:10A86000E7E00C9472F080914F0710924F07882315
:10A8700019F387EC95E50E94AECD80916707882398
:10A88000D9F2ECCF81E090916807913009F080E037
:10A8900023E043E753E0612F0E94A4CCD1CFD1E065
:10A8A000DC1314C0809168078D17B9F080916A019C
:10A8B000882361F06C2F6F1981E0909168079C13D9
:10A8C00080E023E047E653E00E94A4CCCF5FCE11A6
:10A8D00094CFDF5FD0936607C1CF80914F0710926E
:10A8E0004F07882319F38AEE9AE50E94AECD809136
:10A8F00067078823D9F2B2CFD1E0002309F4A0CFB3
:10A90000E5CFB0E0A0E0E7E8F4E50C944FF00E945A
:10A9100058CDC09165076C2E85E0782E7C0E05E839
:10A9200013E89AE2A92E94E0B92ED5E0DC1B27E5C6
:10A93000E22E23E8F22E84E0D82EDC1A83E0C82E23
:10A94000CC1A82E0982E9C1A81E0882E8C1AC111B4
:10A950002CC0809168078823B9F080916A01882310
:10A9600061F0662D619581E090916807911180E01A
:10A9700024E04EE454E00E94A4CCCF5FC711E7CF9F
:10A9800086E0809366070CC080914F0710924F07B6
:10A99000882319F30E94804B809167078823E9F28E
:10A9A000CDB7DEB7EEE00C946BF0C13049F5809185
:10A9B00068078130A1F080916A018823F1F28CE967
:10A9C00093E89F938F9388E494E09F938F938F9263
:10A9D00081E090916807913069F180E02BC080910F
:10A9E0004F0710924F07882331F38CE993E8892BA6
:10A9F00011F00E949C83809167078823E1F2D0CFF9
:10AA0000C23009F08FC0809168078230E9F08091F0
:10AA10006A01882309F4B1CF88ED92E29F938F9366
:10AA20008EE394E09F938F939F9281E090916807CB
:10AA3000923099F68F930E94F0220F900F900F9012
:10AA40000F900F900F9099CF80914F0710924F0762
:10AA50008823E9F20E94D822809167078823B9F2FF
:10AA60009FCF809168078330A9F080916A01882385
:10AA700009F483CF8EE693E89F938F9387E394E066
:10AA80009F938F93CF9281E090916807933009F064
:10AA9000A4CFD0CF80914F0710924F07882329F37E
:10AAA0008EE693E8892B11F00E946E8380916707F0
:10AAB0008823D9F275CF80916807843099F080910E
:10AAC0006A01882309F459CFFF92EF9282E394E060
:10AAD0009F938F93DF9281E090916807943009F003
:10AAE0007CCFA8CF80914F0710924F07882339F36E
:10AAF000E114F10411F00E945783809167078823C5
:10AB0000F1F24ECF80914F0710924F078823B1F09A
:10AB10000115110511F00E94858380916707882334
:10AB200069F03ECFC33009F49CCFC43021F2C53068
:10AB300009F023CF80916807853021F380916A0165
:10AB4000882309F41ACF1F930F93BF92AF92DF931C
:10AB500081E090916807953009F03FCF6BCF80E09E
:10AB600090E0A0E8B0E480937D0190937E01A093F3
:10AB70007F01B09380018AE192E00E945E22809181
:10AB8000EB030E940A7A10929A020C94804BB0E078
:10AB9000A0E0EDECF5E50C9454F00E9458CDC09186
:10ABA000650785E0C82ECC0ED4E0DC1B13E01C1B2F
:10ABB00082E0F82EFC1A81E0E82EEC1ABC2EB1944B
:10ABC000C1112BC0809168078823B1F080916A0180
:10ABD000882359F081E090916807911180E024E08A
:10ABE00045E553E06B2D0E94A4CCCF5FCC12E8CF9B
:10ABF00085E0809366070CC080914F0710924F0745
:10AC0000882321F30E94804B809167078823F1F20B
:10AC1000CDB7DEB7E9E00C9470F0C13089F58091D2
:10AC200068078130C1F080916A018823F1F2DD2448
:10AC3000D39480916807813009F0D12C8DE79DE095
:10AC40000E941F1E00E09C014AE453E06E2D8D2DF2
:10AC50000E94B375CACF80914F0710924F07882387
:10AC600011F30E944CCD4FE75DE26DE77DE08AE491
:10AC700093E00E94BDCD809167078823A1F2C8CFE1
:10AC8000C23009F073C0809168078230B1F08091C2
:10AC90006A01882309F4A9CFDD24D3948091680741
:10ACA000823009F0D12C81E89DE00E941F1E00E057
:10ACB0009C014FE353E06F2DCACF80914F07109254
:10ACC0004F07882321F30E944CCD4EE75DE261E8F7
:10ACD0007DE08FE393E00E94BDCD809167078823DC
:10ACE000B1F296CF809168078330B1F080916A010C
:10ACF000882309F47ACFDD24D394809168078330C8
:10AD000009F0D12C85E89DE00E941F1E00E09C0107
:10AD100044E353E0612F9BCF80914F0710924F0780
:10AD2000882321F30E944CCD4DE75DE265E87DE08C
:10AD300084E393E00E94BDCD809167078823B1F240
:10AD400067CF80914F0710924F078823C9F00E9468
:10AD50004CCD4CE75DE269E87DE089E293E00E943A
:10AD6000BDCD80916707882359F052CFC33009F4D5
:10AD7000B9CFC43009F039CF80916807843009F326
:10AD800080916A01882309F430CFDD24D394809127
:10AD90006807843009F0D12C89E89DE00E941F1ECD
:10ADA00000E09C0149E253E06D2F51CFA3E0B0E0F9
:10ADB000ECEDF6E50C944BF04C013B015A01190106
:10ADC000280181E080939A0240916A0750916B07B5
:10ADD00060916C0770916D07411551056105710512
:10ADE00071F0141615060CF080E08093E9031092C0
:10ADF0006A0710926B0710926C0710926D07109102
:10AE0000E90380914F078B8310924F07811105C092
:10AE100080916A01882309F46FC0C2010E94186FF3
:10AE2000082F80E0C114D10419F0C6010E94186FE8
:10AE30001A821982E114F104B1F4402F50E0282F56
:10AE400030E0CA01820F931F46976CF485E190E0D1
:10AE5000841B950B821B930B97FD01969595879507
:10AE60008A8381E0898301E028E139E6A201BE01FD
:10AE70006F5F7F4FCE0102960E947070E114F10463
:10AE800091F08A81882321F01A8289818F5F8983DA
:10AE900000E02BE139E6A701BE016F5F7F4FCE01D5
:10AEA00002960E947070C114D10459F000E028E1AC
:10AEB00039E6A601BE016F5F7F4FCE0102960E9468
:10AEC000707041E04127B30181E00E945BD4C4016E
:10AED0000E94186F412FB40194E1981B892F0E94A2
:10AEE0005BD4EB81EE2341F0111101C05101A1149B
:10AEF000B10431F0F50109952396E2E10C9467F075
:10AF00000E94804BF9CFCF92DF92EF92FF920F9386
:10AF10001F938EE9C82E85E0D82EF12CE12C00EA93
:10AF200015E030E020E040E357E460EB75E085EBAE
:10AF300095E03CDF1F910F91FF90EF90DF90CF9055
:10AF40000895B0E0A0E0E7EAF7E50C9453F0ADB661
:10AF5000BEB6809123106AE777E0882311F063E2A0
:10AF600070E1FB0101900020E9F7CF01861B970BF0
:10AF700001962DB73EB7281B390B0FB6F8943EBF8C
:10AF80000FBE2DBF8DB79EB701967C0180E2EDB755
:10AF9000FEB78183C70101960E94A7F28AE5C82EF9
:10AFA00085E0D82E0CE515E030E020E04AEF57E4CC
:10AFB00068E675E08FE695E0F9DE0FB6F894BEBE60
:10AFC0000FBEADBEEAE00C946FF0CF92DF92EF922D
:10AFD000FF920F931F9388EBC82E84E0D82EF12C9C
:10AFE000E12C0BE215E030E020E04BED55E66AEB9A
:10AFF00074E08FEB94E0DADE1F910F91FF90EF90F9
:10B00000DF90CF900895CF92DF92EF92FF920F934F
:10B010001F938AE8C82E83E0D82EF12CE12C0CE88F
:10B0200013E02FEA35E546E652E268E973E08DE980
:10B0300093E0BCDE1F910F91FF90EF90DF90CF90D7
:10B040000895B0E0A0E0E7E2F8E50C9453F0ADB667
:10B05000BEB683E392E00E94186F90E001962DB790
:10B060003EB7281B390B0FB6F8943EBF0FBE2DBF5D
:10B070008DB79EB701967C0163E372E00E94ADE854
:10B080008091280700E012E0813031F00BEE11E0F2
:10B09000823011F003E112E084E2C82E82E0D82E63
:10B0A0002EEE37E44DE553E666E272E08DE292E083
:10B0B0007DDE0FB6F894BEBE0FBEADBEEAE00C94C6
:10B0C0006FF08F929F92AF92BF92CF92DF92EF92EA
:10B0D000FF920F9380914F0710924F07882371F0D2
:10B0E00010929A020E94804B0F91FF90EF90DF9098
:10B0F000CF90BF90AF909F908F90089581E0809304
:10B100009A0280916A0790916B07A0916C07B091A9
:10B110006D070097A105B10509F44AC05C01AA0CAE
:10B12000BB1CAA0CBB1C10926A0710926B071092F2
:10B130006C0710926D07B5010B2C000C880B990B56
:10B140000E946BE92091B0073091B1074091B2079E
:10B150005091B3070E94CAE92091561330915713BA
:10B1600040915813509159130E9483F06B017C0158
:10B1700020E030E040EA51EC0E94E6F187FD18C083
:10B1800020E030E040EA51E4C701B6010E9465E9E1
:10B19000181674F0C5010E94D2C8C0925613D092FE
:10B1A0005713E0925813F092591382E080936A018A
:10B1B00080916A01882309F497CFC0905613D090EC
:10B1C0005713E0905813F090591320E030E44CE10D
:10B1D00056E4C701B6010E94CAE94B015C0120E0B8
:10B1E00030E0A901C701B6010E9465E920E030E026
:10B1F00040EA50E487FF04C020E030E040EA50EC31
:10B20000C501B4010E9483F02DEC3CEC4CEC5DE3F5
:10B210000E94CAE90E9462F16B017C018BE2F7FE99
:10B2200009C0F094E094D094C094C11CD11CE11CDE
:10B23000F11C8DE280939B02C701B60120E137E249
:10B2400040E050E00E94B5EF6AE0862E912CA12CE0
:10B25000B12CCA01B901A50194010E94B5EF605D4E
:10B2600060939C02C701B60128EE33E040E050E055
:10B270000E94B5EFCA01B901A50194010E94B5EF82
:10B28000605D60939D028EE280939E02C701B601CD
:10B2900024E630E040E050E00E94B5EFCA01B90179
:10B2A000A50194010E94B5EF605D60939F02C70104
:10B2B000B601A50194010E94B5EF6B01CA01B90165
:10B2C000A50194010E94B5EF605D6093A00260E368
:10B2D0006C0D6093A1026BE972E084EF92E00E9432
:10B2E0004C75C0905613D0905713E0905813F090BF
:10B2F00059138090E5039090E603A090E703B09087
:10B30000E803A5019401C701B6010E9465E98823FD
:10B31000E9F020E030E0A901C701B6010E9465E92B
:10B32000882309F479C0A5019401C701B6010E94E0
:10B3300065E987FD73C081E08093E403C092E50373
:10B34000D092E603E092E703F092E803D090E403A2
:10B350008091AB13813188F48091AD13833068F014
:10B3600044E04D195CEDE52E52E0F52E0CE022E0B4
:10B3700062E487E793E10E9497D58091AB13853112
:10B3800080F48091AD13843160F049EDE42E42E009
:10B39000F42E01E023E044E16CE387E793E10E94AF
:10B3A00097D58091AB138F3308F09ECE8091AD136B
:10B3B0008F3208F499CE40E34D198FEBE82E82E0EE
:10B3C000F82E0DE022E06AE587E793E10E9497D529
:10B3D00041E34D1995EAE92E92E0F92E22E065E06D
:10B3E00087E793E10E9497D525E7E22E22E0F22E2F
:10B3F00000E123E04FE262E187E793E10E9497D505
:10B4000035E4E32E32E0F32E23E04FE267E687E7F0
:10B4100093E10E9497D568CE80E08ECF8FEF8CCFDE
:10B420000F931F93CF93DF93FC01EB0180916A0789
:10B4300090916B07A0916C07B0916D07B7FF08C0A2
:10B4400010926A0710926B0710926C0710926D07AA
:10B450008091590790915A07A0915B07B0915C07C2
:10B4600040916A0750916B0760916C0770916D076E
:10B4700084179507A607B70744F480936A0790934B
:10B480006B07A0936C07B0936D0780916A018823C6
:10B49000E1F060916A0770916B0780916C07909161
:10B4A0006D0700915D0710915E0720915F07309155
:10B4B0006007600F711F821F931F0995BC01809167
:10B4C0006307909164070E944C7580914F0781112A
:10B4D00008C0809156078823A9F180916A018823CA
:10B4E00089F180916107909162070097B1F04091D6
:10B4F0006A0750916B0760916C0770916D0700911E
:10B500005D0710915E0720915F0730916007400F43
:10B51000511F621F731FFE010995E0915707F091BB
:10B520005807309741F080915607811103C08091F0
:10B530004F078111099580914F0710924F07811194
:10B540000E94804BDF91CF911F910F91089565E28A
:10B550007DE18EE39DE164CF62EA7DE183E896E4DC
:10B560005FCF60EB7DE183ED9EE15ACF64EC7DE13E
:10B5700088ED9DE155CF61E17EE18FE996E450CF02
:10B58000E091DD03E63028F581E08E0F8093DD0346
:10B5900040916A0750916B0760916C0770916D073D
:10B5A000209165079091660780919A0239E0E39FA8
:10B5B000F0011124E955FC4FA0917113B091721361
:10B5C000B183A083428353836483758326839783E7
:10B5D00080870895A7E0B0E0E0EFFAE50C944BF027
:10B5E0000E9458CDF09065072F2C85E08F0D8D833C
:10B5F0003324339483E0E82E98EE892E93E0992E3D
:10B60000A12CB12C84E08F198E839E2D9F199F83CE
:10B6100082E0D82EDF18C32CCF18F1102CC08091F7
:10B6200068078823C1F080916A01882361F0622D48
:10B63000619581E090916807911180E024E045E5F3
:10B6400053E00E94A4CCF3949D81F912E6CF85E0EB
:10B65000809366070CC080914F0710924F07882394
:10B6600011F30E94804B809167078823E1F22796AF
:10B67000E2E10C9467F081E0F8122DC09091680728
:10B680009130B9F080916A018823E9F281E091302C
:10B6900009F080E090919C032DE133E0911102C00C
:10B6A00029E133E001E040E253E06C2D0E94B375E4
:10B6B000CACF80914F0710924F07882319F38091CA
:10B6C0009C038F2580939C03E0926A018091670719
:10B6D0008823C1F2CCCF92E0F912D1C080916807E3
:10B6E000823021F180916A01882309F4ACCF11E006
:10B6F00080916807823009F010E060910601709136
:10B700000701072E000C880B990B0E946BE96983D7
:10B710007A838B839C83CE0101960E94964600E03B
:10B720009C0142E153E06D2D812FC0CF80914F07E6
:10B7300010924F078823B1F210E000E025EF30E0CF
:10B7400050E040E066E071E082E193E00E941DCEAF
:10B7500080916707882331F28ACF80916807833010
:10B7600019F180916A01882309F46DCF11E080916D
:10B770006807833009F010E06091040170910501C1
:10B78000072E000C880B990B0E946BE969837A8362
:10B790008B839C83CE0101960E94964600E09C011B
:10B7A0004BE053E06F81C0CF80914F0710924F075D
:10B7B0008823B9F210E000E025EF30E050E040E0EF
:10B7C00064E071E08BE093E00E941DCE80916707FA
:10B7D000882339F24CCF80914F0710924F0788236E
:10B7E00009F459C020E030E048EC52E460910001D7
:10B7F0007091010180910201909103010E94CAE9B8
:10B800000E9467F12B0130926707BADEE0926A016D
:10B8100083E093E0909364078093630780E091E076
:10B82000909362078093610710925D0710925E0704
:10B8300010925F07109260078092590790925A0702
:10B84000A0925B07B0925C07712C612C40926A0752
:10B8500050926B0760926C0770926D0786EB9AE5C9
:10B860009093721380937113109258071092570798
:10B870001092560780916707882369F0F8CE83E01D
:10B88000F81609F46ACF94E0F912DDCE80916807CA
:10B89000843009F4A0CF80916A01882309F4D3CEC3
:10B8A00011E080916807843009F010E040900001B9
:10B8B00050900101609002017090030120E030E09F
:10B8C000A901C301B2010E9465E92DEB37E346E00F
:10B8D00055EB87FD04C02DEB37E346E055E3C3018C
:10B8E000B2010E9483F069837A838B839C83CE01AB
:10B8F00001960E94AF1B00E09C0143E053E06E8183
:10B9000013CFB0E0A0E0E7E8FCE50C945BF08D819C
:10B9100090919410891778F0809394109E01285F7D
:10B920003F4F4E815F8164E570E08FE390E10E94BC
:10B930002DE910923E10E2E00C9477F00F931F93E4
:10B94000CF93DF936F3F11F41092941020919410D5
:10B9500021111EC08C010E94B4E8800F911FEC01E0
:10B96000C01BD10BC535D1053CF00197FC012491DA
:10B97000207C2038D1F3F3CFDD27AE01B8018FE36F
:10B9800090E10E94D5E8C15CDF4E188210923E1013
:10B99000DF91CF911F910F910895A6E8B0E0E3EDFC
:10B9A000FCE50C9456F0C358DF4F188219821A82B6
:10B9B0001B82CD57D04080918E0290918F02A09132
:10B9C0009002B0919102CF57DF4F88839983AA8369
:10B9D000BB83C158D04084E690E090939E12809340
:10B9E0009D121092C2121092C11210921A0464E0B9
:10B9F00070E0CE018F579F4F0E9480D180919D12A1
:10BA000090919E12029690939E1280939D12109296
:10BA1000C2121092C11281E0CA57DF4F8883C65804
:10BA2000D040CE018A579F4F0E94472268E470E0C1
:10BA300089E69DE00E9480D180E1E1E9F1E08E019C
:10BA40000F5F1F4FD80101900D928A95E1F760E1D9
:10BA500070E0C8010E9480D18BE897E00E944F22DD
:10BA60008CE0F80111928A95E9F7C8010E944B22F7
:10BA70007E01FDE6EF0EF11C8FEFF7018083C70119
:10BA80000E94472219821A821B821C82C8010E94CE
:10BA90004F228091B4029091B502A091B602B0916C
:10BAA000B70289839A83AB83BC83C8010E944F226B
:10BAB000C358DF4F188219821A821B82CD57D0409B
:10BAC00083E0F70180838983CE0183589F4F0E94D2
:10BAD0004F22C7010E944722C8010E9447222AE044
:10BAE000D22EDA94DD2031F0CE0183589F4F0E9490
:10BAF0004F22F7CF8EE493E10E944B22C358DF4FD1
:10BB0000188219821A821B82CD57D0409AE0D92E12
:10BB1000DA94DD2031F0CE0183589F4F0E944F22EE
:10BB2000F7CF87E08983F7018083C8010E9447220D
:10BB3000C7010E94472268E070E084E893E00E9419
:10BB400080D168E070E08CE793E00E9480D164ECE3
:10BB500070E088EB92E00E9480D11982DD24DA94B3
:10BB6000F701D082C8010E944322C7010E944722E8
:10BB700064E070E082E292E00E9480D18091E3066E
:10BB80008983C8010E9443226CE070E083E497E05F
:10BB90000E9480D1198A1A8A1B8A1C8A80E090E050
:10BBA000A0E8BFE38D879E87AF87B88B8091B512E1
:10BBB0009091B612A091B712B091B81289839A836E
:10BBC000AB83BC8320E030E543EC50E46091B912D4
:10BBD0007091BA128091BB129091BC120E94CAE976
:10BBE0006D837E838F8398872CEA35EC47E25EE392
:10BBF0006091BD127091BE128091BF129091C012DF
:10BC00000E94CAE969877A878B879C8764E170E024
:10BC1000C8010E9480D184E190E09A83898362E028
:10BC200070E0C8010E9480D1809137079091380759
:10BC3000A0913907B0913A0789839A83AB83BC837B
:10BC400020E030E543EC50E460913B0770913C0705
:10BC500080913D0790913E070E94CAE96D837E83E3
:10BC60008F8398872CEA35EC47E25EE360913F07CB
:10BC70007091400780914107909142070E94CAE964
:10BC800069877A878B879C87C8010E943F228CE056
:10BC9000E1EAF1E0D80101900D928A95E1F7C8013F
:10BCA0000E943F221982C8010E9447228FE78983A0
:10BCB000C8010E944722D982C8010E94472285E01C
:10BCC000EDEAF1E0D80101900D928A95E1F765E087
:10BCD00070E0C8010E9480D11982C8010E944322ED
:10BCE00080E2E2EBF1E0D80101900D928A95E1F754
:10BCF00060E270E0C8010E9480D1F7011082C701A4
:10BD00000E9443221982C8010E94432280E090E0F1
:10BD1000A0EEBFE3C358DF4F88839983AA83BB8318
:10BD2000CD57D040CE0183589F4F0E944F22C35819
:10BD3000DF4F188219821A821B82CD57D040CE0164
:10BD400083589F4F0E944F2282E1F80111928A95F9
:10BD5000E9F762E170E0C8010E9480D184E2E2ED7F
:10BD6000F1E0D80101900D928A95E1F764E270E06C
:10BD7000C8010E9480D180E1F80111928A95E9F70B
:10BD800060E170E0C8010E9480D189E0F801119261
:10BD90008A95E9F769E070E0C8010E9480D1C35834
:10BDA000DF4F188219821A821B82CD57D040CE01F4
:10BDB00083589F4F0E944F228CE0D82EF8018D2D82
:10BDC00011928A95E9F76CE070E0C8010E9480D179
:10BDD0008CE6F80111928A95E9F76CE670E0C801EB
:10BDE0000E9480D18EE094E00E943F22F7011082F1
:10BDF000118212821382148215821682178268E0E1
:10BE000070E0C7010E9480D1F7011192DA94E9F73E
:10BE1000CB57DF4F1882C558D04080E090E0A0E4B7
:10BE2000B0E4ED968CAF9DAFAEAFBFAFED97C7015D
:10BE30000E944B22CE018B579F4F0E944722CE017A
:10BE400087589F4F0E944F2280911A04811127C06A
:10BE500000919D1210919E128091C1129091C21278
:10BE6000F7019183808384E690E090939E12809303
:10BE70009D1264E070E086E292E00E9480D162E070
:10BE800070E0C7010E9480D191E00037F3E01F0706
:10BE900009F490E080911A04892B80931A04809110
:10BEA0001A04811104C060E083E49AE047DD9091B8
:10BEB0001A0481E08927CA57DF4FE7E00C9472F03B
:10BEC0006CCDA3E0B0E0E7E6FFE50C944BF00E94F8
:10BED0003523582E0E9458CD209165072A83422E83
:10BEE0002B5F2B8383E0782E74180CE514E02FE78A
:10BEF000E22E2BE4F22E3DE6C32E34E0D32E40E6B4
:10BF0000A42E4FE5B42E5BE7852E54E0952E82E0FB
:10BF10008419898381E0382E3418242C21948A8155
:10BF200081118EC080916807882309F477C08091C1
:10BF30006A01882359F081E090916807911180E0AF
:10BF400024E043EB54E0622D0E94A4CC51103DC18B
:10BF50008A81833009F029C180916807833009F410
:10BF6000C3C080916A018111D0C084E0682E81E055
:10BF7000860D51104AC09A8189131FC080916807AD
:10BF8000891709F4F4C080916A018823B1F0FF9207
:10BF9000EF92DF92CF928A8184198F9381E0909102
:10BFA00068072A81921380E08F930E94F0220F90FD
:10BFB0000F900F900F900F900F9082E0860D9A8156
:10BFC000891321C080916807891709F4DFC0809127
:10BFD0006A018823C1F080E093E49F938F931F93BD
:10BFE0000F938A8184198F9381E0909168072A8149
:10BFF000921380E08F930E94F0220F900F900F9089
:10C000000F900F900F9083E0860D9A819F5F9A8327
:10C010002B81291384CF809366070EC080914F0730
:10C0200010924F07882309F482CF0E94804B8091A1
:10C030006707882309F47BCF2396E2E10C9467F02D
:10C040009A81913051F5809168078130B9F08091E3
:10C050006A01882309F47ACF81E0909168079130D2
:10C0600009F080E023E041EA54E0632D0E94A4CC73
:10C070005110ABC085E094E0692E7DCF80914F07D1
:10C0800010924F07882319F388EE93E50E94AECDF6
:10C09000809167078823D9F2CFCF2A81223009F017
:10C0A00055CF80916807823081F080916A018823A2
:10C0B00009F44CCF81E090916807923009F080E05C
:10C0C00023E042E954E06981D1CF80914F0710927B
:10C0D0004F07882351F381E698E50E94AECD809109
:10C0E0006707882311F3A8CF80914F0710924F075D
:10C0F000882309F436CF81E894E50E94AECD809183
:10C100006707882309F42DCF97CF81E090916807C6
:10C11000933009F080E023E04AE854E0672D0E9464
:10C12000A4CC23CF80914F0710924F07882309F4A6
:10C1300046C033DC80916707882309F440C07CCF78
:10C14000BF92AF929F928F928A8184198F9381E0E0
:10C15000909168072A81921380E08F930E94F022C9
:10C160000F900F900F900F900F900F902CC0809118
:10C170004F0710924F07882309F405CF0E94724B96
:10C1800080916707882309F4FECE56CF80914F0730
:10C1900010924F07882309F41ACF0E94DC41809146
:10C1A0006707882309F413CF47CF8A81843009F0C9
:10C1B00061CF809168079A81891709F4B3CF809184
:10C1C0006A018111BDCF8A81D1CE9A8184E09330FA
:10C1D00009F01BCFEECFA7E0B0E0E1EFF0E60C9462
:10C1E0004BF08091770787708983809084039090CB
:10C1F0008503A0908603B09087030E9458CD2091BC
:10C2000065072E833981373009F075C085E194E0E8
:10C210009B838A831E81312F3B5F3C83332433947D
:10C22000812F81958D83232C211A84E6482E512C51
:10C23000612C712C2E81222309F462C039813730A0
:10C2400009F434C22E81213009F029C29091680787
:10C25000913009F445C180916A01811154C182E095
:10C26000F82E81E08F0D8F839981973009F063C09C
:10C2700020E030E0A901C501B4010E9465E98823EE
:10C2800009F459C03F818E81381331C09091B302B7
:10C290009F83809168072E81821311C080914F0780
:10C2A00010924F07882359F093259F8383E0809352
:10C2B0006A010E9453228091670781110DC180910C
:10C2C0006A018823A1F06E81611B81E0909168076B
:10C2D0003E81931380E09F8126EF33E0911102C0ED
:10C2E00022EF33E001E049EF53E00E94B375F3948D
:10C2F000F394FF8220C020E134E03B832A838ACF7D
:10C3000080916807882309F4D9C080916A01882345
:10C3100009F494CF81E090916807911180E024E0C6
:10C3200043E254E06D810E94A4CC8981873009F4F6
:10C330001DC193E09F838091B4029091B502A091BA
:10C34000B602B091B7028093280790932907A09373
:10C350002A07B0932B072F813E8123131EC08091A3
:10C360006807821709F407C180916A018823A9F040
:10C37000EE80E11AFF24F394809168073E818313D5
:10C38000F12C88E297E00E94464600E09C0146EED0
:10C3900053E06E2D8F2D0E94B3758F818F5F9E812C
:10C3A000891316C080916807891709F439C18091F3
:10C3B0006A01882369F06E81611B81E090916807B2
:10C3C0002E81921380E023E047ED53E00E94A4CC3D
:10C3D0008F818E5F3E81831316C08091680783171B
:10C3E00009F42FC180916A01882369F06E81611B75
:10C3F00081E0909168072E81921380E023E04AEC5F
:10C4000053E00E94A4CC8F818D5F3E81831323C0B3
:10C4100080916807831709F425C180916A018823F8
:10C42000D1F08FE79BE49F938F938CEB93E09F93E6
:10C430008F938E81811B8F9381E0909168073E815D
:10C44000931380E08F930E94F0220F900F900F9033
:10C450000F900F900F908F818C5F9E81891323C066
:10C4600080916807891709F40CC180916A018823BB
:10C47000D1F080E69FE59F938F938DEA93E09F93A1
:10C480008F938E81811B8F9381E0909168072E811D
:10C49000921380E08F930E94F0220F900F900F90E4
:10C4A0000F900F900F903E813F5F3E838C818313EE
:10C4B000C1CE9F819B5F909366070EC080914F070E
:10C4C00010924F07882309F420CF0E94804B80915F
:10C4D0006707882309F419CF2796E2E10C9467F0E7
:10C4E00080914F0710924F07882309F4B4CE20EFB4
:10C4F00035E03093E5062093E406809167078823B2
:10C5000009F4A9CEE9CF81E0913009F080E020E282
:10C5100049E154E0622D0E94A4CCA1CE909168071D
:10C520003E81931731F080916A01811113C08E8191
:10C5300097CE80914F0710924F078823A1F32A814D
:10C540003B813093E5062093E406809167078823BA
:10C5500051F3C2CF6E81611B81E03E81931380E075
:10C5600020E246E054E00E94A4CCE1CF22E02F83F9
:10C57000FF24F3947DCE80914F0710924F078823BC
:10C5800009F4F2CE0E944CCD6091280770912907E2
:10C5900080912A0790912B070E9467F16B013092DE
:10C5A00067070E94C05A83E080936A0186EE93E099
:10C5B000909364078093630728E237E03093620723
:10C5C0002093610710925D0710925E0710925F073B
:10C5D000109260074092590750925A0760925B0789
:10C5E00070925C07F12CE12CC0926A07D0926B0725
:10C5F000E0926C07F0926D078CEA9AE590937213C3
:10C600008093711329E532E230935807209357073E
:10C610001092560780916707882309F4A5CE5CCF56
:10C6200080914F0710924F07882309F4C0CE81E60E
:10C6300098E50E94AECD80916707882309F4B7CEB4
:10C640004BCF80914F0710924F07882309F4CACE31
:10C6500080EB97E40E94AECD80916707882309F4B0
:10C66000C1CE3ACF80914F0710924F07882309F42B
:10C67000D4CE0E94724B80916707882309F4CDCEF7
:10C680002BCF80914F0710924F07882309F4EDCEEE
:10C6900084D980916707882309F4E7CE1DCF2E81C6
:10C6A000223009F43BCF33E03F8345CE8E81813089
:10C6B00009F434CF92E09F835BCF0E94DC416DD9B7
:10C6C0000C94EE47CF9380919F03811109C08CEDAC
:10C6D00091E09093E3038093E20381E080939F03D2
:10C6E0000E94C05A20E040E070E060E080E493E205
:10C6F0000E94B246C1E0C0939A020E94802D0E941F
:10C70000804BC0939A0260E086EC9DE217D988EDD9
:10C7100091E09093E5068093E406CF910895A6E01A
:10C72000B0E0E5E9F3E60C944BF00E94EA7B382E8A
:10C730008091C91484FB662460F8412C84FF03C0F7
:10C740000E94FD7B482E0E9458CD209165072D83C5
:10C75000522E2B5F298380E009E115E091E0792ECC
:10C760007518952D91959A8392E6E92E93E6F92E08
:10C7700026E3C22E25E0D22E92E095199B8393E00A
:10C7800095199C8335ED832E34E0932E4AEEA42E2A
:10C7900044E0B42E9D812981921709F409C299239E
:10C7A00049F131106AC00E944082882309F47AC19D
:10C7B0009D81913009F444C122E02E832D818E8128
:10C7C00028135FC180916807281709F46EC1809112
:10C7D0006A01882309F455C16D81651981E0909142
:10C7E00068072D81921380E023E042E155E00E942A
:10C7F000A4CC47C180916807882379F180916A01B0
:10C80000882379F281E090916807911180E024E01B
:10C8100042E455E06A810E94A4CC332021F224E056
:10C820002E839D812E8192134AC0809168079817AC
:10C8300009F44CC180916A01882309F440C06D81DC
:10C84000651981E0909168072D81921380E023E0C3
:10C8500046E055E00E94A4CC32C080914F07109270
:10C860004F07882359F20E94804B809167078823E5
:10C8700029F22696E2E10C9467F08D81813009F46B
:10C880007FC0823009F4A6C09D81933041F680912B
:10C890006807833009F4C3C080916A01882309F4D2
:10C8A000BECF81E090916807933009F080E023E0EB
:10C8B00046E255E06C810E94A4CC84E08E838E8198
:10C8C0008F5F9D81981316C080916807981709F4AF
:10C8D0000EC180916A01882369F06D81651981E03C
:10C8E000909168072D81921380E023E048EF54E097
:10C8F0000E94A4CC8E818E5F662009F430C1411065
:10C900003BC09D8198131BC020906807921509F4C5
:10C91000FFC080916A01882391F01F92BF92AF926D
:10C920008D8185198F9381E02D81221180E08F9375
:10C930000E94F0220F900F900F900F900F908E8119
:10C940008D5F9D81981316C080916807981709F430
:10C95000F5C080916A01882369F06D81651981E0D5
:10C96000909168072D81921380E023E049ED54E017
:10C970000E94A4CC8E818C5F9D819F5F9D830ACF96
:10C98000809168078130D1F080916A01882309F491
:10C9900046CFFF92EF92DF92CF927F9281E090910B
:10C9A0006807913009F080E08F930E94F0220F9089
:10C9B0000F900F900F900F900F9031CF80914F07F5
:10C9C00010924F07882301F37DDE8091670788234B
:10C9D000D9F24FCF80916807823091F080916A013F
:10C9E000882309F41CCF81E090916807923009F008
:10C9F00080E023E04BE255E06B810E94A4CC0FCF96
:10CA000080914F0710924F07882341F385EE97E5F9
:10CA10000E94AECD80916707882301F32ACF8091D1
:10CA20004F0710924F07882309F436CF8EE99BE415
:10CA30000E94AECD80916707882309F42DCF19CFCE
:10CA400080916807813009F180916A01882309F497
:10CA5000B3CE80E495E49F938F931F930F937F92BF
:10CA600081E090916807913009F080E08F930E94F7
:10CA7000F0220F900F900F900F900F900F9082E088
:10CA80008E838E818F5F8E83CCCE80914F071092E4
:10CA90004F078823C9F20E94404580916707882389
:10CAA00099F2E7CE91E09E8389CE80914F07109254
:10CAB0004F07882309F48BCE8BE090E50E94AECD22
:10CAC00080916707882309F482CED3CE80914F07E7
:10CAD00010924F07882309F4ADCE87E69DE40E94AB
:10CAE000AECD80916707882309F4A4CEC2CE809191
:10CAF0004F0710924F07882309F4EBCE81E69FE59C
:10CB00000E94AECD80916707882309F4E2CEB1CEB2
:10CB100080914F0710924F07882309F4FACE4FE314
:10CB200050E064EC74E086EE96E00E94BCF28091E6
:10CB30006707882309F4EDCE8D811ECF80914F07C2
:10CB400010924F07882309F404CF89E497E60E94E6
:10CB5000AECD80916707882309F4FBCEEDCF9D8190
:10CB6000981314C0909168072D81291791F0809136
:10CB70006A01882359F06D81651981E02D8129139F
:10CB800080E020E248EC54E00E94A4CC8E818D5FCE
:10CB9000F3CE80914F0710924F07882341F3909274
:10CBA000E5068092E40680916707882301F3C4CFED
:10CBB000809366075ECE10929802109269010E94DF
:10CBC000FD7B9091C91480FB97F99093C91460E0A4
:10CBD0008AEC91E00E949E5C0C94EE470F931F93A9
:10CBE0000E94D6D100919402109195022091960254
:10CBF00030919702601B710B820B930B97FD0CC059
:10CC000089B183FB882780F991E089274A9B82605C
:10CC1000309B846080939302809193028170909105
:10CC2000930291FD826090919E03981749F08130A4
:10CC300009F148F0823079F0833091F080939E03BF
:10CC40001F910F910895913079F09230B9F790913A
:10CC5000920291500CC0992339F09330C1F3EECF7A
:10CC60009130A9F3923051F7909192029F5F909387
:10CC70009202E4CF992359F3933001F7F5CF1F9334
:10CC8000CF93DF93809135018F3708F475C08F57AC
:10CC90009091B41290939E04992309F46BC05D9A0D
:10CCA0009091360790939D04992309F46FC05C9A84
:10CCB0008F5F8093350180919C0491E08927809358
:10CCC0009C0481118BDF8091340191E0980F8530B5
:10CCD0000CF090E0823009F4A8C00CF059C0882311
:10CCE00009F46EC0813009F495C090933401C0916D
:10CCF0007807D0917907209709F42DC0F89413B1E3
:10CD0000147082E00E94FF2C00C000C01C161D069B
:10CD10000CF0B9C02A9A00C000C02B9A00C00000D5
:10CD200082E090E00197F0F72B9800C000C011233B
:10CD300009F4ABC02A9A00C000C0789480917807AB
:10CD4000909179071C161D060CF0A1C001979093D5
:10CD50007907809378078091B10D9091B20D00977B
:10CD600029F001979093B20D8093B10DDF91CF918F
:10CD70001F9108955D9894CF90919E04891708F0B3
:10CD80005D9890919D04891708F492CF5C9890CF9C
:10CD9000843009F461C00CF45BC0853009F0A5CF84
:10CDA00020919B04211102C080939B0480919B04DD
:10CDB000815080939B04882309F497CF95E095CF09
:10CDC000809133018F5F80311CF4809333018DCFCC
:10CDD0001092330180919D03811113C02091AA12FA
:10CDE0003091AB123093AD122093AC1220912C07EE
:10CDF00030912D0730932F0720932E0781E08093E9
:10CE00009D031092AB121092AA1210922D0710924D
:10CE10002C076BCF10927B0087E480937C0080917D
:10CE20007A00806480937A0060CF80917A0086FDDA
:10CE300026C040917800509179002091AA1230913B
:10CE4000AB12240F351F3093AB122093AA124DCF93
:10CE500010927B0086E4E1CF80917A0086FD11C0BC
:10CE6000409178005091790020912C0730912D0746
:10CE7000240F351F30932D0720932C0736CF92E0D7
:10CE800034CF94E032CF2A9846CF2A9854CF0196D7
:10CE90005ECFACE3B0E0EFE4F7E60C944BF08091AA
:10CEA0006907882369F18091C91410E000E084FFCC
:10CEB00023C08EED92E10E94AC258BE1EEEDF2E114
:10CEC000DE01919601900D928A95E1F710E000E065
:10CED000BE016F5F7F4FCE0181960E94B6C51816C6
:10CEE0003CF4CE0101960E94F5D5080F111DF0CF3C
:10CEF000CE0181960E947B271093ED030093EC03F3
:10CF00000E9458CD10916507312E85E0810F8CAFBE
:10CF1000212E219483E6A82E8DE1B82E9BE8892E40
:10CF200095E0992E01E0011B20E9622E25E0722E8A
:10CF3000111113C080916807882391F180916A01D3
:10CF4000882359F081E090916807911180E024E0F6
:10CF500049E955E0622D0E94A4CC8091C91486FF56
:10CF60003EC01130D9F480916807813049F1809139
:10CF70006A01882309F43EC11F927F926F920F933A
:10CF800081E090916807913009F080E08F930E94D2
:10CF9000F0220F900F900F900F900F9082E04FC0F3
:10CFA00080914F0710924F07882341F20E94804BD7
:10CFB00080916707882311F2EC96E2E10C9467F008
:10CFC00080914F0710924F07882389F210926507CE
:10CFD0000E9462DA80916707882349F2EDCF84FFCF
:10CFE0002DC01130D9F6809168078130D1F0809141
:10CFF0006A01882309F4FEC0BF92AF929F928F927C
:10D000000F9381E090916807913009F080E08F9351
:10D010000E94F0220F900F900F900F900F900F90A2
:10D02000BDCF80914F0710924F07882301F30E94D4
:10D03000631D809167078823D1F2BECF81E0909174
:10D040006A01992309F4D7C0582ED12CC12C412E46
:10D050004318852DE090EC03F090ED03CE14DF042F
:10D0600008F0C9C05112A5C091E0E91AF108EC1806
:10D07000FD088EED92E10E94AC258BE1EEEDF2E130
:10D08000DE01919601900D928A95E1F7F12CBE0197
:10D090006F5F7F4FCE0181960E94B6C518167CF453
:10D0A000CE0101960E94F5D5882389F3EF106BC05D
:10D0B000BE016F5F7F4F8AE797E00E9410D6CE01D6
:10D0C00081960E947B278091C9149091680785FF03
:10D0D00075C0911363C080914F0710924F0788234A
:10D0E00009F45CC019821C828091E11269EF72E13F
:10D0F000882311F06EED72E121E04AE757E0CE019E
:10D1000001960E948027882309F43FC08BE1FE012D
:10D110003196AEEDB2E101900D928A95E1F78091E2
:10D12000C9148F7B8093C914A091BF14AA3080F4D6
:10D1300081E08A0F8093BF148BE18A9FD001112474
:10D14000AF54BC4EEEEDF2E101900D928A95E1F7FD
:10D15000CE0101960E947B271092650782E090E045
:10D16000A0E0B0E080936A0790936B07A0936C07F0
:10D17000B0936D0781E0809367071092990283E076
:10D1800080936A0119CFF39482CF0E94038B6AE7E0
:10D1900077E085E795E00E94D0D5DACF80916A01EB
:10D1A000882339F081E0911380E041E0642D0E94F2
:10D1B000E2CC8FEFC81AD80A53944BCF911759F08D
:10D1C00080916A018823A9F381E090916807911307
:10D1D00080E040E0EBCF80914F0710924F0788230B
:10D1E00079F381EA97E50E94AECD809167078823A5
:10D1F00039F3E2CE82E01F5F9CAD911399CE80930C
:10D200006607DACEFC01A081B1811C92A281B381B4
:10D210008C918F5F8C930280F381E02D90818CE064
:10D22000989F800D1124E3E7F3E113AE84AF0895D6
:10D23000FC0184910895FC0180810895009751F0CC
:10D24000FC0180E09191992331F0907C9038D1F3EA
:10D250008F5FF8CF80E00895119800C087FD43C02C
:10D26000419800C0119A00C000C0119800C086FD0E
:10D2700046C0419800C0119A00C000C0119800C07B
:10D2800085FD3BC0419800C0119A00C000C01198B4
:10D2900000C084FD30C0419800C0119A00C000C099
:10D2A000119800C083FD25C0419800C0119A00C0AC
:10D2B00000C0119800C082FD1AC0419800C0119AA8
:10D2C00000C000C0119800C081FD0FC0419800C08F
:10D2D000119A00C000C0119800C0419800C0119A76
:10D2E00000C000C00895419ABCCF419AF0CF419A46
:10D2F000E5CF419ADACF419ACFCF419AC4CF419A34
:10D30000B9CF90E080E00895CF93DF93DB01F9017E
:10D310009C919130C1F0943080F094509C9388306F
:10D32000D1F480819181009771F00197918380837E
:10D33000480F591FEA01188206C08C3539F49C5FEA
:10D340009C93943041F4DF91CF9108958B3339F75A
:10D3500081E08C93F8CF20813181B9016F5F7F4FDD
:10D3600071836083420F531FEA018883808191811A
:10D370008F3591056CF7E7CF0F931F9381E00091F4
:10D38000C5141091C6142091C7143091C81440914F
:10D39000C1145091C2146091C3147091C414041745
:10D3A00015072607370708F480E01F910F910895AD
:10D3B00090E080E0089520910206833021F425FD5D
:10D3C0000CC024FD0CC030E0A90102C05595479562
:10D3D0008A95E2F7CA018170089581E0089580E09E
:10D3E000089580911E0684FD0BC08091200687FD64
:10D3F00007C090912106937081E019F480E00895B0
:10D4000081E008952FEB280F2A3108F047C0E22F62
:10D41000F0E080911E0690911F06A0912006B09129
:10D42000210604C0B695A795979587952A95D2F7BA
:10D4300080FD02C081700895EC5FF94FE081EE231A
:10D4400041F18091890790918A07E80FF92FF11D2A
:10D45000808190ED980F9A3030F08E3251F48181B6
:10D4600080538A3098F4F093F305E093F20581E05D
:10D4700008958D3211F08B3249F4818190ED980F2F
:10D480009A3088F38E3211F48281EACFF0E0E0E046
:10D49000EACF1092F3051092F205E9CF80E00895EB
:10D4A000CF93DF9385E4AEDF882309F188E04091D4
:10D4B0001E0650911F066091200670912106972F3D
:10D4C0009170C92F90E0D92FCC0FDD1F71FB22275F
:10D4D00020F930E0220F331F220F331FC22B67FBCE
:10D4E000442740F9C42B8C2BDF91CF91089580E025
:10D4F000DECF88DF882341F081E02091F205309172
:10D50000F305232B09F480E00895CF93DF93C091B6
:10D510003407D0913507209729F160913007709139
:10D52000310780913207909133070E9462F16E5F5C
:10D530007F4F24976C177D07ACF47093970360932B
:10D5400096030E94D6D1605A75418F4F9F4F6093CA
:10D5500098037093990380939A0390939B03DF91B0
:10D56000CF910895109298031092990310929A0304
:10D5700010929B03F4CFB0E0A0E0E1ECFAE60C944B
:10D5800054F06B01E9014A3009F4D5C0453109F086
:10D5900081C0DB011296ED91FC91F280968187812A
:10D5A000139A00C00000E6E2F0E03197F0F7092F8F
:10D5B000182FEF2CE29420EFE22230E1B32EBF0CC3
:10D5C000E80188EF49DE00C0000086E290E00197A4
:10D5D000F0F7BFE1BF1508F49BC08F2D80778068FE
:10D5E0003BDE8E2D39DE00C0000086E290E0019720
:10D5F000F0F780E831DE80E02FDE00C0000086E238
:10D6000090E00197F0F78AEF27DE00C0000086E285
:10D6100090E00197F0F7005F1F4F8881807F1CDE4C
:10D6200089918295807F18DEC017D107B1F700C0BD
:10D63000000086E290E00197F0F7F394E0E1EE0E4F
:10D64000FB10BECF1398D6011296ED91FC9180810C
:10D650009281980F92832181921708F09FC1948143
:10D660009F5F94839381890F821710F08FEF820F51
:10D670008383458150E0440F551F70E060E0868150
:10D6800097810E9482F281E0CDB7DEB7E9E00C9489
:10D6900070F0DEC1FB0102811381423309F485C1C0
:10D6A00008F48DC1463409F475C1473409F482C1C8
:10D6B0004B3349F789812B81D80112967C911297BF
:10D6C00013963C91213009F4BFC1233009F0A0C169
:10D6D00048EF480F582F91E0341708F490E031E0FC
:10D6E000541708F030E0492F432B61E0571708F436
:10D6F00060E0462311F4932331F2FA8030E0F9011F
:10D70000E25CFD4FD080265C3D4FF901E08099C17D
:10D7100080EE8F0D8068807F9FDD8F2D8295807FCA
:10D720009BDD00C0000086E290E00197F0F780E802
:10D7300093DD80E861CF0B9A1398399A4198099A42
:10D74000119A139A00C0000086E290E00197F0F76A
:10D7500088E790E0CEE9DFE0FE013197F1F701972D
:10D76000D9F788EF79DD00C0000086E290E00197EC
:10D77000F0F780E271DD80E06FDD00C0000086E23E
:10D7800090E00197F0F780E067DD80E865DD00C09C
:10D79000000086E290E00197F0F780E05DDD80E137
:10D7A0005BDD00C0000086E290E00197F0F7CE015B
:10D7B0000197F1F7CE010197F1F7CE010197F1F74B
:10D7C000CE010197F1F7CE010197F1F7CE01019754
:10D7D000F1F7CE010197F1F7CE010197F1F7CE01F4
:10D7E0000197F1F7CE010197F1F7CE010197F1F71B
:10D7F000CE010197F1F7CE010197F1F7CE01019724
:10D80000F1F72197F1F780E227DD80E425DD00C004
:10D81000000086E290E00197F0F780E21DDD80E6EF
:10D820001BDD00C0000086E290E00197F0F7D0E039
:10D83000C0E08C2F807780680FDD8D2F0DDD00C05C
:10D84000000086E290E00197F0F780E805DD80E0D7
:10D8500003DD00C0000086E290E00197F0F78AEF58
:10D86000FBDC00C0000086E290E00197F0F780E268
:10D87000119800C0419800C0119A00C000C01198D2
:10D8800000C0419800C0119A00C000C0119800C0AB
:10D89000419800C0119A00C000C0119800C0419882
:10D8A00000C0119A00C000C0119800C0419800C08B
:10D8B000119A00C000C0119800C0419800C0119A90
:10D8C00000C000C0119800C0419800C0119A00C06B
:10D8D00000C0119800C0419800C0119A00C000C05B
:10D8E000119800C0419800C0119A00C000C0119862
:10D8F00000C0419800C0119A00C000C0119800C03B
:10D90000419800C0119A00C000C0119800C0419811
:10D9100000C0119A00C000C0119800C0419800C01A
:10D92000119A00C000C0119800C0419800C0119A1F
:10D9300000C000C0119800C0419800C0119A00C0FA
:10D9400000C0119800C0419800C0119A00C000C0EA
:10D9500000C00000E6E2F0E03197F0F7815009F0F6
:10D9600087CF88EF79DC00C0000086E290E0019765
:10D97000F0F7CF5FD05FC03209F05BCF80E06CDCA6
:10D9800080EC6ADC00C0000086E290E00197F0F7CE
:10D99000139879CEF8018581888375CE80E0CDB764
:10D9A000DEB7E9E00C9470F053C0B901C8010E94E1
:10D9B000D4D269CED80111968C91888364CE44313B
:10D9C00091F0473109F05FCE1882D80112968C9100
:10D9D0001297898315968C91159781508A83139697
:10D9E0008C918B8350CED80115964C91159750E0B1
:10D9F000440F551F70E060E016968D919C910E9437
:10DA000082F2F801128280818150838314823BCE9E
:10DA1000381708F438CE871708F435CEFA80E12C91
:10DA2000D12C243070F46ACEBE01C8010E94D4D239
:10DA3000898198819D0D98838E0D8983FF0C09F44F
:10DA400022CEF7FEF6CFF0CF58E0580F482F43CE46
:10DA5000EF92FF920F931F93CF93DF93EC018B0113
:10DA60007A018A859B858617970731F0888199818D
:10DA70000E94C1D41B870A87B701888199810E94BF
:10DA80001ACD2E813F81820F932F911D9F838E830C
:10DA900090E080E0CDB7DEB7E6E00C9473F0B0E044
:10DAA000A0E0E5E5FDE60C9453F0EC017B018A0172
:10DAB0008A859B858617970731F0888199810E9416
:10DAC000C1D4FB86EA8688859985019609F5CC80C4
:10DAD000DA808E81D80EA880B980D5015596ED9157
:10DAE000FC91C5010995C80E780110E0F70121915C
:10DAF0007F0121111FC08E819F81810F911D9F8306
:10DB00008E8390E080E0CDB7DEB7EAE00C946FF052
:10DB1000EE80FF80B801888199810E941ACD8E0D18
:10DB20009F2D911D288539852817390780F681E0BA
:10DB300090E0E9CF4C2D6D2DC5010E9419D5D80E6E
:10DB4000180FD4CFB0E0A0E0E8EAFDE60C9456F060
:10DB5000EC01D62E1CAD0BAD7C0184E0E80EF11C6F
:10DB6000E98DFA8DC7010995412F480F2D2D602FA2
:10DB7000C7010E9419D59BAD890F8BAF81E090E062
:10DB8000CDB7DEB7E7E00C9472F0682F70E090E05C
:10DB900080E00C948FB38091F2059091F30500978B
:10DBA00031F04AE050E070E060E00C9486E760E01D
:10DBB00070E0CB0108958091F2059091F3050097F4
:10DBC00031F04AE050E070E060E00C9459E660E02B
:10DBD00070E0CB010895EFDF97FD0AC0ECDF6F3FE7
:10DBE00071058105910509F02CF4E5DF862F089574
:10DBF00080E008958FEF0895CF93C62F7ADC8823B5
:10DC000011F0E9DFC82F8C2FCF9108958091F20594
:10DC10009091F305892B39F0DEDF91E0811101C08D
:10DC200090E0892F089591E0FCCFCF93DF93C82F28
:10DC3000D62F5FDC882321F0E9DFDF91CF910895B3
:10DC40008C2FE0DB8111F9CF8D2FF7CFB4DFCB0123
:10DC50000895CF93DF93EB014CDC882311F0F6DFBE
:10DC6000EC01CE01DF91CF9108950F931F93CF93D5
:10DC70008091F2059091F3050097D9F0FC018F0196
:10DC8000C1912C2F2F7D81F0C53411F0C536B9F725
:10DC9000F801108270E060E00E9403E5F801C083A3
:10DCA000CF911F910F91089570E060E00E9403E50D
:10DCB000F7CF60E070E0CB01F3CFCF92DF92EF922D
:10DCC000FF926A017B0115DC882319F0CEDF6B011E
:10DCD0007C01C701B601FF90EF90DF90CF900895CF
:10DCE000CF92DF92EF92FF92CF93C82F0E94D6D1AE
:10DCF0006B017C0124EA30E74DE75FE360910801A6
:10DD00007091090180910A0190910B010E9465E9CF
:10DD100087FD18C08AEF90E0A0E0B0E08C0D9D1D5B
:10DD2000AE1DBF1D80935F0690936006A0936106B1
:10DD3000B0936206C0935D01CF91FF90EF90DF90AA
:10DD4000CF90089580E090E0DC01E8CFCF93809100
:10DD50002E06811154C01092AE131092AF13109280
:10DD6000B01310927C1310927B1310927E131092BA
:10DD70007D131092801381E080937F1382E2809361
:10DD800081131092861310928513EAE9F3E128EAD1
:10DD900033E18FEF81932E173F07E1F7C1E0C09386
:10DDA000971323EC31EB30938D1320938C13C09396
:10DDB0008E1310928F131092901390E490939113FE
:10DDC0001092921322EC31EB3093A9132093A813F5
:10DDD00025E531E030937A13209379139EE19093F7
:10DDE0009E1391E190939F139CE190939C138093D9
:10DDF0009B1380939A130E9413D3C0932E0681E045
:10DE000080932D068DE492E29093A1128093A0124C
:10DE10001092A3121092A21253985B9A52985A9A97
:10DE20003898409A0E94EE6510929202CF91089520
:10DE3000FC0180E0309749F09491992331F0907C77
:10DE4000903809F08F5F3196F7CF0895B0E0A0E0E9
:10DE5000ECE2FFE60C9453F0EC015B018A01FB015C
:10DE6000099587FD10C0C82ED12CF12CE12C2196EC
:10DE7000F801C082D182E282F382CE01CDB7DEB753
:10DE8000EAE00C946FF0982F907E903CA9F48F718B
:10DE900090E0B0E0A0E06C017D0156E0CC0CDD1C10
:10DEA000EE1CFF1C5A95D1F7CE010196F50109959C
:10DEB0008F73C82A2296DCCF982F907F903E11F561
:10DEC0008F7090E0B0E0A0E06C017D0136E0CC0CFA
:10DED000DD1CEE1CFF1C3A95D1F7CE010196F50131
:10DEE00009958F73C82A46E0CC0CDD1CEE1CFF1C84
:10DEF0004A95D1F7CE010296F50109958F73C82A8C
:10DF00002396B6CF982F987F903F79F5877090E051
:10DF1000B0E0A0E06C017D0186E0CC0CDD1CEE1CC5
:10DF2000FF1C8A95D1F7CE010196F50109958F73F3
:10DF3000C82A96E0CC0CDD1CEE1CFF1C9A95D1F78C
:10DF4000CE010296F50109958F73C82A26E0CC0C04
:10DF5000DD1CEE1CFF1C2A95D1F7CE010396F501BE
:10DF600009958F73C82A249683CF982F907C903878
:10DF700041F4807C803869F42196CE01F501099541
:10DF8000F8CF8E7F8D3F28F02196CE01F5010995BF
:10DF9000F8CFC12CD12C76016BCF9CE0899F802DCE
:10DFA000112491E0980F90932C062CE0280F2093D9
:10DFB000730730E02E5F3F4F4091AB1342171306BB
:10DFC00019F014F080E008952091AD139217D0F766
:10DFD000662341F08E5F0E94F8D3809173078E5FB5
:10DFE0000E94F8D3809173079091AB13891750F377
:10DFF0002091AD1390912C06291720F31092AE13A7
:10E000008093AF1381E0089520912B06022E000C1F
:10E01000330B8217130641F080932B0668EB73E2F3
:10E0200087E793E10C94C1D40895ACE0B0E0EBE154
:10E03000F0E70C9455F06F3F71058105910509F0EB
:10E0400070F483E793E17EDDE0917B13F0917C1324
:10E050003196849190E02C96E8E00C9471F0F09069
:10E06000AE13E090AF1320912D0621110FC04FE1A8
:10E0700052E26E2D8F2D0E9472D590E080E0F80E56
:10E08000F092AE13E092AF139927E5CFC0907B13C7
:10E09000D0907C1327E733E13A8329832F2D30E09A
:10E0A0003C832B832E2D30E03E832D8318861F82E8
:10E0B0002FEF3FEF3A8729871C861B860FE41DE66A
:10E0C0009E012F5F3F4FAB01BC01C6010E94D1B240
:10E0D000B60187E793E10E94C1D48F819885CFCFA5
:10E0E0004F925F926F927F928F929F92BF92CF9248
:10E0F000DF92EF92FF920F931F93CF93DF93CDB7F1
:10E10000DEB728970FB6F894DEBF0FBECDBF7C01F7
:10E110006A014901FB0190818CE0989F800D1124D8
:10E12000982FF7012081822F880F820F880F80930C
:10E13000AE139093AF134115510559F1FA82E9825C
:10E140007C836B8301111EC0AE014B5F5F4FB40136
:10E15000C6017CDE6C016D817E818F8198856115A1
:10E16000710581059105A9F060DFF70180818F5F5E
:10E170008083853148F3CE01019644D8E5CFB12C98
:10E18000860129C08A01B12C26C045284628472887
:10E19000B1F728960FB6F894DEBF0FBECDBFDF9162
:10E1A000CF911F910F91FF90EF90DF90CF90BF9094
:10E1B0009F908F907F906F905F904F900895B39451
:10E1C00007C0B1102DC001151105C9F20F5F1F4F17
:10E1D00001151105A9F2AE014B5F5F4FB401C601F5
:10E1E00035DE6C014D805E806F807884411451046F
:10E1F00061047104A9F0F0E24F1651046104710446
:10E2000001F3D301C2018D97A109B1090297A105BC
:10E21000B10530F04BE2441651046104710479F603
:10E22000F7018081482F4B0D5527551F4631510569
:10E2300034F0853020F0CE0101960E94026981E021
:10E24000411451046104710409F480E0B80EF7012F
:10E2500080818B0D8083BB2009F497CFBA94AE01E7
:10E260004B5F5F4FB401C801F1DD8C016D817E8190
:10E270008F819885DADEEFCFCF93DF93FC0125AD58
:10E28000211104C021E025AF0E9413D3C09179135E
:10E29000D0917A13E091A813F091A91382E0099527
:10E2A000E091A813F091A91381E0099530E020E0F6
:10E2B00044E1BE0187E793E10E940ED32AEA33E1ED
:10E2C00047E1BE0187E793E10E940ED3E091A813D6
:10E2D000F091A91380E00995DF91CF9108954F92B5
:10E2E0005F926F927F928F929F92AF92BF92CF92E6
:10E2F000DF92EF92FF92CF93DF9300D000D0CDB7A3
:10E30000DEB70E94D6D16B017C0180915D018F3F09
:10E31000C1F10E94D6D180905F0690906006A090D7
:10E320006106B0906206681979098A099B0997FD10
:10E3300028C080915F13909160138F5F8F70891751
:10E3400001F1E0915D01E53008F0DCC024E0E29FDE
:10E35000F0011124EE5BFD4F80819181A281B38198
:10E3600089839A83AB83BC8320E030E0A901BE019E
:10E370006F5F7F4F85E791E00E94ADC78FEF80937D
:10E380005D010E94EE658091930282FFC4C080917E
:10E390006E0681111DC091E090936E0680919802E7
:10E3A000892780934F071092980283E080936A0137
:10E3B000109293020E94D6D16C507E4F8F4F9F4F88
:10E3C00060939402709395028093960290939702C3
:10E3D00080916A0690916B06A0916C06B0916D06D3
:10E3E000A7019601281B390B4A0B5B0BDA01C90107
:10E3F000B7FF05C080919902882309F4C5C1D701F0
:10E40000C6018C599F4FAF4FBF4F80936A069093C0
:10E410006B06A0936C06B0936D0660919202062E77
:10E42000000C770B77FF03C071956195710990918E
:10E43000920280916906981371C0633008F06EC033
:10E44000109292028091920280936906643008F0E3
:10E4500075C080914F078111F3C080917113909125
:10E4600072138B509C4741F480915E01882309F41C
:10E47000F9C0815080935E010E9454308090A307C0
:10E480009090A407A090A507B090A60781110E94C4
:10E490006130D501C4013AE0B695A7959795879567
:10E4A0003A95D1F7009741E0A407B10520F08FEF2E
:10E4B0009FEFA0E0B0E09695879520916A01211129
:10E4C000E3C03091990231118BC180917113909109
:10E4D00072138B509C4709F46AC180919A02811192
:10E4E00066C18091650690916606A0916706B0911D
:10E4F0006806C81AD90AEA0AFB0AF7FC66C10E9434
:10E50000EE4763C180916B0190916C01A0916D0108
:10E51000B0916E0125CF10926E065ACF633009F08C
:10E5200091CF8091920287FD07C081E0880F880F0C
:10E530008093920264E086CF8FEFF8CF80917207CC
:10E5400021E030E040E050E0882309F456C080909C
:10E550006E0790906F07A0907007B09071078114BC
:10E560009104A104B104E9F170E090E080E00E9420
:10E5700069E920E030E040E85EE30E94CAE92B014F
:10E580003C01C701B601681979098A099B090E94F3
:10E5900069E99B01AC01C301B2010E94FAF020E0DD
:10E5A00030E04AE754E40E94CAE94B015C0120E0F4
:10E5B00030E040EA52E40E94E6F124E630E040E038
:10E5C00050E087FF12C020E030E040EF51E4C50189
:10E5D000B4010E94E6F12AE030E040E050E087FF1D
:10E5E00004C021E030E040E050E0C0926E07D092DD
:10E5F0006F07E0927007F0927107A09192020A2EC5
:10E60000000CBB0B0E94DBEF24E030E040E050E068
:10E610000E94B5EF80916A0790916B07A0916C07FB
:10E62000B0916D07820F931FA41FB51F80936A07D7
:10E6300090936B07A0936C07B0936D0710929202B2
:10E64000D701C6018856954CAF4FBF4F80936506E2
:10E6500090936606A0936706B093680681E0809366
:10E660006A01FBCE8CE080935E01809163069091FD
:10E670006406009729F001979093640680936306DF
:10E6800081E080936A01F8CE009741F040916306E3
:10E69000509164064817590708F017CF80919902E6
:10E6A000811111C0223038F0243008F43FC02430EA
:10E6B00011F410926A0183E793E1DEDD81E080933B
:10E6C00069078093990283E09FDC81E08093971330
:10E6D000E0917113F091721309951092690780917E
:10E6E0009902811127C010924F0780917113909168
:10E6F00072138B509C4709F0F0CE0E94D6D1DC01FA
:10E70000CB018C199D09AE09BF09809063069090DA
:10E710006406B12CA12C88169906AA06BB0608F03F
:10E72000D4CE9093640680936306CFCE81E080932D
:10E730006A01C1CF87E793E10E9491D491E08111F2
:10E7400001C090E090939902882369F2809171133F
:10E75000909172138B509C47B9F40E94D6D1DC0182
:10E76000CB018C199D09AE09BF09C0906306D090FA
:10E770006406F12CE12CC816D906EA06FB0620F443
:10E7800090936406809363060F900F900F900F9004
:10E79000DF91CF91FF90EF90DF90CF90BF90AF903F
:10E7A0009F908F907F906F905F904F90089548E971
:10E7B000C40E4AE3D41EE11CF11CC0926506D0923F
:10E7C0006606E0926706F0926806809199028111D0
:10E7D000DBCF80916A018130B9F610926A01D4CF03
:10E7E000009709F470CF52CFACE0B0E0EAEFF3E766
:10E7F0000C9455F0F090AE13E090AF1320912D06DD
:10E80000211112C04FEF51E26E2D8F2D0E9472D553
:10E8100090E080E0F80EF092AE13E092AF139927EB
:10E820002C96E8E00C9471F0C0907B13D0907C1390
:10E8300027E733E13A8329832F2D30E03C832B8374
:10E840002E2D30E03E832D8318861F827A876987BC
:10E850001C861B860FE41DE69E012F5F3F4F48E19B
:10E8600059E6BC01C6010E9466B3B60187E793E191
:10E870000E94C1D48F819885CDCFA4E0B0E0E3E4BD
:10E88000F4E70C9451F07C01062F5A01122F862FC9
:10E89000660F990B9C012A5C3D4F690186E0882E2A
:10E8A000912C11160CF03DC0AE014F5F5F4F68E137
:10E8B00079E6C701CBDA7C0169817A818B819C8101
:10E8C000611571058105910561F16D337105810552
:10E8D000910509F450C06E3771058105910509F461
:10E8E0004AC06A3271058105910501F507FF11C023
:10E8F00083E492E20E3F11F08FE392E236E01302DE
:10E90000B001112471DF66E070E00E941DF0161B5B
:10E9100060C065E470E080E090E087DB115069F54D
:10E9200010E0812F2496ECE00C946DF064327105B8
:10E930008105910571F4A114B104D1F0E6E01E0245
:10E94000B0011124C50150DFB4010E941DF0161B57
:10E95000A8CF603471058105910551F41150F6017D
:10E960006081062E000C770B880B990B5EDB99CF2C
:10E970005CDB115096CF07FDBBCF61E089819A81A6
:10E98000AB81BC81CD97A105B10509F460E0600FB2
:10E990006A30A4F01150862F6AE00E94FCEF092F24
:10E9A000682F880F770B605D7F4F072E000C880B58
:10E9B000990B3BDB112309F4B3CF602F062E000C1B
:10E9C000770B605D7F4F072E000C880B990B2DDBBA
:10E9D0001150112309F4A4CF86E01802B0011124CC
:10E9E000C70102DF66E070E00E941DF0161B99CFA0
:10E9F000E3E7F3E183AF64AF6FEF7FEFCA01F4CEDB
:10EA0000ACE0B0E0E6E0F5E70C9455F0F090AE1322
:10EA1000E090AF1320912D06211112C04FED51E26D
:10EA20006E2D8F2D0E9472D590E080E0F80EF0924E
:10EA3000AE13E092AF1399272C96E8E00C9471F096
:10EA4000C0907B13D0907C1327E733E13A8329836E
:10EA50002F2D30E03C832B832E2D30E03E832D8301
:10EA600018861F827A8769871C861B860FE41DE63D
:10EA70009E012F5F3F4F4BE159E6BC01C6010E944A
:10EA800066B3B60187E793E10E94C1D48F81988570
:10EA9000CDCF6FEF7FEFB4CFB0E0A0E0E2E5F5E7D8
:10EAA0000C9453F05C016B01C3D9E82EC6010E949F
:10EAB0001E69F12C03E110E0081B1109C5E20E15D7
:10EAC0001F050CF4CFE18C2F90E09C012E5F3F4F8F
:10EAD0004091AB134217130609F08CF5099720916A
:10EAE000AD13281719065CF1409175075091760710
:10EAF000609174071092AE13C093AF1325E1C50166
:10EB0000BCDED1E0C114D104A9F06AE370E080E07A
:10EB100090E08BDA0E151F05A4F4C45F8091AB134F
:10EB2000C81740F02091AD134C2F4950550B2417B6
:10EB300015064CF4CDB7DEB7EAE00C946FF0D0E0E8
:10EB4000E1CFDD23B9F3802F880F080F000F00936A
:10EB5000AE13C093AF1360E270E080E090E065DA3E
:10EB6000C60197DFE7CFACE0B0E0E9EBF5E70C9446
:10EB700051F0982F862F6A017901B02E692F0DDA96
:10EB8000882309F487C010912D06C701002371F175
:10EB90004FD9A82E80907B1390907C13111142C006
:10EBA0002FEF3FEF122F23E12A1940917507509163
:10EBB000760760917407C60160DEAA2009F46AC076
:10EBC000B6E08B9F600111246AE370E080E090E082
:10EBD0002CDA57E0C516D10408F442C060E270E0B8
:10EBE00080E090E022DAC81AD90AF3CF0E941E69A9
:10EBF000A82E80907B1390907C13112389F2FE0144
:10EC000033968AE0DF011D928A95E9F787E793E161
:10EC10009A83898308E21DE69E012F5F3F4F4BE1F7
:10EC200059E612C0FE0133968AE0DF011D928A95F3
:10EC3000E9F787E793E19A83898308E21DE69E015D
:10EC40002F5F3F4F48E159E6B701C4010E9466B308
:10EC5000B40187E793E10E94C1D42F813885A2CF08
:10EC600040917307212F30E0A6E0AA9EC001112435
:10EC70002E5F3F4F281739070CF49C0180E8821B58
:10EC80008093AE134093AF13BB2041F06FEF7FEF43
:10EC9000C701AADD2C96ECE00C946DF0C701F9DEFB
:10ECA000F9CFE3E7F3E183AF64AFCA01F2CE0C948E
:10ECB000ECB34F925F926F927F928F929F92BF922E
:10ECC000CF92DF92EF92FF920F931F93CF93DF9338
:10ECD00010922306109222062FE32093260610920C
:10ECE00025061092240610921E0610921F061092FE
:10ECF0002006109221069C01F90190812F5F3F4F61
:10ED00009032D1F39E34C9F4818190ED980F9A30FE
:10ED100020F08D3211F08B3281F432969F012F5FFB
:10ED20003F4F808180538A3008F46DC09F012F5F70
:10ED30003F4F8081803209F468C0F0938A07E093E6
:10ED400089078F010F5F1F4FC0816AE270E0C80121
:10ED50000E949CF2009731F0FC0131978081803253
:10ED6000E1F31182CD3421F0C43511F0C734D9F567
:10ED7000F80180810F5F1F4F8032D1F380538A30BA
:10ED800090F5C093260690E080E06AE0AF014F5F07
:10ED90005F4F689F9001699F300D1124C901C09792
:10EDA0002081820F911D27FD9A95FA012081205321
:10EDB0002A3060F39093250680932406DF01319674
:10EDC0002C912032D9F3CD3461F58E31910539F093
:10EDD000F0F48731910519F08C31910511F5B0935C
:10EDE0002306A0932206DF91CF911F910F91FF90F0
:10EDF000EF90DF90CF90BF909F908F907F906F901B
:10EE00005F904F900895F90189CFF9018FCF853731
:10EE1000910538F08737910510F3803A13E0910798
:10EE2000F1F28090890790908A0740E050E0BA01A3
:10EE300030E020E0C12CD12C7601C394FD01319645
:10EE4000DC91DD2309F484C0D132F1F4CD34E1F456
:10EE500080329105C9F440931E0650931F066093BB
:10EE6000200670932106F0932306E093220663E2C6
:10EE700070E0CF010E949CF2009709F4B4CFFC012E
:10EE80001082B1CFDF01DACFD154DA3108F05BC0A4
:10EE9000DF011D91103291F0A0EDA10FAA30E8F032
:10EEA0001E3271F4A181A053AA30B8F021153105AA
:10EEB00019F49F0121503109B12C13C0FD01E8CF95
:10EEC0001D3211F01B3291F7A181B0EDBA0FBA30AB
:10EED00020F0AE3259F7A281E6CFBE2EB818309797
:10EEE00059F3AD2FB0E02601370104C0440C551C86
:10EEF000661C771CDA95D2F74429552966297729AB
:10EF0000AC5FB94FBC92A081A154AA3108F4BACF2A
:10EF1000DF01D191DD2309F491CF00EDB02EBD0EBC
:10EF200019E01B15A8F713EDB12EBD0E11E01B154E
:10EF300078F7DB3269F3FD013196DC91D03209F0CC
:10EF40007DCFDF01F8CF21153105E9F69D01DBCF3B
:10EF5000309323062093220640931E0650931F06EB
:10EF600060932006709321063ECFFC016591759158
:10EF70008591949108958F929F92AF92BF92CF9274
:10EF8000DF92EF92FF92CF93DF93EC018090B40277
:10EF90009090B502A090B602B090B70220E030E0A9
:10EFA000A901C501B4010E9465E9882309F452C092
:10EFB000C880D980EA80FB80A7019601C501B40111
:10EFC0000E9465E918160CF04AC02091EE053091B8
:10EFD000EF054091F0055091F105C701B6010E947F
:10EFE00065E9882321F1C092EE05D092EF05E09209
:10EFF000F005F092F1052091EA053091EB05409182
:10F00000EC055091ED05C701B6010E94CAE99B01CC
:10F01000AC0160E070E080E89FE30E9482F06093C2
:10F020004A0170934B0180934C0190934D01609184
:10F030004A0170914B0180914C0190914D01DF91FB
:10F04000CF91FF90EF90DF90CF90BF90AF909F90C7
:10F050008F90089560E070E080E89FE3F0CF60E07B
:10F0600070E0CB01ECCFB0E0A0E0E9E3F8E70C946E
:10F070004DF0EC0120917C0330917D0340917E03A3
:10F0800050917F03688179818A819B810E9482F0FF
:10F090004B015C01209180033091810340918203F8
:10F0A000509183036C817D818E819F810E9482F0CB
:10F0B0006B017C01A50194016091420170914301B3
:10F0C00080914401909145010E9465E9882309F4EB
:10F0D00054C08092420190924301A0924401B092A8
:10F0E00045012091E2053091E3054091E4055091FE
:10F0F000E505C501B4010E94CAE92B013C010E944B
:10F1000093F14B015C0120E030E040EA50E40E94C2
:10F1100065E9181634F4812C912CC0EAAC2EC0E4B9
:10F12000BC2E20E030E0A901C501B4010E94E6F147
:10F1300087FF03C0812C912C5401A5019401C301C8
:10F14000B2010E9482F06093DA057093DB05809330
:10F15000DC059093DD05C501B4010E9462F1609366
:10F16000D805062E000C770B6F5F7F4F6630710558
:10F1700014F066E070E06093D605D09140011091E4
:10F18000D805A701960160914601709147018091D1
:10F190004801909149010E9465E9811123C0D11372
:10F1A00075C02091BE053091BF054091C0055091BA
:10F1B000C1056091DA057091DB058091DC059091C5
:10F1C000DD050E94CAE92091C2053091C305409136
:10F1D000C4055091C5050E9483F0CDB7DEB7E0E1CC
:10F1E0000C9469F0C0924601D0924701E092480128
:10F1F000F09249012091E6053091E7054091E8053C
:10F200005091E905C701B6010E94CAE94B015C01B2
:10F210000E9493F16B017C0120E030E040EA50E471
:10F220000E9465E9181634F4C12CD12CB0EAEB2EFB
:10F23000B0E4FB2E20E030E0A901C701B6010E9436
:10F24000E6F187FF03C0C12CD12C7601A7019601FE
:10F25000C501B4010E9482F06093DE057093DF0562
:10F260008093E0059093E105C701B6010E9462F129
:10F270006093D905062E000C770B6F5F7F4F6630C9
:10F28000710514F066E070E06093D705C091D90570
:10F29000D11305C0809141018C1709F470C0809191
:10F2A000D8059091D90590934101809340010C2E8F
:10F2B000000CDD0B27E01203C0011124FC01EC0F50
:10F2C000FD1FEE0FFF1FEE0FFF1FE854FD4F2081C3
:10F2D0003181428153812093D2053093D3054093ED
:10F2E000D4055093D5050091D705002E000C110BC5
:10F2F000FC01E00FF11FEE0FFF1FEE0FFF1FE854A0
:10F30000FD4F60817181828193810E9482F06093C0
:10F31000CE057093CF058093D0059093D1052091B1
:10F32000D60537E02303F0011124CE0FDF1FCC0FE9
:10F33000DD1FCC0FDD1FC854DD4F288139814A8184
:10F340005B812093CA053093CB054093CC05509345
:10F35000CD05E00FF11FEE0FFF1FEE0FFF1FE8546A
:10F36000FD4F60817181828193810E9482F0609360
:10F37000C6057093C7058093C8059093C905809012
:10F38000DE059090DF05A090E005B090E1052091AA
:10F39000CE053091CF054091D0055091D105C501E2
:10F3A000B4010E94CAE92091D2053091D305409161
:10F3B000D4055091D5050E9483F06B017C01C09269
:10F3C000C205D092C305E092C405F092C505209114
:10F3D000C6053091C7054091C8055091C905C501C2
:10F3E000B4010E94CAE92091CA053091CB05409131
:10F3F000CC055091CD050E9483F0A70196010E9493
:10F4000082F06093BE057093BF058093C005909312
:10F41000C105C7CEACE0B0E0E0E1FAE70C945AF0E9
:10F42000182F882379F020E030E0A901609184034F
:10F430007091850380918603909187030E9465E90E
:10F440008823F1F08091B3028117D1F00E94802DC2
:10F450008CE0EAE2F2E0DE01119601900D928A95CD
:10F46000E1F7CE010196FFDD8091B302882361F0C0
:10F4700085E791E00E94D62D1092B3020E9493403E
:10F480002C96E3E00C9476F081E08093B30285E75C
:10F4900091E00E94A22DF2CFCF92DF92EF92FF92E5
:10F4A00080E0B8DF109280031092810310928203F3
:10F4B0001092830310927C0310927D0310927E03BE
:10F4C00010927F03109288031092890310928A038E
:10F4D00010928B031092840310928503109286037E
:10F4E0001092870348EB52E027E0C12CD12C60EC4E
:10F4F000E62E6FE7F62E90E080E0FC01EE0FFF1F96
:10F50000EE0FFF1FE40FF51FC082D182E282F3826B
:10F5100001968730910589F72150445E5F4F211194
:10F52000EACFFF90EF90DF90CF9008954F925F92D7
:10F530006F927F928F929F92AF92BF92CF92DF9203
:10F54000EF92FF921F93CF93DF93EC01162F209140
:10F55000B4023091B5024091B6025091B702688171
:10F5600079818A819B810E9465E9882309F497C08B
:10F57000B090B30280E04EDFC880D980EA80FB8083
:10F5800020E030E0A901C701B6010E94E6F187FF43
:10F5900003C0C12CD12C7601C092B402D092B50226
:10F5A000E092B602F092B7022DEB37E346E855EB56
:10F5B000C701B6010E9465E987FD0BC02DEB37E35B
:10F5C00046E855E3C701B6010E94E6F118160CF0B3
:10F5D00076C0A701960160E070E080E89FE30E949A
:10F5E000FAF06093EA057093EB058093EC05909335
:10F5F000ED0580EF9FEFA9E7B4EC8093EE059093C3
:10F60000EF05A093F005B093F105BB2009F447C0C6
:10F61000409075015090760160907701709078016C
:10F620008090790190907A01A0907B01B0907C014C
:10F63000C0907D01D0907E01E0907F01F09080012C
:10F6400081E0E8DE112359F1A30192016091750177
:10F650007091760180917701909178010E9465E91F
:10F6600081111BC0A50194016091790170917A010B
:10F6700080917B0190917C010E9465E981110DC010
:10F6800020917D0130917E0140917F015091800158
:10F69000C701B6010E9465E981110E94E140DF9136
:10F6A000CF911F91FF90EF90DF90CF90BF90AF90E0
:10F6B0009F908F907F906F905F904F90089560E043
:10F6C00070E0CB018ECF8F929F92AF92BF92CF927C
:10F6D000DF92EF92FF92C0908403D0908503E09078
:10F6E0008603F090870320E030E0A901C701B6014E
:10F6F0000E9465E98823E1F1A701960160E070E0CE
:10F7000080E89FE30E94FAF06B017C0180908803FF
:10F7100090908903A0908A03B0908B0320E030E0A2
:10F72000A901C501B4010E9465E9882329F1A50159
:10F73000940160E070E080E89FE30E94FAF0C092DC
:10F74000E205D092E305E092E405F092E5056093CE
:10F75000E6057093E7058093E8059093E905FF902F
:10F76000EF90DF90CF90BF90AF909F908F900895D3
:10F77000C12CD12C7601CACF60E070E0CB01DFCF85
:10F78000CF92DF92EF92FF926B017C0183E3C81668
:10F79000D104E104F10470F082E3C81AD108E10851
:10F7A000F10862E370E080E090E00E944DD10E9499
:10F7B000C22AECCFC701B6010E944DD10E94C22AD5
:10F7C000FF90EF90DF90CF900895BC0190E080E033
:10F7D0000C948FB380918707813069F09091C914A0
:10F7E00092FB882780F992FF07C097FB882780F952
:10F7F00091E08927089581E008959091C91494FBC0
:10F80000882780F994FF06C081E09091C61291117B
:10F8100001C080E00895A4E0B0E0E1E1FCE70C94D1
:10F820004DF01092720780914F0710924F07882376
:10F8300061F020E040E070E060E08FE893E60E9435
:10F84000B2462496E0E10C9469F0209110013091C9
:10F85000110140916A0750916B07CA01820F931FF3
:10F860002436310509F01DC44730510544F0069790
:10F870008A3091050CF024C48AE090E02BC40696EF
:10F880004A3F5F4FACF380916907882309F4C8C1F0
:10F890006091B2127091B312072E000C880B990B75
:10F8A0000E946BE9B1E0B9832091AE123091AF12A2
:10F8B0004091B0125091B1120E94E6F118160CF06E
:10F8C00019826091340770913507072E000C880B60
:10F8D000990B0E946BE920913007309131074091DC
:10F8E0003207509133070E94E6F118161CF4E981A3
:10F8F000E260E983C980C0925E06C0907501D09035
:10F900007601E0907701F0907801809179019091F3
:10F910007A01A0917B01B0917C0189839A83AB83AA
:10F92000BC8380907D0190907E01A0907F01B0907B
:10F93000800120E030E04AE754E4C501B4010E94B0
:10F94000CAE92B013C0120E030E0A901C501B40166
:10F950000E9465E920E030E040EA50EC87FD04C0F9
:10F9600020E030E040EA50E4C301B2010E9483F09D
:10F970002DEC3CEC4CEC5DE30E94CAE90E9462F184
:10F980004B015C0180E2B7FE09C0B094A094909452
:10F990008094811C911CA11CB11C8DE280939B0260
:10F9A00060E290E1891697E29906A104B1048CF017
:10F9B000C501B40120E137E240E050E00E94B5EF1C
:10F9C000CA01B9012AE030E040E050E00E94B5EF02
:10F9D000605D60939C0260E2A8EE8A16A3E09A063E
:10F9E000A104B1048CF0C501B40128EE33E040E07D
:10F9F00050E00E94B5EFCA01B9012AE030E040E0D2
:10FA000050E00E94B5EF605D60939D02C501B401B6
:10FA100024E630E040E050E00E94B5EF6AE0462E78
:10FA2000512C612C712CCA01B901A30192010E94D1
:10FA3000B5EF605D60939E02C501B401A301920120
:10FA40000E94B5EF4B01CA01B901A30192010E94C6
:10FA5000B5EF882009F44EC32EE220939F02605D2B
:10FA60006093A002B0E38B0E8092A1026BE972E07A
:10FA700086E596E00E94A7F220E030E0A901C701E8
:10FA8000B6010E9465E920E030E040E05FEB87FDD1
:10FA900004C020E030E040E05FE3C701B6010E940F
:10FAA00083F00E9462F1CB010E949245BC0181E586
:10FAB00096E00E94A7F220E030E0A90169817A81F6
:10FAC0008B819C810E9465E920E030E040E05FEBA3
:10FAD00087FD04C020E030E040E05FE369817A8187
:10FAE0008B819C810E9483F00E9462F1CB010E9475
:10FAF0009245BC018CE496E00E94A7F28091C91463
:10FB000083FD0AC37ADE882309F409C38091C114F6
:10FB10009091C214A091C314B091C4140097A10590
:10FB2000B10509F4FCC2BC01CD016D597F4F8F4F67
:10FB30009F4F24E630E040E050E00E9493EF609158
:10FB4000C5147091C6148091C7149091C8140E9476
:10FB500093EF29830E94D1444B015C01162F8091C1
:10FB60005C01C9808C15C1F0C0925C0128E4C29E82
:10FB7000B001112490E080E00E9469E92AE037EDAD
:10FB800043E25CE30E94CAE90E9467F160934B067E
:10FB9000C110C7C21092460680915B01181709F484
:10FBA0003FC080925B01C501B40120E13EE040E02E
:10FBB00050E00E9493EF690189019CE3492E512C8A
:10FBC000612C712CC501B401A30192010E9493EF35
:10FBD0004B015C01CA01B901A30192010E9493EF9C
:10FBE000C114D10409F0C4C29F928F927F936F9386
:10FBF00083E692E29F938F9386E396E09F938F93A1
:10FC00000E94FEE80FB6F894DEBF0FBECDBF85E0C0
:10FC1000982F990F990F891B880F8058809335066C
:10FC20000E94D6D100913006109131062091320603
:10FC3000309133066B017C01C01AD10AE20AF30A43
:10FC40009701860137FD11C020912F062095209342
:10FC50002F066A547C4F8F4F9F4F609330067093EE
:10FC600031068093320690933306D0902F06D982C6
:10FC700081E00E9404708091AB13873180F4809101
:10FC8000AD13843060F086E4E82E83E2F82E03E1C1
:10FC900026E044E064E087E793E10E9497D58091F5
:10FCA0005E06982F927048E00CE081FD02C042E1B0
:10FCB00002E08091AB13843180F48091AD138417FE
:10FCC00060F0992309F473C282E293E27C0123E09D
:10FCD00060E587E793E10E9497D58091AB1384316B
:10FCE000C0F48091AD138230A0F0C980CC2009F41B
:10FCF00061C28091A707882309F45CC286EE92E274
:10FD00007C0102E123E042E068E687E793E10E949C
:10FD100097D58091AB138C3108F09DC08090AE12C6
:10FD20009090AF12A090B012B090B112C090B212E9
:10FD3000D090B312843198F48091AD13883078F06C
:10FD400080915E0680FF39C288E992E27C010CE076
:10FD500022E048E069E387E793E10E9497D580912C
:10FD6000AB13883040F4D7FE2BC24CE752E267E079
:10FD700087E30E94F8748091AB138C31B0F48091CA
:10FD8000AD13843190F020E030E040E05FE3C50146
:10FD9000B4010E9483F00E9462F177FF34C24CE705
:10FDA00052E26CE187E30E94F874C0903007D09073
:10FDB0003107E0903207F09033078091AB13883021
:10FDC00060F4809134079091350797FF3FC24CE76C
:10FDD00052E267E081E50E94F8748091AB138C31A8
:10FDE000B0F48091AD13843190F020E030E040E039
:10FDF0005FE3C701B6010E9483F00E9462F177FFC2
:10FE000047C24CE752E26CE181E50E94F8748091B0
:10FE1000AB138C3100F58091AD138431E0F080910B
:10FE2000A7078823C1F024E6829FC00111248158CE
:10FE30009F4F6FEF70E00E941DF0CB010E941146B2
:10FE4000AC016CE187E60E94517665E270E080E0EB
:10FE500090E00E941570D1DC882379F18091AB137A
:10FE6000843358F58091AD138A3238F107E028E0E9
:10FE70004AE26AE287E793E10E943ED405E022E08D
:10FE80004CE262E387E793E10E943ED424E04AE03B
:10FE900061E38AE20E940ED46091791370917A1323
:10FEA00082E3809393138BE28093941323E933E1ED
:10FEB00042E387E793E10E940ED38091AB13853331
:10FEC00050F48091AD13813330F024E04AE461E3D3
:10FED00086E30E940ED48091AB13843368F4809142
:10FEE000AD13823348F002E020914B0642E367E312
:10FEF00087E793E10E943ED48091AB138033D8F41E
:10FF00008091AD138832B8F080914606882361F065
:10FF100046E456E060E387E30E94517665E270E0D4
:10FF200080E090E00E94157046E356E060E3809127
:10FF300035060E9451768091AB13883208F060C07C
:10FF40008091AD138D3108F45BC02BE040E86DE18A
:10FF500080E00E940ED48091AB13873208F050C02D
:10FF60008091AD138F3108F44BC083E08093AE13C2
:10FF700016E21093AF1368E570E080E090E00E9415
:10FF800015708BE08093AE131093AF13C980CC2013
:10FF900009F4A1C181E596E00E94497588E2809349
:10FFA000AE1316E21093AF1369E570E080E090E0C5
:10FFB0000E94157080E38093AE131093AF13C98035
:10FFC000CC2009F4ABC18CE496E00E9449758DE425
:10FFD0008093AE1316E21093AF136AE570E080E0F1
:10FFE00090E00E94157085E58093AE131093AF13D7
:10FFF000C980CC2009F4B5C186E596E00E94497518
:020000021000EC
:100000008091AB13833338F58091AD138B3218F1A7
:1000100083E00E94047083E08093AE1383E38093B7
:10002000AF1366E070E080E090E00E94157081E020
:100030000E94047080911001909111010E9411465C
:10004000AC0163E38CE00E94517665E270E080E0F1
:1000500090E00E9415708091AB13813408F0F1CBD1
:100060008091AD13863308F4ECCB1092AE138EE37F
:100070008093AF138FE390E10E941E69182F8631A1
:1000800008F092C18FE390E10E944975153109F49F
:10009000D8CB60E270E080E090E00E9415701F5FB6
:1000A000F5CF243631054CF48536910504F58A30B8
:1000B000910534F48AE090E009C084369105BCF0E3
:1000C000883EA3E09A0714F087EE93E028173907DB
:1000D00009F4D9CB909311018093100110926A0713
:1000E00010926B0710926C0710926D07CCCB84E6D0
:1000F00090E0F0CF662351F02EE220939F02605DE6
:100100006093A00280E28093A102B0CC80E2809351
:10011000A00280939F02F6CFE4E6E9831BCD19820B
:1001200019CD498180E2443628F0842F64E60E948C
:10013000F0EF805D80939F02698190E26A3040F029
:100140002AE0862F622F0E94F0EF0E94F0EF905D70
:100150009093A00289816AE00E94F0EF905D9093F5
:10016000A1026FE972E086E496E00E94A7F214CD46
:100170000436110538F47F936F93DF92CF9287E5B1
:1001800092E238CD7F936F93DF92CF928DE492E22B
:100190009F938F9386E396E09F938F930E94FEE850
:1001A0000FB6F894DEBF0FBECDBF86E031CD8CE137
:1001B00093E28CCD80EB92E2A3CD80E892E2C6CDB3
:1001C000C6010E941146FC01808193E0803229F42F
:1001D000818192E0803209F491E043E050E0491BD4
:1001E00051094E0F5F1F892F880F880F981B892F89
:1001F00067E0805C0E94517669E070E080E090E00A
:100200000E941570B8CDCB010E941146FC0180817F
:1002100093E0803229F4818192E0803209F491E008
:1002200043E050E0491B51094E0F5F1F892F880F93
:10023000880F981B892F6CE1805C0E94517669E0E1
:1002400070E080E090E00E941570AFCD0E941146F2
:10025000FC01808193E0803229F4818192E0803238
:1002600009F491E043E050E0491B51094E0F5F1F34
:10027000892F880F880F981B892F67E0865A0E9464
:10028000517669E070E080E090E00E941570A5CDA5
:10029000CB010E941146FC01808193E0803229F459
:1002A000818192E0803209F491E043E050E0491B03
:1002B00051094E0F5F1F892F880F880F981B892FB8
:1002C0006CE1865A0E94517669E070E080E090E02F
:1002D0000E9415709CCD87E00E94403C80FF13C0B7
:1002E00001E516E0D8016D918D01662309F456CE23
:1002F0006F320CF06FE3062E000C770B880B990B16
:100300000E941570EFCF8091770780FD43CE6FEF8D
:100310007FEF87E792E20E94F47340CE87E00E946D
:10032000403C81FF13C00CE416E0D8016D918D01B3
:10033000662309F44CCE6F320CF06FE3062E000CEE
:10034000770B880B990B0E941570EFCF8091770780
:1003500081FD39CE6FEF7FEF87E792E20E94F47361
:1003600036CE87E00E94403C82FF13C006E516E0CF
:10037000D8016D918D01662309F442CE6F320CF0E5
:100380006FE3062E000C770B880B990B0E941570FB
:10039000EFCF8091770782FD2FCE6FEF7FEF8FE653
:1003A00092E20E94F4732CCE81E0C980C11001C09A
:1003B00080E0909134068917C9F0D0903E10D98220
:1003C000809334068FE390E10E941E69D81608F0EE
:1003D00054C029812F5F2983E22FF0E0E15CFF4EBA
:1003E0008081807C8038A9F320933E1000913E10DC
:1003F00010E0015C1F4EC8010E941E69898360E8FD
:1004000070E0C8010E9400754981453108F019CAA1
:1004100060E270E080E090E00E94157069816431D4
:1004200009F40FCA60E270E080E090E00E9415706D
:100430008981833109F405CA60E270E080E090E0D0
:100440000E9415709981923109F4FBC9292F30E07F
:100450002E5F3F4F4AEF4203B001439F700D1124BE
:1004600060587F4F8FE390E10E94007560E270E07A
:1004700080E090E00E941570E4C910923E10B6CF63
:1004800080918707823059F0B8D9882349F080914C
:10049000C91482FB882780F991E08927089581E0BB
:1004A000089581E00895DC01EC918E2F90E0FC012D
:1004B000EE0FFF1FE80FF91FEA5DFC4E80818F777A
:1004C00080830895892B79F41092900082E08093C4
:1004D00091001092950010929400C19A8091710041
:1004E0008260809371000895B0E0A0E0EAE7F2E84E
:1004F0000C9450F0EC017B0188818C3008F0A4C092
:1005000090E0FC01EE0FFF1FE80FF91FEA5DFC4EC3
:1005100080818F770E9417B619821A8288812CE019
:10052000622F0E94F0EF829FB001112430E020E0A2
:10053000AB01420F531FFA01EE0FFF1FE40FF51F2F
:10054000EA5DFC4E908197FD07C02F5F3F4F2C3036
:10055000310571F790E0B6DF7880072D10E0680173
:10056000CC0CDD1CF601E00FF11FEA5DFC4E808132
:100570008068808377FC68C080E2E81682E0F80635
:100580000CF03FC08A8128E532E0281B310987FD45
:100590003395220F331F220F331F032E000C440B01
:1005A000550B898178E8872E912C881A910887FD50
:1005B0009394880C991C880C991C092C000CAA088F
:1005C000BB0860E070E0CB01F7FC0AC0B701653BF7
:1005D000710514F064EB70E0072E000C880B990B8A
:1005E000281939094A095B090E9484EF24EB30E09D
:1005F00040E050E00E94B5EF820E931EA41EB51E8F
:1006000074018BE08715D8F0298188E890E0821B7F
:10061000910927FD9395880F991F880F991FE81658
:10062000F906BCF402972FB7F894E601C00FD11F6A
:10063000CA5DDC4E880F991F9A8389832FBF62E3BE
:1006400070E080E090E09CD8CDB7DEB7EDE00C9490
:100650006CF02A8188E592E0821B910927FD939531
:10066000880F991F880F991FE816F906DCF6C70155
:10067000D9CFCF93DF93EB01682F70E08BE493E148
:1006800033DF688179818A819B81643F21E0720731
:100690008105910520F464EF71E080E090E070D86E
:1006A00080B182FB882780F9DF91CF910895A4E083
:1006B000B0E0EDE5F3E80C945BF08EEE92E0A0E0A4
:1006C000B0E089839A83AB83BC83BE016F5F7F4FA9
:1006D0008AE5CFDF2496E2E00C9477F0A4E0B0E066
:1006E000E4E7F3E80C945BF08EEE92E0A0E0B0E07B
:1006F00089839A83AB83BC83BE016F5F7F4F8AE09F
:10070000B8DF2496E2E00C9477F0A4E0B0E0EBE8E8
:10071000F3E80C945BF084EF91E0A0E0B0E0898313
:100720009A83AB83BC83BE016F5F7F4F8CE3A1DFF5
:100730002496E2E00C9477F0A4E0B0E0E2EAF3E87B
:100740000C945BF084EF91E0A0E0B0E089839A83A1
:10075000AB83BC83BE016F5F7F4F80EA8ADF249644
:10076000E2E00C9477F01F920F920FB60F921124D3
:100770000BB60F922F933F934F935F936F937F939B
:100780008F939F93AF93BF93EF93FF938091AF05A8
:1007900087FF27C010929500109294008091AF05BA
:1007A0008F5F8093AF058091AF05082E000C990BE9
:1007B00020914A132817190629F024F08091AF05DB
:1007C0008C30DCF1809194009091950004968034F7
:1007D0009C4908F47DC08091940090919500049606
:1007E00079C08091AF05082E000C990B20914A1317
:1007F0002817190699F294F2E091AF058E2FEE0FAB
:10080000990BFC01EE0FFF1FE80FF91FEA5DFC4E8C
:10081000808187FFC3CFE091AF058E2FEE0F990B3C
:10082000FC01EE0FFF1FE80FF91FEA5DFC4E80810F
:1008300060E08F770E94F1D0B1CF20919400309189
:100840009500E091AF058E2FEE0F990BFC01EE0F96
:10085000FF1FE80FF91FEA5DFC4E81819281820F34
:10086000931F9093990080939800E091AF058E2F8D
:10087000EE0F990BFC01EE0FFF1FE80FF91FEA5D69
:10088000FC4E808187FF11C0E091AF058E2FEE0FE7
:10089000990BFC01EE0FFF1FE80FF91FEA5DFC4EFC
:1008A000808161E08F770E94F1D0FF91EF91BF913D
:1008B000AF919F918F917F916F915F914F913F91F8
:1008C0002F910F900BBE0F900FBE0F901F90189599
:1008D00080E49CE990939900809398008FEF809337
:1008E000AF05E3CF9091C00095FFFCCF8093C60089
:1008F0000895CF93DF93EC018991882311F0F2DF03
:10090000FBCFDF91CF910895CF93DF93EC018991D5
:10091000882311F0E7DFFBCF8DE0E4DF8AE0E2DF40
:10092000DF91CF910895CF93DF93EC01FE01849185
:100930002196882311F0D6DFF9CFDF91CF9108956A
:100940000F931F93CF938C01C62F81EC9FE1EBDFB8
:10095000C801E9DF8AE3C6DF80E38C0FC3DF8AE0EA
:10096000C1DFCF911F910F910895CF92DF92EF9247
:10097000FF926A017B01D7DF42E0C701B6010E9406
:1009800036B6FF90EF90DF90CF900895CF93DF932E
:1009900068ED7FE10E942BC8C0915A13D0915B1380
:1009A000488159816A817B818FEC9FE1DEDF4C8138
:1009B0005D816E817F8189ED9DE2D7DF4091561385
:1009C00050915713609158137091591386ED9DE221
:1009D000CCDF8CEC9FE1A7DF86EC9FE1A4DF8AE00F
:1009E00081DFDF91CF910895C0DF8AE07BCFADE555
:1009F000B0E0EDEFF4E80C944BF070E060E085E4DB
:100A00000E94296E7C01182F8F3FB1F1882341F09D
:100A10008BEB91E288DFC35ADF4FE2E10C9467F081
:100A20006EEB70E083E50E94296E5C0165E070E08A
:100A300083E40E94296E6C0160E085E50E94156EDA
:100A40002C968FAF2C9760E08EEA91E20E949E5C1C
:100A50000E94D6D169877A878B879C871F3F09F0D0
:100A600067C434E7A316B1040CF489C183E891E2AA
:100A70005ADF0E94AFC8CFCF6CE370E0D3CF20E045
:100A800030E040E05EE32BAF3CAF4DAF5EAFABC1BB
:100A90002AE939E949E15FE323962CAF3DAF4EAF38
:100AA0005FAF2397ADC14090AE125090AF126090EF
:100AB000B0127090B11251C22B96EEADFFAD2B97D4
:100AC0004083A4C24BEEC42ED12CE12CF12C22C3C6
:100AD00084E190E0A0E0B0E08D879E87AF87B88B7F
:100AE00034E1C32ED12CE12CF12C24C3CD86DE863B
:100AF000EF86F88A1FC32B96EEADFFAD2B97808350
:100B0000E9C3D501C4012EA53FA548A959A9821B57
:100B1000930BA40BB50BB7FD47C02D968FAD2D974A
:100B20000E9439288AE0DEDED501C4018053984F47
:100B3000AF4FBF4F8EA79FA7A8ABB9AB9AA9911192
:100B40006FC02BA93CA94DA95EA9C301B2010E94A7
:100B5000E6F118160CF050C020E030E040E050E420
:100B6000C301B2010E9483F06BAB7CAB8DAB9EAB3B
:100B70002AA53BA54CA55DA5280D391D4A1D5B1D69
:100B80002FAB38AF49AF5AAF6D966CAD7DAD8EAD22
:100B90009FAD6D970E946BE9A30192010E9465E9E8
:100BA000881F8827881F8AAB89859A85AB85BC8575
:100BB000898F9A8FAB8FBC8F29893A894B895C8941
:100BC000281739074A075B0720F4298F3A8F4B8F84
:100BD0005C8F898D9A8DAB8DBC8D881A990AAA0A73
:100BE000BB0A91E889169FE4990692E1A906B1042F
:100BF00060F187EA90E22DC2D501C4012FA938AD7A
:100C000049AD5AAD821B930BA40BB50B47EF52E1D4
:100C100066E073E1B7FDC8CF812F0E948029C4CF61
:100C200069966CAD7DAD8EAD9FAD69970E946BE905
:100C30009B01AC01C301B2010E9465E987FFB4CFFB
:100C400044E353E164E473E1E7CF2996AEADBFAD71
:100C50002997A215B3050CF08FC0B3E02B16310411
:100C60000CF48AC08AE490E25EDE1F3F09F066C0A1
:100C7000EAE3F0E2FE83ED8389E290E254DE8D81C7
:100C80009E8151DE49815A816B817C8186E490E2AC
:100C9000ABDE89E290E247DE8D819E8144DE4D8DA0
:100CA0005E8D6F8D78A182E490E29EDE89E290E213
:100CB0003ADE8D819E8137DE49A15AA16BA17CA1CC
:100CC0008EE390E291DE2C963FAD2C97332309F40E
:100CD000D0CE2CEA35EC47E25EE36D8D7E8D8F8DB4
:100CE00098A10E94CAE96B017C0120E030E543EC49
:100CF00050E469A17AA18BA19CA10E94CAE9298133
:100D00003A814B815C811F3FF1F420933707309388
:100D100038074093390750933A07C0923B07D09267
:100D20003C07E0923D07F0923E0760933F077093C7
:100D3000400780934107909342079BCE29E23DE212
:100D40003E832D8399CF2093B5123093B6124093F2
:100D5000B7125093B812C092B912D092BA12E09260
:100D6000BB12F092BC126093BD127093BE128093BE
:100D7000BF129093C0127DCE0E946F71CEC08FE6DD
:100D800091E2D1DD0E94E2288FE7809336072CE3C1
:100D900030E0C9A6A8EEB3E00E94E1EF6AA77BA706
:100DA0008CA79DA729853A854B855C85260F371F23
:100DB000481F591F2FAB38AF49AF5AAF81E080931E
:100DC000690160E08BE591E20E949E5C02E00E0DFD
:100DD000023008F054CE8BEA9AEAAAEABEE38BAF5F
:100DE0009CAFADAFBEAF023008F052CE8DEC9CECA4
:100DF000ACE4BEE323968CAF9DAFAEAFBFAF2397FD
:100E0000023008F4E12C2D96EFAE2D9789859A8556
:100E1000AB85BC85898B9A8BAB8BBC8B8EA79FA730
:100E2000A8ABB9AB19A21AA21BA21CA21D8E1E8EC2
:100E30001F8E18A219821A821B821C822FE730E0B3
:100E400040E050E02D873E874F87588B80E090E44C
:100E5000ACE1B6E48D839E83AF83B8871D8A1E8A7A
:100E60001F8A188EFFE7CF2ED12CE12CF12C1AAA65
:100E70001BAA1CAA1DAA1EAA1DA21EA21FA218A65A
:100E800091E024969FAF2497312C212C412C512C9A
:100E9000320195010B2C000C440B550B61962CAFC5
:100EA0003DAF4EAF5FAF619749A5042E000C550BC7
:100EB00029965FAF4EAF299757E11502C001112463
:100EC000DC01AC54BD4E2B96BFAFAEAF2B97C50126
:100ED0004E969C01092E000C440B550B65962CAFC9
:100EE0003DAF4EAF5FAF6597CC979C01990F440B18
:100EF000550B69962CAF3DAF4EAF5FAF699736E0AB
:100F0000A31AB108C5010B2C000CAA0BBB0B6D96E4
:100F10008CAF9DAFAEAFBFAF6D9780916901882355
:100F200009F498C00E94D6D14B015C0190919D03B9
:100F30006E969FAF6E97992309F47BC00E945B2A3F
:100F400010929D031F3F09F0AECD409030075090A6
:100F500031076090320770903307A30192016D89C9
:100F60007E898F89988D0E94E6F187FF04C04D8AA3
:100F70005E8A6F8A788EA30192016D817E818F8156
:100F800098850E9465E9181624F44D825E826F826E
:100F9000788661966CAD7DAD8EAD9FAD61970E94F8
:100FA0006BE9698F7A8F8B8F9C8F2496AFAD2497D6
:100FB000AA2309F454C09B01AC01C301B2010E94F1
:100FC000E6F11816B4F5D501C40129893A894B898F
:100FD0005C89821B930BA40BB50BAC01BD01485877
:100FE00053416109710977FD24C04D855E856F8588
:100FF00078894C195D096E097F0975956795579534
:1010000047951F3F09F058CD409336078DA39EA307
:10101000AFA3B8A7298D3A8D4B8D5C8D2D8B3E8B60
:101020004F8B588F89869A86AB86BC8624961FAED6
:10103000249765966CAD7DAD8EAD9FAD65970E9492
:101040006BE9A30192010E9465E987FF5ACD85EC07
:1010500090E269DC109269010E94E2280ACD298D94
:101060003A8D4B8D5C8DC301B2010E9465E987FF0B
:10107000E0CFD501C40129853A854B855C85821B6B
:10108000930BA40BB50BAC01BD014858534161094A
:10109000710977FDCECF2114310409F40AC12DA1C5
:1010A0003EA14FA158A5280F391F4A1F5B1F298B4E
:1010B0003A8B4B8B5C8B2DA13EA14FA158A5281BD1
:1010C000390B4A0B5B0BC701B6010E9484EF2989DB
:1010D0003A894B895C890E94B5EFCD84DE84EF8428
:1010E000F888C20ED31EE41EF51E34E1C316D104E7
:1010F000E104F1040CF4ECCC4CEEC416D104E10490
:10110000F1040CF0DFCC50E8C516D104E104F10481
:101110000CF4ECCCCD86DE86EF86F88A8EEF90E07C
:10112000A0E0B0E09C01AD012C193D094E095F091A
:1011300069017A0183E591E2F6DB6D857E858F8515
:1011400098890E9457768EE491E2EDDBC701B601E3
:101150000E9457764D815E816F81788587E491E2A8
:1011600004DC4D895E896F89788D80E491E2FDDB36
:1011700093E0291631040CF49CC0C701B6010E940B
:101180006BE920E030E040E850E40E94CAE969835E
:101190007A838B839C832D813E814F8158856D8915
:1011A0007E898F89988D0E9482F02BED3FE049EC7B
:1011B0005FE30E94CAE99B01AC0169817A818B815E
:1011C0009C810E94FAF027966CAF7DAF8EAF9FAFE7
:1011D000279769897A898B899C890E946BE92FE618
:1011E00032E143E85AE30E94CAE96D837E838F832C
:1011F000988723962CAD3DAD4EAD5FAD23972796D6
:101200006CAD7DAD8EAD9FAD27970E94CAE9698315
:101210007A838B839C839B01AC010E9483F02D8198
:101220003E814F8158850E94FAF06D8F7E8F8F8F9F
:1012300098A32BAD3CAD4DAD5EAD6D817E818F81B0
:1012400098850E94CAE929813A814B815C810E947C
:10125000CAE969A37AA38BA39CA327964CAD5DAD85
:101260006EAD7FAD27978AE391E27FDB4D815E8192
:101270006F81788584E391E2B7DB85E291E2023009
:1012800010F086E191E24FDB49815A816B817C81CC
:1012900080E191E26ADB4D8D5E8D6F8D78A18AE0F1
:1012A00091E263DB49A15AA16BA17CA184E091E2A8
:1012B0009BDB8D859E85AF85B8898C0D9D1DAE1DF0
:1012C000BF1DB595A795979587951F3F09F013CC3E
:1012D000809336072996FFAD2997FF9329A52F9371
:1012E0003F922F9280EF90E29F938F938BEF90E24B
:1012F0009F938F931F920E94815C3FEF231A330AC2
:101300000FB6F894DEBF0FBECDBF898D9A8DAB8D21
:10131000BC8D8D839E83AF83B887898A9A8AAB8A76
:10132000BC8A6E969FAD6E9724969FAF249781CE10
:101330008E2C0E2C000C9908F40183E0EE0FFF1F99
:101340008A95E1F7EF59FE4F868197810F978A15AD
:101350009B050CF48BCB8FE691E2E5DA0E94E22844
:1013600087E1889DF001899DF00D1124E655FD4E21
:101370008FE7828724E130E00CCDCF93DF936AE1E1
:1013800079E10E942BC8CCE2D7E04B855C856D8566
:101390007E8581E199E1E9DA20E030E543EC50E433
:1013A0006F85788989899A890E94CAE9AB01BC0155
:1013B0008EE099E1DADA2CEA35EC47E25EE36B89FC
:1013C0007C898D899E890E94CAE9AB01BC018BE0B2
:1013D00099E10ADBDF91CF9108956CE978E10E94F1
:1013E0002BC86091790D70917A0D80917B0D909151
:1013F0007C0D0E9469E9AB01BC0183E998E1B5DA93
:101400004091A90D5091AA0D6091AB0D7091AC0D5A
:1014100080E998E1AADA4091AD0D5091AE0D60914E
:10142000AF0D7091B00D8DE898E19FDA40918B0778
:1014300050918C0760918D0770918E078AE898E132
:10144000D3CACF93DF9360E478E10E942BC8C9E64A
:10145000DDE04CA95DA96EA97FA987E398E185DA53
:1014600048AD59AD6AAD7BAD84E398E17EDA4CAD11
:101470005DAD6EAD7FAD8DE898E1B6DADF91CF91CD
:101480000895CF93DF936CE178E10E942BC8C9E601
:10149000DDE04CA15DA16EA17FA183E198E165DA59
:1014A00048A559A56AA57BA589ED9DE25EDA4CA504
:1014B0005DA56EA57FA586ED9DE257DA48A959A9DD
:1014C0006AA97BA983ED9DE28FDADF91CF91089520
:1014D000CF93DF9367EF77E10E942BC8C9E6DDE089
:1014E000688179818A819B810E9469E9AB01BC0195
:1014F0008EEE97E13ADA6C817D818E819F810E9428
:1015000069E9AB01BC0189ED9DE22FDA6885798537
:101510008A859B850E9469E9AB01BC0186ED9DE24D
:1015200024DA6C857D858E859F850E9469E9AB01F3
:10153000BC0183ED9DE258DADF91CF9108958F923F
:101540009F92AF92BF92EF92FF920F931F93CF9310
:10155000DF9387E596E1E7D9C0E0D7E0D15019F0F5
:1015600080E2C0D9FBCF8C2F0E94C56DCF5FC73002
:10157000A1F78AE0B7D908EB12E0C0E080E2B2D967
:101580008C2F0E94C56D7801D7E080E2ABD9F701BE
:1015900080809180A280B38020E030E0A901C50165
:1015A000B4010E94E6F187FD02C08BE29BD943E0C3
:1015B000C501B4010E9436B6D150FCE1EF0EF11C1A
:1015C000D111E3CF8AE08ED9CF5F0C5F1F4FC730B8
:1015D000A9F68AE087D9DF91CF911F910F91FF90F3
:1015E000EF90BF90AF909F908F900895811105C0AC
:1015F00080E596E198D98AE075C984E596E1FACF4D
:1016000089E496E190C983E496E18DC9CF9384E59E
:101610000E94796AC0E08823D9F00E94EB6DC82F40
:101620001816B4F4F0DF8DE45DD980912406909112
:1016300025060E94E57B86EE99E175D96C2FCC0FCB
:10164000770B880B990B0E94ECB38AE04BD9CFEF54
:101650008C2FCF910895CF93C82F60E079E10E943D
:1016600014C8C11101C0CFDF4091B5125091B6121C
:101670006091B7127091B81287EF98E176D920E0A7
:1016800030E543EC50E46091B9127091BA12809148
:10169000BB129091BC120E94CAE9AB01BC0184EF5D
:1016A00098E163D92CEA35EC47E25EE36091BD1224
:1016B0007091BE128091BF129091C0120E94CAE92F
:1016C000AB01BC0181EF98E150D98AE00BD9CF91F1
:1016D0000895B0E0A0E0EFE6FBE80C9455F061E07F
:1016E00083E50E94156EC1E0C82769ED79E18C2F72
:1016F0000E9414C8C11101C086DF81ED99E113D9A0
:1017000086EC9FE110D98AE0EDD86FEB79E18C2F60
:101710000E9414C8C11101C076DF82EA99E103D9A1
:101720008C2F0E9434C88C2FACDE8C2FD1DE8C2FF6
:1017300088DE8C2F52DE66E579E18C2F0E942BC863
:10174000D091B3028DE499E1EED86D2F70E090E076
:1017500080E00E94ECB34091B4025091B5026091D8
:10176000B6027091B70286ED9DE2FFD880E499E160
:10177000DAD88091B3023ADF20E030E0A90160912D
:1017800084037091850380918603909187030E9462
:1017900065E9882379F188EBE82E82E0F82E10E0E5
:1017A000670100E0C11101C02EDF88E999E1BBD8D3
:1017B000802F0E94C56D85E999E1B5D8812F0E94DF
:1017C000C56D86ED9DE2AFD8F601608171818281A1
:1017D000938145E00E9436B68AE084D80F5FFCE131
:1017E000CF0ED11C0730F1F61F5F84E0E80EF11C2C
:1017F0001730B1F66AE779E18C2F0E9414C803E430
:1018000017E0D0E0C11101C0FEDE81E799E18BD87D
:101810008D2F0E94C56DF80160817181072E000C2B
:10182000880B990B0E946BE9AB01BC018EE699E134
:101830009CD8F80162817381072E000C880B990BEC
:101840000E946BE9AB01BC018BE699E18ED8F801EF
:10185000E480F58088E699E166D8C7010E94E57BBF
:101860008AE040D80A5F1F4FD13059F48C2FF3DE45
:101870008C2F83DD8C2F8AD8CDB7DEB7E8E00C94AF
:1018800071F0D1E0BFCFACE1B0E0E9E4FCE80C944A
:101890004BF083E50E94026A182F882309F41CC1CB
:1018A0000E94066E8D838091750190917601A091C2
:1018B0007701B0917801898F9A8FAB8FBC8F20917F
:1018C000790130917A0140917B0150917C012D8BFF
:1018D0003E8B4F8B588F80917D0190917E01A0911E
:1018E0007F01B09180018D879E87AF87B88B1123D0
:1018F00031F09D81911103C080E00E940A7A8091AD
:101900001E0690911F06A0912006B091210635E198
:10191000B695A795979587953A95D1F79C01AD0116
:10192000217033274427552729873A874B875C87BF
:1019300020E030E0A90160918403709185038091DB
:101940008603909187030E9465E9882309F4C8C043
:1019500083E40E94026A882309F493C00E94356ED2
:10196000698B7A8B8B8B9C8B48EB52E05F834E8329
:101970008A0157E05887412C512C98EC692E92EC43
:10198000792E812C912C28ECA22E22E4B22E312C1F
:10199000212CF101EE0FFF1FEE0FFF1FE00FF11FD3
:1019A000C080D180E280F380A7019601C501B40117
:1019B0000E9465E9181614F446015701A701960123
:1019C000C301B2010E94E6F187FF02C02601370180
:1019D0008FEF281A380A97E029163104D1F6A88526
:1019E000A150A887045E1F4FA111D1CFA30192017E
:1019F000C501B4010E9483F020E030E040E05FE3E5
:101A00000E94CAE929893A894B895C890E9483F03E
:101A10004B015C012DEB37E346E855EB0E9465E98D
:101A200087FD0AC02DEB37E346E855E3C501B40155
:101A30000E94E6F118162CF580E00E940A7A17E061
:101A4000EE80FF8007E0F7016191719181919191A2
:101A50007F016F01F4E0CF1AD108A50194010E9423
:101A600082F0D6016D937D938D939C9313970150D3
:101A700051F71150EE81FF817C96FF83EE831111A7
:101A8000DFCF89859A85AB85BC85892B8A2B8B2BEB
:101A900079F020E030E0A901609184037091850322
:101AA00080918603909187030E9465E9811147DD4B
:101AB0008AE50E94026A882359F00E94356E698384
:101AC0007A838B839C8360E0CE0101960E94967A94
:101AD0008D810E940A7A14C02091B3022D83E3CE37
:101AE000FD81F11108C029853A854B855C85232B42
:101AF000242B252BE9F287DD89E297E10E9493846C
:101B00009D81992349F08091B302811105C078DD50
:101B10008AE097E10E94938476DD8CEF96E10E9443
:101B200093848091B30262DD6EDD8FEE96E10E94B8
:101B30009384C090B402D090B502E090B602F090C9
:101B4000B70220E030E0A901C701B6010E94E6F12A
:101B500018160CF040C042E0C701B6010E9436B62C
:101B60008DE00E9472848AE00E947284298D3A8DF1
:101B70004B8D5C8D6091750170917601809177013C
:101B8000909178010E9465E981111FC02D893E89DD
:101B90004F89588D6091790170917A0180917B0114
:101BA00090917C010E9465E981110FC020917D0117
:101BB00030917E0140917F01509180016D857E853D
:101BC0008F8598890E9465E981110E94E1406C9699
:101BD000E2E10C9467F08AEE96E10E949384C6CF0E
:101BE000CF93DF93EB010E949384BE01DD0F880B3E
:101BF000990B0E94ECB3DF91CF9108950E94E228E7
:101C00000E94664580912707813099F0F9DC8CECC1
